:020000040000FA
:1000000000800020110500008D0500008F05000014
:100010009105000093050000950500000000000018
:100020000000000000000000000000009705000034
:1000300099050000000000009B050000B13F000092
:100040009F050000A3050000A7050000AB05000008
:10005000AF050000B3050000B7050000BB050000B8
:10006000BF050000C3050000C7050000CB05000068
:10007000CF050000D3050000D7050000DB05000018
:10008000DF050000E3050000E7050000EB050000C8
:10009000EF050000F3050000F7050000FB05000078
:1000A000FF05000003060000070600000B06000025
:1000B0000F06000013060000890500001706000067
:1000C0001B0600001F060000230600002706000094
:1000D000890500002B0600002F06000033060000F3
:1000E000370600003B060000890500003F060000BF
:1000F00043060000470600004B0600004F060000C4
:100100008905000053060000570600005B0600004A
:100110005F06000063060000670600006B06000033
:100120006F06000073060000770600007B060000E3
:100130007F06000083060000870600008B06000093
:100140008F06000093060000970600009B06000043
:100150009F060000A3060000A7060000AB060000F3
:10016000AF060000B3060000B7060000BB060000A3
:10017000BF060000C3060000C7060000CB06000053
:10018000CF060000D3060000D7060000DB06000003
:10019000DF060000E3060000E7060000EB060000B3
:1001A000EF060000F3060000F7060000FB06000063
:1001B000FF06000003070000070700000B07000010
:1001C0000F07000013070000170700001B070000BF
:1001D0001F07000023070000270700002B0700006F
:1001E0002F07000033070000370700003B0700001F
:1001F0003F07000043070000470700004B070000CF
:100200004F07000053070000570700005B0700007E
:100210005F07000063070000670700006B0700002E
:100220006F07000073070000770700007B070000DE
:100230007F07000083070000870700008B0700008E
:100240008F07000093070000970700009B0700003E
:100250009F070000A3070000A7070000AB070000EE
:10026000AF070000B3070000B7070000BB0700009E
:10027000BF070000C3070000C7070000CB0700004E
:10028000CF070000D3070000D7070000DB070000FE
:10029000DF070000E3070000E70700008905000012
:1002A0008905000089050000EB070000EF0700004A
:1002B000F3070000F7070000FB070000FF0700003E
:1002C00003080000070800000B0800000F080000EA
:1002D00013080000170800001B0800001F0800009A
:1002E00023080000270800002B0800002F0800004A
:1002F00033080000370800003B0800003F080000FA
:1003000043080000470800004B0800004F080000A9
:1003100053080000570800005B0800005F08000059
:1003200063080000670800006B0800006F08000009
:1003300073080000770800007B0800007F080000B9
:1003400083080000870800008B0800008F08000069
:1003500093080000970800009B0800009F08000019
:10036000A3080000A7080000AB080000AF080000C9
:10037000B308000000A0F0F700A0F0F700A0F0F72D
:1003800000A0F0F700A0F0F700A0F0F700A0F0F751
:1003900000A0F0F700A0F0F700A0F0F700A0F0F741
:1003A00000A0F0F700A0F0F700A0F0F700A0F0F731
:1003B00000A0F0F700A0F0F700A0F0F700A0F0F721
:1003C00000A0F0F700A0F0F700A0F0F700A0F0F711
:1003D00000A0F0F700A0F0F700A0F0F700A0F0F701
:1003E00000A0F0F700A0F0F700A0F0F700A0F0F7F1
:1003F00000A0F0F700A0F0F700A0F0F700A0F0F7E1
:10040000FFFFFFFFFFFFFFFFFFFFFFFFFE7FFFFF7D
:100410005830315F50423033355F535750425F3070
:100420003030302E303030312E30300000000000BF
:100430004D6172203139203230323400000000002A
:1004400031303A32353A313400000000000000000B
:10045000303030303030303030303030000000005C
:10046000000000000000000000000000000000008C
:10047000000000000000000000000000000000007C
:1004800000000000000000000C0000002000000040
:10049000000000000000000000000000000000005C
:1004A000000000000000000000000000000000004C
:1004B000000000000000000000000000000000003C
:1004C000000000000000000000000000000000002C
:1004D000000000000000000000000000000000001C
:1004E000000000000000000000000000000000000C
:1004F00000000000000000000000000000000000FC
:1005000000000000000000000000000000000000EB
:1005100072B61348134901600A6882F308881249C9
:10052000124A521A013A05DD0020042308601944DA
:10053000043AFBDA0E490F4A0F4B9A42BEBF51F8FC
:10054000040B42F8040BF8E70C490D4A00209142D5
:10055000BCBF41F8040BFAE762B60A480047000046
:1005600008ED00E00000000000100020FF7F0020E8
:10057000C4560000001000200C11002010110020B3
:10058000E8440020FD0F0000FFF7FEBFFEE7FEE796
:10059000FEE7FEE7FEE7FEE7FEE7FEE7FEE7C6480A
:1005A0000047C6480047C6480047C6480047C648F7
:1005B0000047C6480047C6480047C6480047C648E7
:1005C0000047C6480047C6480047C6480047C648D7
:1005D0000047C6480047C6480047C6480047C648C7
:1008B0000047C64800470000890500008905000080
:1008C00089050000890500008905000089050000F0
:1008D00089050000890500008905000089050000E0
:1008E00089050000890500008905000089050000D0
:1008F000890500008905000089050000AD1700008A
:10090000D117000089050000891100008905000049
:10091000890500008905000089050000413B0000B1
:10092000473B00004D3B0000593B0000533B00009B
:100930005F3B0000653B00006B3B0000773B000025
:10094000713B00007D3B0000833B0000893B0000C1
:10095000953B00008F3B00009B3B0000A13B00004B
:10096000A73B0000B33B0000AD3B00008905000041
:10097000890500008905000089050000890500003F
:1009800089050000613200006F3200007D320000F6
:100990008B32000099320000A7320000B53200000F
:1009A000C3320000D1320000DF320000ED3200001F
:1009B000FB3200000933000017330000253300002C
:1009C00033330000413300004F3300005D3300003B
:1009D0006B3300007933000087330000953300004B
:1009E000A3330000B1330000BF330000CD3300005B
:1009F000DB330000E9330000F7330000053400006A
:100A000013340000213400002F3400003D34000076
:100A10004B34000059340000673400007534000086
:100A200083340000913400009F340000AD34000096
:100A3000BB340000C9340000D7340000E5340000A6
:100A4000F3340000013500000F3500001D350000B3
:100A50002B350000393500004735000055350000C2
:100A600063350000713500007F3500008D350000D2
:100A70009B350000A9350000B7350000C5350000E2
:100A8000D3350000E1350000EF350000FD350000F2
:100A90000B360000193600002736000035360000FE
:100AA00043360000513600005F3600006D3600000E
:100AB0007B3600008936000097360000A53600001E
:100AC000B3360000C1360000CF360000DD3600002E
:100AD000EB360000F936000007370000153700003C
:100AE00023370000313700003F3700004D3700004A
:100AF0005B3700006937000077370000853700005A
:100B00009337000089050000890500008905000071
:100B1000890500008905000089050000890500009D
:100B2000890500008905000089050000890500008D
:100B3000890500008905000089050000890500007D
:100B4000890500008905000089050000890500006D
:100B5000890500008905000089050000351900009D
:100B60003B19000041190000471900004D19000011
:100B7000890500008905000089050000890500003D
:100B8000890500008905000089050000890500002D
:100B90008905000089050000611200008905000038
:100BA000890500008905000089050000890500000D
:100BB00089050000890500008905000069380000EA
:100BC0006F380000890500008905000089050000D4
:100BD000844641EA000313F003036DD1403A41D348
:100BE00051F8043B40F8043B51F8043B40F8043B07
:100BF00051F8043B40F8043B51F8043B40F8043BF7
:100C000051F8043B40F8043B51F8043B40F8043BE6
:100C100051F8043B40F8043B51F8043B40F8043BD6
:100C200051F8043B40F8043B51F8043B40F8043BC6
:100C300051F8043B40F8043B51F8043B40F8043BB6
:100C400051F8043B40F8043B51F8043B40F8043BA6
:100C500051F8043B40F8043B51F8043B40F8043B96
:100C6000403ABDD2303211D351F8043B40F8043B36
:100C700051F8043B40F8043B51F8043B40F8043B76
:100C800051F8043B40F8043B103AEDD20C3205D346
:100C900051F8043B40F8043B043AF9D2043208D03E
:100CA000D2071CBF11F8013B00F8013B01D30B88B0
:100CB00003806046704700BF082A13D38B078DD08E
:100CC00010F003038AD0C3F10403D21ADB071CBF60
:100CD00011F8013B00F8013B80D331F8023B20F8CA
:100CE000023B7BE7043AD9D3013A11F8013B00F803
:100CF000013BF9D20B7803704B7843708B7883708B
:100D00006046704753B94AB9002908BF00281CBF84
:100D10004FF0FF314FF0FF3000F06EB9ADF1080C2D
:100D20006DE904CE00F006F8DDF804E0DDE9022309
:100D300004B070472DE9F047089D04468C46002B0F
:100D400040F083808A42174647D9B2FA82F242B114
:100D5000C2F1200024FA00F09140974040EA010CD3
:100D600094404FEA1748230CBCFBF8F61FFA87FEA5
:100D700008FB16C143EA014306FB0EF1994209D96B
:100D8000FB1806F1FF3080F01981994240F216817C
:100D9000023E3B445B1AA4B2B3FBF8F008FB1033ED
:100DA00044EA034400FB0EFEA64509D93C1900F1B4
:100DB000FF3380F00581A64540F2028102383C44B1
:100DC00040EA0640A4EB0E0400261DB1D4400023E7
:100DD000C5E900433146BDE8F08702B9FFDEB2FA4B
:100DE00082F2002A50D1CB1B4FEA174E1FFA87F828
:100DF0000126B3FBFEFC210C0EFB1C3341EA034130
:100E000008FB0CF38B4207D979180CF1FF3002D2A2
:100E10008B4200F2E9808446C91AA3B2B1FBFEF00E
:100E20000EFB101143EA014408FB00F8A04507D966
:100E30003C1900F1FF3302D2A04500F2D9801846D8
:100E4000A4EB080440EA0C40BFE78B4209D9002D0F
:100E500000F0B1800026C5E9000130463146BDE80A
:100E6000F087B3FA83F6002E4AD18B4202D3824236
:100E700000F2B880841A61EB030101208C46002D3A
:100E8000A8D0C5E9004CA5E7C2F1200320FA03F67B
:100E9000974001FA02F04FEA174ED9403043030C55
:100EA000B1FBFEF61FFA87F80EFB161143EA014369
:100EB00006FB08F1994204FA02F409D9FB1806F17D
:100EC000FF3C80F08D80994240F28A80023E3B4494
:100ED0005B1A81B2B3FBFEF00EFB103341EA034113
:100EE00000FB08F38B4207D9791800F1FF3C73D25D
:100EF0008B4271D902383944CB1A40EA064678E76A
:100F0000C6F1200C03FA06F422FA0CF31C4320FA73
:100F10000CF701FA06F34FEA144E21FA0CF11F43C5
:100F20003B0CB1FBFEF91FFA84F80EFB191143EAE2
:100F3000014109FB08FA8A4502FA06F200FA06F3B3
:100F400008D9611809F1FF3048D28A4546D9A9F17C
:100F500002092144A1EB0A01BFB2B1FBFEF00EFB76
:100F6000101147EA014700FB08F8B84507D9E7190F
:100F700000F1FF312ED2B8452CD90238274440EA7F
:100F80000940A7EB0807A0FB02894F45C646494622
:100F90001AD317D05DB1B3EB0E0267EB010707FA66
:100FA0000CFCF2404CEA0202F740C5E9002700269B
:100FB0003146BDE8F0872E4628460BE70646E9E6AF
:100FC0001846FDE64345E5D2B8EB020E69EB040195
:100FD0000138DFE70846D2E760468DE78146B9E78A
:100FE000664675E730464AE7ACF1020C394413E730
:100FF00002383C4424E700BF704700BF08B503F047
:1010000047F9002008BD00F061B800F043B801B90D
:101010004008C301421143EAD01302F00202134315
:10102000C21002F004021343421002F008021343FC
:10103000420002F010021343C20002F020024001FD
:10104000134300F040001843C0B2704730B5037836
:10105000087840EA432085B040F4807085B20021D2
:10106000C0F307200192FFF7D2FF01210446E8B246
:10107000FFF7CDFF40EA042040F48070ADF80E0089
:10108000019A01230DF10E01002002F0B7FF05B017
:1010900030BD000013B50C4C00230DF10602611C9D
:1010A0002046ADF80630FFF7D1FF0DF10602E11C36
:1010B000A01CFFF7CBFF0DF10602611D201DFFF7FD
:1010C000C5FF02B010BD00BF0010002073B50E4672
:1010D0001C4611460546E8B930784000294600F024
:1010E000FE00FFF794FF0002ADF806000123224640
:1010F0000DF10601284602F081FF01210546207806
:101100002688FFF784FF26F0FF0606432680284640
:1011100002B070BD1A463046FFF798FF0546F6E765
:1011200082B00023084A01939368DB0102D50020B6
:1011300002B07047019BB3F5801F03D2019B0133BE
:101140000193F1E70120F3E70020054072B607B4F0
:1011500003480449044A0160026007BC62B6704754
:1011600014200540C4A1D9B00F3B1E1A08B5FFF7E3
:10117000EDFF044B9A686FF300029A60BDE80840E7
:10118000FFF7CEBF0020054008B5034B1B6803B135
:101190009847BFF34F8F08BD10110020094BDA6943
:1011A000002ABCBF4FF0B642DA61DA6960F341024F
:1011B000DA61DA6942F00102DA61DA6942F000428A
:1011C000DA61704700400640124BDA6A002ABCBF61
:1011D0004FF0B642DA62DA6A417861F31242DA62BB
:1011E000DA6A017861F30102DA62DA6A017961F39D
:1011F0000F22DA62DA6A417A61F30412DA62DA6A99
:10120000017A61F34512DA62DA6A42F00042DA6288
:10121000704700BF00400640074B5A69002ABCBF18
:101220004FF0B6425A615A696FF349225A615A69BE
:1012300042F000425A61704700400640074BDA69AD
:10124000002ABCBF4FF0B642DA61DA696FF3492277
:10125000DA61DA6942F00042DA6170470040064024
:1012600008B51A4B5A69510311D55A69002ABCBFF7
:101270004FF0B6425A615A6942F480225A615A6963
:1012800042F000425A61124B1B68CBB198470F4B9A
:10129000DA69520311D5DA69002ABCBF4FF0B642B1
:1012A000DA61DA6942F48022DA61DA6942F00042F6
:1012B000DA61074B5B6833B19847BFF34F8F08BDC6
:1012C000FFF7AAFFE3E7FFF7B9FFF6E700400640A4
:1012D000141100208C2800F280806B281FD8482829
:1012E00075D82B286AD8282800F284800B286BD860
:1012F000042801D008287DD1544B800853F82030B1
:101300001A68002ABCBF4FF0B6421A601A6861F32F
:101310000B221A601A6842F000421A607047A0F16E
:101320006C03202B66D801A252F823F0F9120000BA
:10133000F5130000F5130000F5130000F91200008A
:10134000F5130000F5130000F5130000F91200007A
:10135000F5130000F5130000F5130000F91200006A
:10136000F5130000F5130000F5130000F91200005A
:10137000F5130000F5130000F5130000F91200004A
:10138000F5130000F5130000F5130000F51300003D
:10139000F71300001B14000035140000F9120000C0
:1013A000F5130000F5130000F5130000F91200001A
:1013B000012202FA03F313F0113F1AE0A0F12C030B
:1013C000DAB201239340F6E7A0F10C03F8E7A0F1AD
:1013D0004C03DBB21C2BEBD97047A0288CD000F15A
:1013E0005003DBB2102B05D8012202FA03F3184A8E
:1013F000134281D17047174BDA68002ABCBF4FF007
:10140000B642DA60DA6822F4706242EA0121D960F9
:10141000DA6842F00042DA60ECE70E4BDA68002A44
:10142000BCBF4FF0B642DA60DA6822F0F00242EA5E
:101430000111ECE7074BDA68002ABCBF4FF0B64257
:10144000DA60DA6822F00F021143E0E7C44E0000D0
:1014500011110100004006408208504B82B053F841
:10146000223080284FF000028DF8072059D86328D9
:101470000BD840283ED8232823D80438C0B21C28D3
:101480002CD901238DF8073017E06438C0B201224F
:1014900002FA00F010F0113FF3D01A68002ABCBF26
:1014A0004FF0B6421A6001295BD11A6861F3061247
:1014B0001A601A6842F000421A609DF8070002B0F4
:1014C000704724380122C0B202FA00F000F0113255
:1014D00022F01102F2B910F0110FDDE7012202FA39
:1014E00000F000F0113222F00102002AD5D110F0F4
:1014F000010F27E04438C0B21C28C2D8012202FAEA
:1015000000F000F0113222F01102002AC5D110F0D3
:10151000110FB6D01A68002ABCBF4FF0B6421A604D
:1015200021E0A0282BD004D800F0FB008828A8D107
:1015300009E05030C0B21028A3D8012202FA00F00E
:10154000174A10429DD01A68002ABCBF4FF0B6421D
:101550001A600129A9D00229A7D00329A5D00429FE
:1015600006E00229A1D003299FD004299DD0052996
:101570009BD0002999D001228DF8072099E71A689D
:10158000002ABCBF4FF0B6421A6003298DD004294F
:101590008BD0052989D00629EAE700BFC44E000098
:1015A0001111010082B000230138019304283FD8B3
:1015B000DFE800F033271B0F0300204A2049936A1D
:1015C000DB032FD4019B8B4232D8019B0133019363
:1015D000F5E71A4A1A495369D80323D4019B8B4271
:1015E00026D8019B01330193F5E7144A1449D369C6
:1015F000D80317D4019B8B421AD8019B0133019366
:10160000F5E7104A104913689B050BD4019B8B42E8
:101610000ED8019B01330193F5E70C4A0849536842
:101620005B0702D5002002B07047019B8B4201D9B5
:101630000120F8E7019B01330193F0E700400640E9
:10164000A086010000900740404B4C0000D00740AE
:1016500010B5154CA36A002BBCBF4FF0B643A36274
:10166000A36A43F40073A362A36A60F34103A36215
:10167000A36A43F00103A362A36A43F00043A36299
:101680000520FFF78FFF70B94FF0B643A362A36A3E
:1016900043F00073A362A36A60F34923A362A36AC1
:1016A00043F00043A36210BD0040064010B4174B46
:1016B0009C69002CBCBF4FF0B6449C619C6960F3F0
:1016C00082049C61986962F3000098619A6942F013
:1016D00002029A619A6942F000429A615A69002AAC
:1016E000BCBF4FF0B6425A61084B5A6961F34102E0
:1016F0005A615A6942F001025A615A6942F0004245
:101700005A615DF8044B0420FFF74CBF00400640CF
:10171000012808B517D10320FFF744FF08B10120C5
:1017200008BD1D4BDA68002ABCBF4FF0B642DA6034
:10173000DA6822F4E02242F48032DA60DA6842F0B9
:101740000042DA60ECE7022811D10420FFF72AFFFB
:101750000028E4D1104BDA68002ABCBF4FF0B64233
:10176000DA60DA6822F4E02242F40032E5E7032886
:10177000D5D10520FFF716FF0028D0D1064BDA6837
:10178000002ABCBF4FF0B642DA60DA6822F4E022E9
:1017900042F44032D1E700BF00400640024B9A6855
:1017A00060F303029A6070470000024008B5064BE0
:1017B0005A686FF3C7125A60044B1B6803B198470D
:1017C000BFF34F8F08BD00BF000002401C11002076
:1017D000104B10B51C685A68144004F440321A606B
:1017E000E20303D50C4A52684AB19047A30303D5DC
:1017F000094B9B6843B19847BFF34F8F10BD5A68A0
:1018000022F480325A60F1E7024A536823F400332D
:101810005360F1E7000002401C1100200B4B8008D0
:1018200053F820301A68002ABCBF4FF0B6421A6045
:101830001A686FF355521A601A6842F400121A605F
:101840001A6842F000421A60704700BF984F0000CB
:101850000B4B8008012153F820301A68002ABCBFC6
:101860004FF0B6421A601A6861F301021A601A68F2
:1018700042F400121A601A6842F000421A6070477F
:10188000984F00000B4B800853F820301A68002A4C
:10189000BCBF4FF0B6421A601A686FF301021A60BB
:1018A0001A686FF355521A601A6842F000421A60C3
:1018B000704700BF984F00002DE9F84F1A4BDFF832
:1018C00070A053F82050194BD5F8907053F8209021
:1018D000064600244FF0B64B4FF0010827FA04F3F8
:1018E000DB0705D5DAF8002072B1E1B23046904747
:1018F00008FA04F301343B40202CC5F89030EDD1B8
:10190000BFF34F8FBDE8F88F231D49F823B055F87A
:10191000231062F3134145F8231055F8232042F4B5
:10192000004245F82320E3E7805000009450000077
:10193000281100200020FFF7BFBF0120FFF7BCBF28
:101940000220FFF7B9BF0320FFF7B6BF0420FFF75F
:10195000B3BF0000244B043153F8203010B553F8C6
:101960002140240441BF214C54F820004FF0B644DC
:1019700040F8214053F82140107860F3000443F808
:10198000214053F82140C0F3400060F3410443F884
:10199000214053F82100547864F3C30043F8210038
:1019A00053F82100947864F3041043F8210053F8AD
:1019B0002100D47864F3451043F8210053F8210046
:1019C000147964F3DF7043F82100507953F8212033
:1019D00060F31C6243F8212053F8212042F40042B6
:1019E00043F8212010BD00BF80500000945000003B
:1019F0000E4B043153F8203010B553F82140240425
:101A000041BF0B4C54F820004FF0B64440F8214041
:101A100053F8210062F30A2043F8210053F82120F3
:101A200042F4004243F8212010BD00BF8050000066
:101A300094500000064B10B553F820400120636914
:101A4000884023EA000302FA01F10B43636110BDF1
:101A50006C500000064B10B553F82040012023685D
:101A6000884023EA000302FA01F10B43236010BD12
:101A70006C500000104A10B5034652F820401F2950
:101A800001F01F024FF0010000FA02F202D82263B7
:101A9000002010BD3F2901D8E262F9E75F2904D890
:101AA000063B012BF5D86267F2E77F29F1D8063BA8
:101AB000012BEED82267EBE74C5100000E4B53F898
:101AC00020301A6802F07F028A4212D3052801D81A
:101AD0003F290ED81A68C2F3407092000AD55B6B9A
:101AE000C3F303635B0007338B4234BF0020012044
:101AF00070470120704700BF2C510000194B82B085
:101B000053F820301848002101911A6842F08042B1
:101B10001A601A6842F080521A601A688A42BEBF80
:101B20001A6861F3DF721A600146019A824205D891
:101B3000019A013201921A681201F6D5019A8A427D
:101B400004D800220192019A8A4202D9012002B0EF
:101B50007047019A013201921A68D201F3D5002030
:101B6000F5E700BF2C5100003F4B4C000F4B82B0FB
:101B700053F8203000220192196862F31C71196039
:101B8000196862F39E71196042F20F71019A8A42DC
:101B900001D9012007E0019A013201921A68C2F3CB
:101BA0000060D201F2D402B0704700BF2C51000097
:101BB000104B53F820301A68120519D5D3F8000CD1
:101BC00029B9C0F30140C11C0120884006E0012969
:101BD00006D1C0F3C140033001FA00F0C0B2704733
:101BE000022902D1C0F38150EDE7C0F34160EAE77A
:101BF0000820F3E72C5100002DE9F74F9A46204BBF
:101C000053F82030009305460E4617460AB10023CC
:101C10001370062D4FF0000434BF4FF0010B4FF04E
:101C2000030B22464FF40078E1B22846B61A019120
:101C3000FFF7BEFF4FEA44290830F6B2B8FBF0F2D6
:101C40000FB101993970964214D2009B03F18008BC
:101C5000C84400FB0680CAF80000062D34BF4FF4CC
:101C600080604FF4006048458CBF0020012003B025
:101C7000BDE8F08F0134A3454FEA4429D4D2ECE704
:101C80002C5100002DE9F3471D466E4B0A9E53F878
:101C90002090144601AB0DF1030280468A46FFF7FF
:101CA000ABFF012803D1012002B0BDE8F0876378C3
:101CB000402BF8D851464046019FFFF7FFFE012810
:101CC000F1D0D9F800301B0508D56379012B02BF8C
:101CD000D9F8003C43F00043C9F8003C9DF80310DC
:101CE00094F801904046FFF763FF8145DBD86178A7
:101CF000082908464DD90C294DD910294ED9142947
:101D00004FD9182950D9202951D9312935BF30222E
:101D100040220E200F20002E4CD1019900220A6093
:101D20004A600B6860F313430B6023789DF8300022
:101D3000012B00F0070079D125F060454D604B681C
:101D400060F35F734B600B6843F400130B600B6828
:101D500062F396530B60A378012B02BF0B6843F428
:101D600080130B600B686FF31B630B60E378012B30
:101D700002BF0B6843F000430B6062790B6862F3AB
:101D80009E730B600B680B9A62F31B630B60002061
:101D90008AE70A46BFE70C220920BCE710220A2086
:101DA000B9E714220B20B6E718220C20B3E7202253
:101DB0000D20B0E7DDF804E08908B4464FF00008D4
:101DC0005FFA88F38B420CF1040C0ED308378900BC
:101DD00063788B421FD8D2B29A429ED983F0030116
:101DE00026797E540133DBB2F6E71CF8033C1CF87D
:101DF000049C1B0443EA09631CF8019C43EA0903A1
:101E00001CF8029C43EA092308F1020908F10108C1
:101E10004EF82930D4E781F0030303F03F0316F8AE
:101E200001C007F803C00131C9B2D1E74B6865F3BF
:101E30009C434B604B6860F35F734B600B6862F3CD
:101E4000555383E72C5100002DE9F34115461C46FC
:101E50000DF1030201ABDDF8208006460F46FFF7C7
:101E6000CBFE012803D1012002B0BDE8F081394644
:101E70003046FFF723FE0128F5D001990020012DFF
:101E80000860486013D124F060444C600B6843F450
:101E900000130B600B6860F396530B60B8F10F0FE3
:101EA0001EBF0B6868F31B630B600020DCE74B6808
:101EB00064F39C434B600B6860F35553E9E7000003
:101EC0002D4B2DE9F04753F820A02C4BDAF8006099
:101ED00053F82040DFF8A890236BA26A06F07F0633
:101EE000013603EA0208102E4FF04C071FFA88F85B
:101EF00028BF10260025474328FA05F3DA070FD537
:101F0000DAF800309B0020D5072D1ED8052D11D101
:101F100009EB0703DB6A43B198470123AB40236316
:101F20000135AE42E8D1BDE8F087A36A23F0200373
:101F3000A362F2E7062D14D109EB07031B6B002BFC
:101F4000EAD1A36A23F04003F2E759F8073013B14E
:101F500028469847E1E7A36A0122AA4023EA020340
:101F6000E6E7072DD9D109EB07035B6B002BD3D133
:101F7000A36A23F08003DBE72C5100004C510000E2
:101F80006C1100201D4B1E4A53F820302DE9F047FC
:101F900052F820901C68D9F83030D9F82820DFF8A2
:101FA00064A004F07F04013403EA02084FEA1848F1
:101FB000202C4FF04C074FEA084828BF202410255A
:101FC0004743A54201D3BDE8F08728FA05F301266F
:101FD000DB0706FA05F605D50AEB07035B682BB1AC
:101FE00028469847C9F830600135EAE7D9F8283023
:101FF00023EA0603C9F82830F4E700BF2C5100009B
:102000004C5100006C1100201B4B1C4A53F820302F
:102010002DE9F0471C6852F82060DFF864A0F76AE9
:10202000736A04F07F0401341F40302C4FF04C09D8
:10203000BFB228BF3024202509FB00F9A54201D3F7
:10204000BDE8F087A5F120034FF0010808FA03F876
:1020500027FA03F3DB0705D50AEB09039B6833B1C5
:10206000284698470135C6F82C80EDB2E6E7736A3A
:1020700023EA08037362F5E72C5100004C5100007D
:102080006C1100201C4B1D4A53F820302DE9F047FD
:1020900052F820701C68FD6A7B6ADFF864A004F0C7
:1020A0007F0401341D402D0C402C4FF04C094FEAA9
:1020B000054528BF4024302609FB00F9A64201D37C
:1020C000BDE8F087A6F120034FF0010808FA03F8F5
:1020D00025FA03F3DB0705D50AEB0903DB682BB10F
:1020E00030469847C7F82C800136E7E77B6A23EA39
:1020F00008037B62F6E700BF2C5100004C51000042
:102100006C1100202C4B2DE9F04753F820A02B4BED
:10211000DAF8006053F82050DFF8A4802A6BAB6A2D
:1021200006F07F060136202E4FF04C0702EA030925
:1021300028BF20260024474329FA04F3DA070FD5E5
:10214000DAF800309B002BD5072C29D8052C11D1AB
:1021500008EB0703DB6A43B198470123A3402B63D5
:102160000134A642E8D1BDE8F087AB6A23F0200332
:10217000AB62F2E7062C08D108EB07031B6B002BC0
:10218000EAD1AB6A23F04003F2E7072CE5D108EB74
:1021900007035B6B002BDFD1AB6A23F08003E7E71B
:1021A00058F8073013B120469847D6E7AB6A0122AA
:1021B000A24023EA0203DBE72C5100004C5100004F
:1021C0006C110020194B1A4A53F820302DE9F047C2
:1021D0001C6852F82060DFF85CA0F26A736A04F0B1
:1021E0007F040134402C4FF04C0902EA030828BF59
:1021F0004024202509FB00F9A54201D3BDE8F08762
:10220000A5F1200301279F4028FA03F3DB0705D53A
:102210000AEB09035B6823B128469847F76201354A
:10222000EAE7736A23EA07037362F7E72C510000B9
:102230004C5100006C1100201A4B1B4A53F82030FF
:102240002DE9F0471C6852F82060DFF860A0726F3B
:10225000F36E04F07F040134602C4FF04C0902EA65
:10226000030828BF6024402509FB00F9A54201D3DB
:10227000BDE8F087A5F1400301279F4028FA03F34A
:10228000DB0705D50AEB09039B682BB12846984765
:1022900001357767EDB2E9E7F36E23EA0703F366EA
:1022A000F6E700BF2C5100004C5100006C110020DB
:1022B000184B194A53F820302DE9F04752F82060A6
:1022C0001C68326FB36EDFF854A004F07F044FF047
:1022D0004C09013402EA0308602509FB00F9A54214
:1022E00001D3BDE8F087A5F1600301279F4028FADC
:1022F00003F3DB0705D50AEB0903DB6823B12846A6
:10230000984737670135EAE7B36E23EA0703B366F8
:10231000F7E700BF2C5100004C5100006C11002069
:10232000F8B5274B53F820402368C3F30067DB015F
:1023300006460D4606D5042D3ED8DFE805F0091601
:10234000263D3900FFF7DAFB0028F4D0012036E003
:1023500063686FF3C303636063686FF30C33636098
:1023600023686FF3D753236007E0636843F00803E3
:10237000636063686FF30C336360FFB93046FFF747
:10238000F5FB003818BF012019E063686FF3C30341
:102390006360636843F48053636023686FF3514361
:1023A0002360D4F8003C6FF3CF33C4F8003CE4E77B
:1023B000236843F00043D6E7032DDED10020F8BDAB
:1023C0002C510000114B82B053F8203000210191B4
:1023D0001A68C2F30050D20215D51A6861F3DF7291
:1023E0001A6042F20F71019A8A4205D8019A0132AD
:1023F00001921A68D202F6D4019842F20F73984201
:1024000094BF0020012002B0704700BF2C51000093
:10241000104B82B053F82030002001901A6882429D
:1024200015DB1A6842F000421A6042F20F71019AFD
:102430008A4205D8019A013201921A68D202F6D571
:10244000019842F20F73984294BF0020012002B01D
:10245000704700BF2C510000F8B5214B53F82040C5
:102460002368C3F30067DB0106460D462FD5D5F878
:1024700000C0BCF1000F2ED0696861B3A86850B3EA
:10248000EB6843B32A6932B365680CF1FF3C6CF327
:10249000020565606568013860F312456560606833
:1024A000013961F3D54060606168013BDBB263F3E1
:1024B0001F6161606368013A62F39753636067B9B3
:1024C0003046FFF753FB003818BF012004E0FFF748
:1024D00015FB0028CBD00120F8BD0020FCE700BF91
:1024E0002C510000F8B5204B53F820402368C3F36B
:1024F0000067DB0106460D462ED5D5F800C0BCF1BD
:10250000000F2DD0696859B3A86848B3EA683AB398
:102510002B692BB3256D0CF1FF3C6CF38F252565E2
:10252000256D013860F304052565206D013961F3DF
:1025300049102065216D013A62F35E512165226DDB
:10254000013B63F31442226567B93046FFF70EFB87
:10255000003818BF012004E0FFF7D0FA0028CCD0E3
:102560000120F8BD0020FCE72C510000F8B5244BF9
:1025700053F820402368C3F30067DB0106460D468D
:1025800036D5D5F800C0BCF1000F37D06968A9B3C3
:10259000A86898B3EA688AB32B697BB3D4F8045C63
:1025A0006CF38E25C4F8045CD4F8045C013860F345
:1025B0000205C4F8045CD4F8040C013961F3471037
:1025C000C4F8040CD4F8041C013A62F31D51C4F899
:1025D000041CD4F8042C013B63F31242C4F8042C0D
:1025E00000241FB93046FFF7C1FA28B92046F8BDCC
:1025F000FFF784FA0028C4D00124F7E70124F0E7AC
:102600002C510000BF4B2DE9F04F53F82040BE4B3A
:1026100053F820702368002B85B005460E4680F2E3
:1026200057812846FFF7CEFE002840F05481284607
:10263000FFF764FA002840F04E81236843F00073EE
:10264000236042F20F720390039B934205D8039BD1
:102650000133039323689B01F6D4039A42F20F736C
:102660009A4200F23881236843F480532360636BFD
:10267000062D43F0805334BF4FF480724FF4007244
:10268000636307F1800334BF4FF0400A4FF0800AC4
:1026900003EB8202002143F8041B9342FBD107F5B0
:1026A000086202EB8A014FF0FF3342F8043B8A4292
:1026B000FBD13B6104F698227B610021BB61BB64C6
:1026C00004F5286343F8041B9A42FBD14FF0FF3214
:1026D000C4F8A02A04F52B63C4F8A42A0021C4F886
:1026E000A82AC4F8AC2A04F52E6243F8041B9A42C7
:1026F000FBD104F6287204F58051002342F8043B14
:102700008A42FBD1626BA5F106095FFA89F963F38E
:102710001C72B9F1010F6263BB627B629CBFFB66F6
:10272000BB664FF0FF33B9F1010F3B63FB629CBF07
:102730007B673B67754B3B624FF45023C7F8FC3A0D
:102740004FF44033C7F8083B307F226800F00103A4
:1027500063F3CB222260226842F480322260226D31
:1027600063F3DF722265D4F8002C6FF3CF32C4F824
:10277000002C626B012863F30C32626306F10801DE
:1027800040F0B380727FD4F8003C62F31143C4F888
:10279000003CB27FD4F8003CB9F1010F62F3D4439E
:1027A000C4F8003C0ED8F27FD4F8003C62F3975393
:1027B000C4F8003C96F82020D4F8003C62F35A6339
:1027C000C4F8003C2846FFF78DFE012800F0838006
:1027D00006F124012846FFF7C9FE01287BD03368A3
:1027E000019300212846FFF7E3F9012100F10808D1
:1027F0002846FFF7DDF9B9F1010F4FF4007B00F136
:102800000800BBFBF8F8BBFBF0F0804411D80221B4
:102810002846FFF7CDF9032181462846FFF7C8F97E
:1028200009F108090830BBFBF9F9BBFBF0F3994447
:10283000C844019B5FFA88F843454CD83368534538
:1028400049D82268013B63F306022260F17902292C
:102850001EBF236843F4003323603379012B48D132
:10286000337F002B37D1236843F000532360727904
:10287000636B62F31B636363B279236862F3CF33E4
:1028800023604FF0FF33BB64236843F4802323604D
:102890002846FFF745FDF0B9F379032B03D028460E
:1028A000FFF764F9B8B9636B43F000536363D4F87E
:1028B000E03A60F3DF73C4F8E03AD4F8E03A60F34A
:1028C000C713C4F8E03A636B60F35D73636303E0BE
:1028D000FFF714F918B1012005B0BDE8F08F2846C4
:1028E000FFF796FD0028F6D19BE62846FFF7B4FDDA
:1028F00073E723686FF35D732360B379012BC3D152
:10290000E9E700BF2C5100004C51000007001B00FC
:10291000F8B50F4B53F820502B68C3F30067DB0169
:1029200004460E4606D52B6866F310432B603FB174
:102930000020F8BDFFF7E2F80028F4D00120F8E706
:102940002046FFF713F9003818BF0120F1E700BF58
:102950002C5100002DE9F04799461A4B154653F8C3
:102960002030194A1F6852F820808A4629460646B8
:10297000FFF7A4F8C7F30067044618B10124204606
:10298000BDE8F0874FB105F50875BAF1000F0AD020
:1029900029F0604348F825300AE03046FFF7AEF8EA
:1029A0000028EBD1EFE7094A02EA894248F82520DE
:1029B000002FE4D13046FFF7D9F8041E18BF0124D8
:1029C000DDE700BF2C5100004C5100000000FC1F4F
:1029D000F7B504460D4616461F46FFF74BF8E8B913
:1029E0000F23009332463B462046FFF72DFA98B955
:1029F00000903B46324629462046FFF725FA58B953
:102A000029462046FFF736F830B9042300933246B2
:102A10003B462046FFF718FA03B0F0BD0120FBE764
:102A2000F0B587B016461F460DF1130205AB0446FC
:102A30000D46FFF7E1F8012802D1012007B0F0BDF3
:102A400029462046FFF73AF80128F6D0059B1B6877
:102A500013F0706FC3F3036104D0083101F00F016C
:102A6000012910D829462046FFF704F80028E4D1B0
:102A70000C2301930C9B0290009332463B46204668
:102A8000FFF700F9DAE70220D8E72DE9F34117460E
:102A900098460DF1030201AB05460E46FFF7ACF870
:102AA000012803D1012002B0BDE8F081314628465B
:102AB000FFF704F80128F5D0019B1B6813F0706F35
:102AC000C3F3036404D0083404F00F04012C06D8C7
:102AD00043463A4631462846FFF77AFFE3E70220AD
:102AE000E1E700002DE9F3413C4B0C4653F8206030
:102AF000154601AB0DF10302C9B28046FFF77CF821
:102B0000012803D1012002B0BDE8F08121464046F2
:102B1000019FFEF7D3FF0128F4D0019B9DF803101D
:102B20001A681C68C4F30344082C82BF093C2C4B70
:102B3000E4B2404688BF1C5DFFF73AF8A04205D2D8
:102B40009DF803104046FFF733F80446019A85F8D4
:102B5000484013682B60136813F4001F536814BFB8
:102B600023F06043C3F38A436B60C4F3870E05F11F
:102B700008030021C8B2864503F104030AD804F013
:102B8000FC0303F1080208371544A3421BD3B368C2
:102B90000020B8E702EB81000131D0F808C04FEA0D
:102BA0001C6C03F804CCD0F808C04FEA1C4C03F8A6
:102BB00003CCD0F808C04FEA1C2C03F802CC806884
:102BC00003F8010CD6E783F0030202F03F02013361
:102BD000BA5C05F8012BDBB2D7E700BF4C5100000F
:102BE000A8500000052809D8032907D8132303FBA0
:102BF0000011034B002043F821207047012070474B
:102C00006C1100202DE9F74F0F469849DDF830A0F0
:102C100051F820509649DDF8349051F82040296849
:102C20009846CB010646C1F3006B14D5102F2FD860
:102C3000DFE817F04E004E00660066008700870050
:102C40009D00AF00AF00AF00BB00BB00BB00D400D5
:102C5000D4001900E3000192FEF750FF002840F075
:102C60004381019AE2E7B11FC9B2F2B9A26A42EA0E
:102C70000802A262636A012943EA0A03636207D871
:102C8000E36E0E9A43EA0903E366A36E1343A36659
:102C9000BBF1000F40F02A813046FEF767FF003895
:102CA00018BF012003B0BDE8F08FA26A22EA080332
:102CB000A362636A012923EA0A036362E8D8E36E28
:102CC0000E9A23EA0903E366A36E23EA0203DEE712
:102CD000684B6948694D53F8271055F8275050F84C
:102CE000263032B962682A4362600B4340F82630CE
:102CF000CEE7626822EA0502626023EA0103F5E793
:102D00005C4B5D495D4853F827C051F8263050F8B8
:102D100027705AB9286840F40010286062683A4366
:102D2000626043EA0C0341F82630B1E72A686FF38A
:102D300055522A60626822EA0702626023EA0C03A5
:102D4000F1E74C4B4C494D4D53F8270055F82750AF
:102D500051F8263022B9626B2A4362630343E2E7EB
:102D6000626B22EA0502626323EA0003DBE7424961
:102D700051F8263032B9226842F08062226043F076
:102D80000103D0E7226822F08062226023F0010371
:102D9000C9E73A4B53F827301AB9A26A1343A36222
:102DA00076E7A26A22EA0303F9E76B6B43F000536C
:102DB0006B63D5F8E03A6FF3DF73C5F8E03A2F4B59
:102DC00053F827302AB9D4F8E02A1343C4F8E03A7C
:102DD0005EE7D4F8E02A22EA0303F7E7274B53F82B
:102DE00027302AB9D4F8002B1343C4F8003B4FE72F
:102DF000D4F8002B22EA0303F7E7B11F1E48A36AA9
:102E0000C9B2002A3ED14FF0FF33A362626A636207
:102E100001299FBFE26EE366A26EA366636843F476
:102E20004C436360636B43F0404363636B6B43F0FD
:102E300000536B63D5F8E03A6FF3DF73C5F8E03AFF
:102E4000D4F8E03A43F45023C4F8E03A2B6843F056
:102E500080632B602B6843F400132B60D4F8003B95
:102E600043F44033C4F8003B054B3FE72C510000CE
:102E70004C510000B05000004C110020F0500000F8
:102E800007001B000023A362626A636201299FBFDF
:102E9000E26EE366A26EA366636823F44C4363604C
:102EA000636B23F0404363636B6B43F000536B63CE
:102EB000D5F8E03A6FF3DF73C5F8E03AD4F8E03ABA
:102EC00023F45023C4F8E03A2B686FF39A632B6025
:102ED0002B686FF355532B60D4F8003B23F4403339
:102EE000C4F8003B002301E70120DBE60020D9E61F
:102EF0001A4B53F820201A4B30B553F82030156A7E
:102F00001D40184B2B4013626A0785B0044606D556
:102F1000154A4C2303FB00231B6963B198472B031D
:102F200019D5114A4C2303FB04231B6A5BB105B07E
:102F3000BDE83040184702930193009301221946DF
:102F4000FFF760FEEBE70293019300930122042157
:102F50002046FFF757FE05B030BD00BF4C510000C2
:102F60004C110020040008006C1100201FB50D4A10
:102F700052F820204FF4003111620B4A4C2101FB22
:102F800000239B691BB105B05DF804EB1847029361
:102F90000193009301220221FFF734FE05B05DF892
:102FA00004FB00BF4C5100006C1100201FB50D4AFE
:102FB00052F820204FF4803111620B4A4C2101FB62
:102FC0000023DB691BB105B05DF804EB18470293E1
:102FD0000193009301220321FFF714FE05B05DF871
:102FE00004FB00BF4C5100006C1100200F4B53F844
:102FF000203030B50E4D196A45F8201002211962B3
:103000000C494C2303FB001385B05B6904462BB1CC
:103010009847002345F8243005B030BD01220293C3
:10302000019300931146FFF7EDFDF2E74C510000CC
:103030002C1100206C110020104B53F8203030B5BB
:103040000F4D196A45F820104FF4801119620D498F
:103050004C2303FB001385B05B6A04462BB19847F1
:10306000002345F8243005B030BD0293019300934E
:1030700001220521FFF7C6FDF2E700BF4C51000019
:103080002C1100206C1100201A4B53F8203030B561
:10309000D3F8082BD3F8005B154005F44032C3F891
:1030A000082BEA0385B0044606D5134A4C2303FBDC
:1030B00000235B6C63B19847AB0319D50E4A4C23D0
:1030C00003FB04239B6C5BB105B0BDE8304018479F
:1030D00002930193009301220D21FFF793FDEBE78B
:1030E00002930193009301220E212046FFF78AFDEF
:1030F00005B030BD4C5100006C1100201FB50B4ACB
:1031000052F8201001220A6209494C2404FB0013E2
:103110009B6A1BB104B0BDE81040184702930193AD
:1031200000930621FFF76EFD04B010BD4C51000066
:103130006C110020234B53F8203030B5D3F8FC2A13
:10314000D3F8E05A154005F45022290385B004460F
:10315000C3F8FC2A06D51C4A4C2303FB00239B6BB7
:10316000ABB198476A0306D5174A4C2303FB0423E7
:10317000DB6BA3B19847EB0322D5134A4C2303FB27
:1031800004231B6CA3B105B0BDE83040184702937F
:103190000193009301220A21FFF734FDE2E7029335
:1031A0000193009301220B212046FFF72BFDE2E75C
:1031B00002930193009301220C212046FFF722FD88
:1031C00005B030BD4C5100006C110020234B1F296D
:1031D00010B553F820404FF001030CD803FA01F169
:1031E000A36A1AB90B43A362104610BD23EA010378
:1031F000A3620022F8E73F290BD820398B401AB987
:10320000616A0B436362EFE7626A22EA0303636267
:10321000EFE75F290ED8063801281CD840398B40CB
:103220001AB9E16E0B43E366DEE7E26E22EA0303BE
:10323000E366DEE77F290ED8063801280BD860390F
:103240008B401AB9A16E0B43A366CDE7A26E22EAAA
:103250000303A366CDE71A46C6E700BF4C51000042
:1032600008B50020FFF744FEBFF34F8F08BD08B537
:103270000020FFF77BFEBFF34F8F08BD08B500208D
:10328000FFF794FEBFF34F8F08BD08B50020FFF78E
:10329000ADFEBFF34F8F08BD08B50020FFF7CCFE91
:1032A000BFF34F8F08BD08B50020FFF7EDFEBFF359
:1032B0004F8F08BD08B50020FFF720FFBFF34F8FE9
:1032C00008BD08B50020FFF735FFBFF34F8F08BDDD
:1032D00008B50020FEF7F4FDBFF34F8F08BD08B519
:1032E0000020FEF74FFEBFF34F8F08BD08B500204A
:1032F000FEF78AFEBFF34F8F08BD08B50020FEF72A
:10330000C1FEBFF34F8F08BD08B50120FFF7F0FDE8
:10331000BFF34F8F08BD08B50120FFF727FEBFF3AD
:103320004F8F08BD08B50120FFF740FEBFF34F8F58
:1033300008BD08B50120FFF759FEBFF34F8F08BD48
:1033400008B50120FFF778FEBFF34F8F08BD08B521
:103350000120FFF799FEBFF34F8F08BD08B501208C
:10336000FFF7CCFEBFF34F8F08BD08B50120FFF774
:10337000E1FEBFF34F8F08BD08B50120FEF7A0FDA9
:10338000BFF34F8F08BD08B50120FEF7FBFDBFF36B
:103390004F8F08BD08B50120FEF736FEBFF34F8FF3
:1033A00008BD08B50120FEF76DFEBFF34F8F08BDC5
:1033B00008B50220FFF79CFDBFF34F8F08BD08B58D
:1033C0000220FFF7D3FDBFF34F8F08BD08B50220E1
:1033D000FFF7ECFDBFF34F8F08BD08B50220FFF7E4
:1033E00005FEBFF34F8F08BD08B50220FFF724FE8E
:1033F000BFF34F8F08BD08B50220FFF745FEBFF3AE
:103400004F8F08BD08B50220FFF778FEBFF34F8F3E
:1034100008BD08B50220FFF78DFEBFF34F8F08BD32
:1034200008B50220FEF74CFDBFF34F8F08BD08B56D
:103430000220FEF7A7FDBFF34F8F08BD08B502209D
:10344000FEF7E2FDBFF34F8F08BD08B50220FEF77F
:1034500019FEBFF34F8F08BD08B50320FFF748FDE5
:10346000BFF34F8F08BD08B50320FFF77FFDBFF303
:103470004F8F08BD08B50320FFF798FDBFF34F8FAE
:1034800008BD08B50320FFF7B1FDBFF34F8F08BD9E
:1034900008B50320FFF7D0FDBFF34F8F08BD08B577
:1034A0000320FFF7F1FDBFF34F8F08BD08B50320E0
:1034B000FFF724FEBFF34F8F08BD08B50320FFF7C9
:1034C00039FEBFF34F8F08BD08B50320FEF7F8FCA7
:1034D000BFF34F8F08BD08B50320FEF753FDBFF3C0
:1034E0004F8F08BD08B50320FEF78EFDBFF34F8F49
:1034F00008BD08B50320FEF7C5FDBFF34F8F08BD1B
:1035000008B50420FFF7F4FCBFF34F8F08BD08B5E2
:103510000420FFF72BFDBFF34F8F08BD08B5042033
:10352000FFF744FDBFF34F8F08BD08B50420FFF738
:103530005DFDBFF34F8F08BD08B50420FFF77CFD8C
:10354000BFF34F8F08BD08B50420FFF79DFDBFF303
:103550004F8F08BD08B50420FFF7D0FDBFF34F8F94
:1035600008BD08B50420FFF7E5FDBFF34F8F08BD88
:1035700008B50420FEF7A4FCBFF34F8F08BD08B5C3
:103580000420FEF7FFFCBFF34F8F08BD08B50420F1
:10359000FEF73AFDBFF34F8F08BD08B50420FEF7D4
:1035A00071FDBFF34F8F08BD08B50520FFF7A0FCE4
:1035B000BFF34F8F08BD08B50520FFF7D7FCBFF359
:1035C0004F8F08BD08B50520FFF7F0FCBFF34F8F04
:1035D00008BD08B50520FFF709FDBFF34F8F08BDF3
:1035E00008B50520FFF728FDBFF34F8F08BD08B5CC
:1035F0000520FFF749FDBFF34F8F08BD08B5052033
:10360000FFF77CFDBFF34F8F08BD08B50520FFF71E
:1036100091FDBFF34F8F08BD08B50520FEF750FCA4
:10362000BFF34F8F08BD08B50520FEF7ABFCBFF315
:103630004F8F08BD08B50520FEF7E6FCBFF34F8F9E
:1036400008BD08B50520FEF71DFDBFF34F8F08BD6F
:1036500008B50620FFF74CFCBFF34F8F08BD08B537
:103660000620FFF783FCBFF34F8F08BD08B5062087
:10367000FFF79CFCBFF34F8F08BD08B50620FFF78E
:10368000B5FCBFF34F8F08BD08B50620FFF7D4FC8B
:10369000BFF34F8F08BD08B50620FFF7F5FCBFF359
:1036A0004F8F08BD08B50620FFF728FDBFF34F8FE9
:1036B00008BD08B50620FFF73DFDBFF34F8F08BDDD
:1036C00008B50620FEF71EFDBFF34F8F08BD08B5F5
:1036D0000620FEF777FDBFF34F8F08BD08B5062023
:1036E000FEF7AAFDBFF34F8F08BD08B50620FEF711
:1036F000DFFDBFF34F8F08BD08B50720FFF7F8FBCC
:10370000BFF34F8F08BD08B50720FFF72FFCBFF3AD
:103710004F8F08BD08B50720FFF748FCBFF34F8F58
:1037200008BD08B50720FFF761FCBFF34F8F08BD48
:1037300008B50720FFF780FCBFF34F8F08BD08B521
:103740000720FFF7A1FCBFF34F8F08BD08B5072086
:10375000FFF7D4FCBFF34F8F08BD08B50720FFF774
:10376000E9FCBFF34F8F08BD08B50720FEF7CAFC80
:10377000BFF34F8F08BD08B50720FEF723FDBFF349
:103780004F8F08BD08B50720FEF756FDBFF34F8FDA
:1037900008BD08B50720FEF78BFDBFF34F8F08BDAE
:1037A0002D4B2DE9F04153F820502C4B53F820704D
:1037B0002B4BFE6853F820301E4026F00103FB60BF
:1037C000F307044607D51423264A4343D35843B38B
:1037D00098470123FB60B00706D5224A142303FB58
:1037E00004235B6813B39847710706D51D4A142359
:1037F00003FB04239B68F3B19847320706D5194AA7
:10380000142303FB0423DB68D3B19847B30520D509
:103810001448142303FB04042369B3B1BDE8F04149
:1038200018472A6963F300022A61D2E72A6963F321
:1038300041022A61D8E72A6963F382022A61DCE740
:103840002A6963F3C3022A61E0E72A6963F3451238
:103850002A61BDE8F08100BF6C5100007451000086
:10386000CC130020D41300200020FFF799BF0120C3
:10387000FFF796BF1A4B53F8203088789A680228D1
:103880001DBF6FF304129A605A6942F0100216BF0E
:1038900060F3CF329A605A615A69487860F31042F7
:1038A0005A615A69087860F352425A615A69C87875
:1038B00060F3CB225A615A69087960F3D5425A61A4
:1038C0005A69886860F39F525A619A68C96861F3BF
:1038D000D5229A609A6842F480629A60704700BF6D
:1038E0006C51000010B50A4B0A7853F82030586923
:1038F00062F3000058614C78586964F34500012A6E
:10390000586101BF89785A6961F387125A6110BD05
:103910006C510000034B53F82020936843F00103DF
:10392000936070476C510000034B53F820309A6845
:103930006FF300029A6070476C510000174B82B021
:1039400053F82030002201925A69162161F3450292
:103950005A619A6842F001029A609A6842F0020243
:103960009A6042F20F71019A8A4201D9012007E060
:10397000DA6852060ED59A686FF341029A60002009
:103980009A686FF300029A605A696FF345025A61B0
:1039900002B07047019A01320192E4E76C510000D5
:1039A000034B53F82020936A43F00103936270475E
:1039B0006C510000034B53F82030186AC0F310001C
:1039C000704700BF6C510000044B53F82030DB6897
:1039D00023FA01F101F00100704700BF74510000AB
:1039E00008B50B4B53F820301B6ADB0705D51423B1
:1039F000084A4343D3581BB19847BFF34F8F08BDC4
:103A0000054A52F82020D16963F30001D161F4E73F
:103A10008C510000FC1300207C51000007B50F4BB7
:103A20000F4A53F8203052F82020116A5A6A02F0E7
:103A3000010201928A0706D50A4A142101FB0020DF
:103A400042682AB19047BFF34F8F03B05DF804FB83
:103A5000D96962F34101D961F5E700BF7C510000EB
:103A60008C510000FC13002008B50C4B53F820309B
:103A70001B6ADB0606D50A4A142303FB00231B69D5
:103A80001BB19847BFF34F8F08BD064A52F820205C
:103A9000D16963F30411D161F4E700BF8C510000D8
:103AA000FC1300207C51000007B50F4B0F4A53F860
:103AB000203052F82020116ADA6A02F001020192E5
:103AC0004A0706D50A4A142101FB002082682AB160
:103AD0009047BFF34F8F03B05DF804FBD96962F3E1
:103AE0008201D961F5E700BF7C5100008C510000D4
:103AF000FC13002007B50F4B0F4A53F8203052F843
:103B00002020116A9A6A02F0010201920A0706D582
:103B10000A4A142101FB0020C2682AB19047BFF372
:103B20004F8F03B05DF804FBD96962F3C301D9611B
:103B3000F5E700BF7C5100008C510000FC13002011
:103B40000020FFF74DBF0020FFF768BF0020FFF700
:103B50008BBF0020FFF7A8BF0020FFF7CBBF0120DD
:103B6000FFF73EBF0120FFF759BF0120FFF77CBFE1
:103B70000120FFF799BF0120FFF7BCBF0220FFF72C
:103B80002FBF0220FFF74ABF0220FFF76DBF0220C0
:103B9000FFF78ABF0220FFF7ADBF0320FFF720BF6A
:103BA0000320FFF73BBF0320FFF75EBF0320FFF7B3
:103BB0007BBF0320FFF79EBF00292BD0164B53F885
:103BC000203008781A6860F355521A60DA688889DC
:103BD00060F30F02DA604A681868013A62F3144031
:103BE00018601A68087A60F386121A601A68487AB0
:103BF00060F3C7121A60887A1A6860F309221A60A3
:103C000008691A6960F301021A6149691A6961F366
:103C100011421A61704700BF7C510000044B53F8F9
:103C200020301A68013961F314421A60704700BFEE
:103C30007C510000034B53F82020936843F00103AC
:103C4000936070477C510000034B53F820309A6812
:103C50006FF300029A6070477C510000034B53F8E9
:103C600020309A6861F311429A6070477C510000DD
:103C7000024B53F820301966704700BF8C5100008A
:103C8000024B53F82030186E704700BF8C51000073
:103C9000044B53F8203001209B6988401840C840ED
:103CA000C0B270478C510000002808DB4209012394
:103CB00000F01F0003FA00F0014B43F822007047A8
:103CC00000E100E00028ACBF00F16040064B4FEA85
:103CD0000111ACBF00F5614000F00F00C9B2B4BFE4
:103CE000195480F80013704714ED00E010B500215E
:103CF0008520FDF7EFFA00218620FDF7EBFA012180
:103D000000220846FDF7D2FC4248FDF75DFA01208B
:103D1000FDF79EFC0220FDF741FD0320FDF7F8FCB6
:103D200004460028F9D1A020FDF7ACFD0421A02015
:103D3000FDF792FB0421A020FDF7CCFAA020FDF7AF
:103D400087FD05216420FDF787FB21466420FDF7F0
:103D5000C1FA05216820FDF77FFB21466820FDF7A9
:103D6000B9FA6420FDF75AFD6420FDF771FD682063
:103D7000FDF754FD6820FDF76BFDB020FDF768FDF1
:103D8000B420FDF765FDB820FDF762FDBC20FDF70E
:103D90005FFDC020FDF75CFDD020FDF759FD04213B
:103DA0008820FDF759FB04218C20FDF755FB2146A7
:103DB0008820FDF78FFA21468C20FDF78BFA8820AA
:103DC000FDF72CFD8C20FDF729FD8820FDF740FD37
:103DD0008C20FDF73DFD04213020FDF73DFB214601
:103DE0003020FDF777FA3020FDF718FD3020FDF781
:103DF0002FFD0521B020FDF72FFB0121B020FDF79D
:103E000069FAB020FDF724FDBDE81040D020FDF791
:103E10001FBD00BF0810002008B50120FDF7BEF946
:103E20000120FDF775FC58B901218520FDF752FAF4
:103E300001218620FDF74EFA03218720FDF74AFA7B
:103E4000BDE8084000213020FDF706BB08B5FFF7AC
:103E5000E3FF00F07BF86420FDF7E0FC6820FDF74D
:103E6000DDFC0020FFF7F0FE0120FFF7EDFE6420EF
:103E7000FDF708FD6820FDF705FD8820FDF7CEFC65
:103E80008C20FDF7CBFC0020FFF74EFD0120FFF753
:103E90004BFD8820FDF7F6FCBDE808408C20FDF7BF
:103EA000F1BCFDF763B9F7B50026054637462A7819
:103EB000B3B29A4201D803B0F0BD68688DF80170C2
:103EC00006EBC604031901369A788DF80020DA78DB
:103ED0008DF802201A7A8DF804208DF803708DF881
:103EE00005705978005D6A46FDF734FD6B68191955
:103EF000185D4A794978FDF77BFD6B681919185DE3
:103F00008A794978FDF796FD6B681919185DCA79A9
:103F10004978FDF79FFDCAE70A4B0B4900226FF075
:103F20007F401A6008604A601A6842F004021A6012
:103F30001A6842F002021A601A6842F001021A601E
:103F4000704700BF10E000E014E000E0044B0021E7
:103F500059604FF0FF3099601960FFF7B3BE00BFA2
:103F600010E000E00E490F4838B50268D1E900457D
:103F700000686FF07F439A1A1B1A9A428ABFD1E9F0
:103F8000004542EA040043EA040028304FF05002A2
:103F90004FF0000345F10001FCF7B4FE38BD00BF4F
:103FA0005014002018E000E008B5FFF7DBFF08BD63
:103FB000054930B5D1E9002312F1807443F10005C1
:103FC000C1E9004530BD00BF5014002070B5044663
:103FD00000262378F5B2AB4200D870BD636803EBCE
:103FE000C50213F835005168FFF7E6FD636813F862
:103FF0003500FFF71FFE0136EBE700002DE9F04F1B
:10400000984687B0364B039015464FEA48025E68E3
:1040100001921B78049305EB48024FF0000A0F460B
:104020000292D146049B5FFA8AFB5B4503D848465F
:1040300007B0BDE8F08F06EBCB04039B62789A4291
:1040400040D1626816F83B000592FFF7FDFD059A26
:1040500016F83B005168FFF7E1FD16F83B00FFF74B
:10406000E9FD16F83B00A178FFF7F8FD4FF0011BC2
:1040700020780121FFF70CFE28B1B9F1000F05D11E
:104080004FF0000B0EE0BBF1010BF1D14DF6AD632B
:104090002B804FF0010915E037F82B10FFF7E8FDF2
:1040A0000BF1010BC3452078F6D1019B4FF0011BAA
:1040B0001F4420780321FFF7EBFD30B1AB46029B94
:1040C0009B4506D10AF1010AACE7BBF1010BF0D127
:1040D000DCE72078FFF7D4FD2BF8020BEFE700BFF9
:1040E0000856000070B5044600262278F3B29A42C2
:1040F00000D870BD62681D0102EB0313505D596862
:10410000FFF7B8FB63685A19127B12B1585DFFF7CD
:1041100015FC6368585DFFF7FDFB0136E5E700001D
:1041200073B50E460DF107020DF10601C0B200F0A5
:10413000FFF8054638BB154B5C689DF8063004EB6C
:10414000031218019DF807309168205C03EB4303CC
:104150001944FFF7C7FB9DF806301B01E05CFFF731
:104160001FFC9DF806301B010721E05CFFF72CFCCB
:104170000128F6D09DF806301B01E05CFFF71AFC21
:10418000C0F30B003080284602B070BD48560000D6
:1041900007B50090ADF804100020694600F0CAF998
:1041A00003B05DF804FB000010B5074C0021224667
:1041B0000120FEF797FC94F8481004F10800FFF77F
:1041C000E7FF0023636010BD581400207047000013
:1041D00010B518490120FEF715FA174A00210120F1
:1041E000FEF700FD002211460120FEF7EFFF01213E
:1041F0004B20FFF767FD4B20FFF756FD02214620BD
:10420000FFF760FD4620FFF74FFD0022114640F208
:10421000F1630120FEF739FC01210846FEF778FB27
:104220000022BDE8104040F2FF7311460120FEF766
:1042300091BB00BF14100020A9410000FFF7C8BFC8
:1042400030B597B0002305AD039340F243630C46AD
:1042500004930A464FF055330146284605936B6098
:10426000FCF7B6FCE3B261071EBF23F00703083377
:10427000DBB201218DF85430044A009540F24363CB
:104280000846FEF7CDFB012017B030BD9C51000061
:1042900007B5FFF72BFDFFF704FE1448FFF703FEF9
:1042A0000020FFF739FE1248FFF790FE43238DF8F8
:1042B000053000220DF106030DF105010120FCF788
:1042C000A2FEBDF806104FF6FD5245F60123002967
:1042D00008BF1346074A1360FCF797FE0648FFF72E
:1042E00001FFFFF775FF00F0A9FBFEE7F85500009E
:1042F00008560000800900204856000010B5012B28
:10430000094B14BFD2434FF0FF320144884201D120
:10431000D04310BD10F8014B6240D4B253F8244092
:1043200084EA1222F2E700BFA4510000FFF7E6BFC3
:10433000032809D8054B00EB4000184443780B7064
:104340008378137000207047012070475C5600008E
:10435000704700002DE9F843FFF770FF00F0F8F810
:1043600000F02EFD72B60020FFF71EFE224C00F179
:10437000E503206000F22F60E360A06162B6DFF821
:1043800080801E4E0020FFF70FFE00238146336021
:104390000C273368022B02D9FFF7DAFFF1E708EBAD
:1043A00003121901926802B307FB03F2A258A9EBAA
:1043B0000202002A19DB012507FB03431B7A13B114
:1043C00058F80130984775B1336807FB03F108EBE3
:1043D000031362589B681A44625033680133336098
:1043E000002DD6D0CDE70125F7E707FB034255683E
:1043F000002DF2D00025DFE76C100020A41400206F
:10440000685600001C2202FB00F30349C85C012827
:1044100004BF0022CA5470479C100020074B10B5FF
:104420001C2404FB00300323038143687F241C7099
:104430004368597043689A7010BD00BF9C100020FB
:1044400061B9074A1C2101FB002041680A7840320B
:104450000A709B890289013313440381704700BFAE
:104460009C10002010B5094A1C2303FB00239C7EEE
:1044700019B10CB100229A7610BD012C08BF9976B3
:104480001C23584301231354F6E700BF9C1000205F
:1044900030B51C22074C02FB00F3E2180125907E88
:1044A00030B9103395762344158B95820B6030BD5F
:1044B0002846FCE79C100020034B1C2202FB003026
:1044C00000230381704700BF9C10002038B51C23D7
:1044D000054C03FB00F5281D204400F030F810B116
:1044E0002C440023A37338BD9C100020F0B5104C61
:1044F0001C2505FB00404D1C0769868A7C191C6041
:1045000081F47F4484F0FF0426449E80068B264479
:10451000DE80466835449D6000259D8185892C4458
:10452000DC817B5C735403695B5C1370F0BD00BF7E
:104530009C1000200B468988186800F06DB98188AE
:10454000006808B500F014F9013818BF012008BD53
:1045500000F0FAB800F056BA13B50023CDE90033E5
:104560000A46F1230C4601460DF101008DF800309A
:10457000FCF72EFB611C89B26846FFF761FE012043
:1045800002B010BD1FB50446ADF80610002003A907
:10459000FFF77EFF0398BDF8063082889BB29A42EF
:1045A0000AD3BDF80620006892B22146FCF710FB42
:1045B000039BBDF806209A8000210846FFF752FFB2
:1045C000012004B010BD01210020FFF74BBF000007
:1045D00008B5FFF7F8FF034B00221A80BDE808403A
:1045E000FFF7F1BFCE240020FFF7F2BF2DE9F04125
:1045F0001B4C2588A84206460F46904615D0A28936
:10460000904221D0238B984220D00DBB0020FFF791
:10461000CBFC0C235D4363194FF47A7101FB070057
:1046200066535860C3F808800BE000250020FFF7B0
:10463000BBFC0C2303FB05444FF47A7303FB070018
:1046400060600120BDE8F0810125EFE70225EDE77C
:1046500012B11BB90225D9E70125D7E70020F1E700
:10466000A824002037B5234A234C13782588591CE9
:104670001170224903F00F0343F02003294406225E
:104680000DF101008DF80030FCF7A2FA1C4B1988DF
:10469000491B89B205299ABF013189B207216846B1
:1046A0001D46FFF759FF01281FD123882A880633AA
:1046B0009BB29A42238003D80023238003B030BDED
:1046C000104B1A78511C19700F4B1B789A4207D364
:1046D00033B10E4A4FF47A710220FFF787FFEDE7FE
:1046E0000B4B0C4A19780120F7E700232380FFF7D2
:1046F0006AFFE3E7D0240020CE240020A814002085
:10470000D2240020CD240020D4240020D145000054
:10471000D52400206546000007B530238DF804300D
:10472000074B1B788DF80530064B03211B788DF85D
:10473000063001A8FFF710FF03B05DF804FB00BFCF
:10474000CC240020D1240020054B064800211980EC
:10475000054B1970054B2422197000F063BB00BF94
:10476000CE240020A8240020D1240020CC24002026
:10477000B1F5805FF7B505460C463FD20629CAB2AF
:1047800010D81F4E304600F8012B0A462946FCF788
:104790001FFA611C89B23046FFF7DEFE0446204650
:1047A00003B0F0BD0B0A052743F0100301468DF856
:1047B00001200DF102003A468DF80030FCF708FAAE
:1047C000224629460E480F4EFCF702FA0E4B378060
:1047D00001221A700D4B00251D700D4B07216846F4
:1047E0001C80FFF7B9FE0128044606D1094A4FF4A0
:1047F0007A710220FFF7FAFED1E735800024CEE778
:10480000A8140020CE240020D0240020CD24002095
:10481000D2240020D145000073B50278ADF806100F
:10482000432A034609D1427802F0F00120292ED014
:1048300005D8002937D0102945D002B070BD3029E5
:10484000FBD1654A1188022900F0C18091890229B3
:1048500000F0BF80118B022903D10C2041430020BE
:104860005052BDF8062092B2022AE6D95A7812F0C8
:104870000E00E2D159499C780C70D978584B1970C8
:10488000584B1870D307D8D4574A01203BE0524AFE
:10489000118803293CD09189032951D0118B032918
:1048A0003BD1022035E05148062A0180C5D8BDF829
:1048B000060080B2824291B2BFD2981C02B0BDE81D
:1048C0007040FFF75FBE8178120202F470620A4402
:1048D0004649062A0A8002D800230B80ADE705244A
:1048E0002246C11C4248FCF773F9424B1C80424BE4
:1048F00001221A703B4B00221A70FFF70DFF3F4A4E
:104900004FF47A71032002B0BDE87040FFF76EBE2D
:1049100000200C2141430020505234490A880E46A1
:10492000002A8AD0344C5878227800F00F00824256
:1049300008D000230B8002B0BDE87040FFF743BEF3
:104940000120E6E7013202F00F022270294CBDF887
:104950000620258815FA82F2B2F5805F24DABDF8C8
:104960000620234892B2052A98BFBDF806202844A5
:1049700003F1020194BF92B20622FCF729F9BDF8B7
:1049800006309BB2052B96BFBDF8063006239BB2BE
:104990001D442580318823888B4208D31448FFF7B3
:1049A000F1FD0023338048E7FFF70DFEF2E70B4BE4
:1049B0001B78002BA3D00B4A1149137809780133D7
:1049C000DBB2994213709AD80023137095E7002147
:1049D00043E7012141E700BFA8240020D4240020A0
:1049E000D5240020CD24002065460000CE240020E0
:1049F000A8140020D2240020D0240020E945000083
:104A0000CC24002070B50025094C2E4623884BB1DC
:104A10000020FFF7C9FA6368C01A002802DBA36808
:104A2000268098470135032D04F10C04EED170BDAA
:104A3000A824002081F30888004700002DE99F4842
:104A40004C4B4D4D1B684D494D4A4E4E4E4C0193BB
:104A50002B60DFF858A1DFF858B10023ADF808301B
:104A6000ADF80A30ADF80C30ADF80E300B70337085
:104A7000137023700927894690460020FFF794FAA7
:104A8000424A00F57A70106002A90020FFF748FB47
:104A90000DF10A010120FFF743FB03A90220FFF7F4
:104AA0003FFB0DF10E010320FFF73AFBBDF80800B4
:104AB0004EF612314143514534D899F80010013176
:104AC00089F80010BDF80A00314B43F6DB3148434A
:104AD00098420ED2BDF80C00DFF8D8E0484370458C
:104AE00007D9BDF80E00414399423EBF21780131FC
:104AF00021700020FFF758FA244A1168401A002854
:104B0000F7DB013F17F0FF07B7D199F80030042B0E
:104B100016D9204B1B682B602378042B17D9FFF77D
:104B200019FCFEE71C485944814295BF317898F83A
:104B300000100131013194BF317088F80010C1E7D5
:104B40003378042B01D9154BE4E7019BE3E7FFF72A
:104B50007DF9134B134A1B6893420CBF4FF480330B
:104B60004FF48023104A1360D3E90010FFF762FF6F
:104B7000D7E700BFB056000004080020D62400206C
:104B8000D8240020D7240020E0240020DC240020AA
:104B9000C05C1500A8560000BF29CD02AC5600002D
:104BA000FC7F0200AA44AA4408ED00E04F7B890084
:104BB000B08476FF8FBD98004278037843EA0223E1
:104BC0008278C07843EA024343EA006000BA704743
:104BD00008B506490068052200F0F4F818B9044B3E
:104BE00001221A7008BD3120FCE700BFB456000056
:104BF000E22400200168F8B505460846FFF7DCFF0F
:104C0000AB88AF680024043B3C70AC81074D9AB27E
:104C100010FA83F3AB4207D8054B984204D3043112
:104C2000FBF7D6FF2046F8BD3120FCE7000002204C
:104C3000008000208388082B70B5044624D10168C9
:104C40000846FFF7B9FF0646081DFFF7B5FF012329
:104C5000014605464FF0FF323046FFF767FBA2687A
:104C6000010ED170010C9170010A51701070042373
:104C7000A381A068FFF7A0FF7359834202D1034BC1
:104C800001221A70002000E0312070BDE1240020D4
:104C900008B50B4B1B7873B100680378012B0CD15E
:104CA0000130FFF789FF074A4368106043F00103B2
:104CB0009847002008BD1020FCE73120FAE700BF2C
:104CC000E124002008ED00E000207047002070473C
:104CD000F7B5264D8DF8070028880128164643D8D9
:104CE000234B9DF807C033F81170224B013080B27E
:104CF00053F82140288000239AB2974201D811240A
:104D00001BE02268624503F1010329D16379012B7D
:104D100002D1194B1B782BB323798B421CD0C1B223
:104D20000DF1070200203346FFF7E0FB21799DF8E3
:104D300007003246FFF7CCFF04462988013989B2C3
:104D4000298034B99DF807203346C9B22046FFF7C1
:104D500077FB204603B0F0BDA36830469847EBE7E9
:104D60000C34C9E77F24E8E71124F2E7E4240020AB
:104D7000B810002004110020E22400207FB500209C
:104D8000FFF740FBC8B10020FFF796FB0021084663
:104D900002AB0DF10702FFF7A9FB02AA9DF807007D
:104DA0000021FFF795FF024620B19DF80710002073
:104DB000FFF734FB0020FFF789FB07B05DF804FB29
:104DC00070470000032A70B412D940EA0105AD070C
:104DD00004460B461ED11946204653F8045B54F88E
:104DE000046BAE4216D1043A032A20461946F2D883
:104DF000561EA2B10139441E01E0C3180CD014F8AC
:104E0000015F11F8012F9542A6EB0403F5D0A81A13
:104E100070BC7047561EEDE7184670BC70471046D0
:104E2000F6E700BFF0B4860746D0541E002A3CD0F7
:104E3000CAB2034601E0013C37D303F8012B9D07BA
:104E4000F9D1032C2AD9CDB245EA05250F2C45EA24
:104E5000054534D9A4F1100222F00F0C03F120070C
:104E60001609674403F1100242E9045542E902556C
:104E70001032BA42F8D1721C14F00C0F03EB02127C
:104E800004F00F0613D0331F23F00303043313443D
:104E900042F8045B9342FBD106F003042CB1CAB282
:104EA0001C4403F8012B9C42FBD1F0BC70473446F4
:104EB0001346002CF3D1F8E714460346C1E71A461F
:104EC0002646E0E7005006400450064008500640E1
:104ED0000C50064010500640145006401850064032
:104EE0001C500640205006402450064028500640E2
:104EF0002C50064030500640345006403850064092
:104F00003C50064040500640445006404850064041
:104F10004C500640505006405450064058500640F1
:104F20005C500640605006406450064068500640A1
:104F30006C50064070500640745006407850064051
:104F40007C50064080500640845006408850064001
:104F50008C500640905006409450064098500640B1
:104F60009C500640A0500640A4500640A850064061
:104F7000AC500640B0500640B4500640B850064011
:104F8000BC500640C0500640C4500640C8500640C1
:104F9000CC500640D0500640005006400450064019
:104FA000085006400C500640105006401450064071
:104FB000185006401C500640205006402450064021
:104FC000285006402C5006403050064034500640D1
:104FD000385006403C500640405006404450064081
:104FE000485006404C500640505006405450064031
:104FF000585006405C5006406050064064500640E1
:10500000685006406C500640705006407450064090
:10501000785006407C500640805006408450064040
:10502000885006408C5006409050064094500640F0
:10503000985006409C500640A0500640A4500640A0
:10504000A8500640AC500640B0500640B450064050
:10505000B8500640BC500640C0500640C450064000
:10506000C8500640CC500640D050064000F00F40DB
:1050700040F00F4080F00F40C0F00F4000F10F40B3
:105080000090044000A0044000B00440000005402F
:10509000001005400090044000A0044000B004400F
:1050A00000000540001005400C101418203040008E
:1050B00004000000020000000000020000000100E7
:1050C00000000800000010000100000020000000A7
:1050D0004000000080000000000008000000040004
:1050E00000000100000001000000020000000000BC
:1050F00000800000004000000008000000040000E4
:1051000000000040000000800000000420000000BB
:1051100040000000800000000000080000000400C3
:1051200000000100000001000000020000400240F9
:1051300000500240008003400090034000400440C3
:1051400000500440006005400070054000400240EF
:1051500000500240008003400090034000400440A3
:1051600000500440006005400070054000B003405E
:105170000070024000B003400070024000C00240D6
:1051800000D00240000003400010034000C0024075
:1051900000D002400000034000100340000800005F
:1051A0000001000000000000963007772C610EEE31
:1051B000BA51099919C46D078FF46A7035A563E96E
:1051C000A395649E3288DB0EA4B8DC791EE9D5E095
:1051D00088D9D2972B4CB609BD7CB17E072DB8E794
:1051E000911DBF906410B71DF220B06A4871B9F3E9
:1051F000DE41BE847DD4DA1AEBE4DD6D51B5D4F422
:10520000C785D38356986C13C0A86B647AF962FD86
:10521000ECC9658A4F5C0114D96C0663633D0FFAD3
:10522000F50D088DC8206E3B5E10694CE44160D5D9
:10523000727167A2D1E4033C47D4044BFD850DD2C3
:105240006BB50AA5FAA8B5356C98B242D6C9BBDBD6
:1052500040F9BCACE36CD832755CDF45CF0DD6DCD1
:10526000593DD1ABAC30D9263A00DE518051D7C878
:105270001661D0BFB5F4B42123C4B3569995BACF03
:105280000FA5BDB89EB802280888055FB2D90CC624
:1052900024E90BB1877C6F2F114C6858AB1D61C19D
:1052A0003D2D66B69041DC760671DB01BC20D298BC
:1052B0002A10D5EF8985B1711FB5B606A5E4BF9F49
:1052C00033D4B8E8A2C9077834F9000F8EA809963C
:1052D00018980EE1BB0D6A7F2D3D6D08976C6491A7
:1052E000015C63E6F4516B6B62616C1CD8306585C0
:1052F0004E0062F2ED95066C7BA5011BC1F408829D
:1053000057C40FF5C6D9B06550E9B712EAB8BE8BDD
:105310007C88B9FCDF1DDD62492DDA15F37CD38C66
:10532000654CD4FB5861B24DCE51B53A7400BCA364
:10533000E230BBD441A5DF4AD795D83D6DC4D1A496
:10534000FBF4D6D36AE96943FCD96E34468867AD6D
:10535000D0B860DA732D0444E51D03335F4C0AAA0C
:10536000C97C0DDD3C710550AA41022710100BBE0F
:1053700086200CC925B56857B3856F2009D466B956
:105380009FE461CE0EF9DE5E98C9D9292298D0B08B
:10539000B4A8D7C7173DB359810DB42E3B5CBDB738
:1053A000AD6CBAC02083B8EDB6B3BF9A0CE2B603B9
:1053B0009AD2B1743947D5EAAF77D29D1526DB046E
:1053C0008316DC73120B63E3843B64943E6A6D0DB9
:1053D000A85A6A7A0BCF0EE49DFF099327AE000A04
:1053E000B19E077D44930FF0D2A3088768F2011E97
:1053F000FEC206695D5762F7CB67658071366C192E
:10540000E7066B6E761BD4FEE02BD3895A7ADA104E
:10541000CC4ADD676FDFB9F9F9EFBE8E43BEB7172F
:10542000D58EB060E8A3D6D67E93D1A1C4C2D838B9
:1054300052F2DF4FF167BBD16757BCA6DD06B53F1F
:105440004B36B248DA2B0DD84C1B0AAFF64A03365E
:10545000607A0441C3EF60DF55DF67A8EF8E6E31DD
:1054600079BE69468CB361CB1A8366BCA0D26F2526
:1054700036E2685295770CCC03470BBBB916022273
:105480002F260555BE3BBAC5280BBDB2925AB42B88
:10549000046AB35CA7FFD7C231CFD0B58B9ED92C9D
:1054A0001DAEDE5BB0C2649B26F263EC9CA36A7502
:1054B0000A936D02A906099C3F360EEB85670772B9
:1054C00013570005824ABF95147AB8E2AE2BB17B20
:1054D000381BB60C9B8ED2920DBED5E5B7EFDC7CA7
:1054E00021DFDB0BD4D2D38642E2D4F1F8B3DD68FE
:1054F0006E83DA1FCD16BE815B26B9F6E177B06FF9
:105500007747B718E65A0888706A0FFFCA3B0666E5
:105510005C0B0111FF9E658F69AE62F8D3FF6B6172
:1055200045CF6C1678E20AA0EED20DD75483044E14
:10553000C2B30339612667A7F71660D04D476949A2
:10554000DB776E3E4A6AD1AEDC5AD6D9660BDF40B5
:10555000F03BD83753AEBCA9C59EBBDE7FCFB24768
:10556000E9FFB5301CF2BDBD8AC2BACA3093B3534D
:10557000A6A3B4240536D0BA9306D7CD2957DE5456
:10558000BF67D9232E7A66B3B84A61C4021B685D2F
:10559000942B6F2A37BE0BB4A18E0CC31BDF055AA8
:1055A0008DEF022D0002000000000000000003004B
:1055B000000000000000000C0000000300000000DC
:1055C0000D000000030100000302000000000000C5
:1055D00000010500000004010000040000000002BA
:1055E00001000004010000000200000004020000AD
:1055F000000201000000000009000000A4550000A6
:1056000000000100105600000100000000560000DC
:105610000100000010000000010000005E01000019
:105620000200000002000000000000000200000074
:10563000640000003F0000000000000002000000C5
:10564000640000003F000000020000004C10002039
:10565000000704000204000104000004000000012F
:105660000100020101030102CD4100003D420000A2
:105670006400000000000000554500005145000096
:10568000E8030000E50000007D4D0000C14D000072
:10569000102700002F06000000000000000000009E
:1056A00000000000000000000101FEFE0202FDFDFE
:1056B0000303FCFCF83F82F51E00000078B6FF7F74
:1056C00001000000040302040317000002060000AA
:1056D00078000000010100000E0000000000000042
:1056E00008000000040000000300000002000000A9
:1056F00003000000000000000000000002000000A5
:105700000300000002000000010000000100000092
:105710000000000028560000505600000000000065
:105720000100000038560000535600000000000041
:105730000000000000000000010000000000000068
:105740000000000001000000000000000000000058
:105750000100000000000000000000000000000048
:1057600000000000E63400200010000000100000DF
:10577000E6240020001000000010000005000100D9
:10578000BA00000000000000D14B0000BB00000088
:1057900001000000CD4C0000BD0000000001000031
:1057A000F54B0000BC00000000010000354C00007B
:1057B000BE00000000010000914C0000FF0000004E
:1057C00001000000C94C0000BC100020F8100020AF
:1057D00000A0F0F700A0F0F700A0F0F700A0F0F7AD
:1057E00000A0F0F700A0F0F700A0F0F700A0F0F79D
:1057F00000A0F0F700A0F0F700A0F0F700A0F0F78D
:1058000000A0F0F700A0F0F700A0F0F700A0F0F77C
:10FFF00000A0F0F700A0F0F700A0F0F7942AB419E1
:020000040001F9
:100000000000022075030100E5030100E703010081
:10001000E9030100ED030100F1030100000000000D
:10002000000000000000000000000000F5030100D7
:10003000F703010000000000FB0301005B850100E5
:10004000FF03010003040100070401000B04010089
:100050000F04010013040100170401001B04010038
:100060001F04010023040100270401002B040100E8
:100070002F04010033040100370401003B04010098
:100080003F04010043040100470401004B04010048
:100090004F04010053040100570401005B040100F8
:1000A0005F04010063040100670401006B040100A8
:1000B0006F04010073040100E103010077040100F3
:1000C0007B0401007F040100830401008704010018
:1000D000E10301008B0401008F040100930401007F
:1000E000970401009B040100E10301009F0401004B
:1000F000A3040100A7040100AB040100AF04010048
:10010000E1030100B3040100B7040100BB040100D6
:10011000BF040100C3040100C7040100CB040100B7
:10012000CF040100D3040100D7040100DB04010067
:10013000DF040100E3040100E7040100EB04010017
:10014000EF040100F3040100F7040100FB040100C7
:10015000FF04010003050100070501000B05010074
:100160000F05010013050100170501001B05010023
:100170001F05010023050100270501002B050100D3
:100180002F05010033050100370501003B05010083
:100190003F05010043050100470501004B05010033
:1001A0004F05010053050100570501005B050100E3
:1001B0005F05010063050100670501006B05010093
:1001C0006F05010073050100770501007B05010043
:1001D0007F05010083050100870501008B050100F3
:1001E0008F05010093050100970501009B050100A3
:1001F0009F050100A3050100A7050100AB05010053
:10020000AF050100B3050100B7050100BB05010002
:10021000BF050100C3050100C7050100CB050100B2
:10022000CF050100D3050100D7050100DB05010062
:10023000DF050100E3050100E7050100EB05010012
:10024000EF050100F3050100F7050100FB050100C2
:10025000FF05010003060100070601000B0601006F
:100260000F06010013060100170601001B0601001E
:100270001F06010023060100270601002B060100CE
:100280002F06010033060100370601003B0601007E
:100290003F0601004306010047060100E10301009B
:1002A000E1030100E10301004B0601004F060100DC
:1002B00053060100570601005B0601005F060100BE
:1002C00063060100670601006B0601006F0601006E
:1002D00073060100770601007B0601007F0601001E
:1002E00083060100870601008B0601008F060100CE
:1002F00093060100970601009B0601009F0601007E
:10030000A3060100A7060100AB060100AF0601002D
:10031000B3060100B7060100BB060100BF060100DD
:10032000C3060100C7060100CB060100CF0601008D
:10033000D3060100D7060100DB060100DF0601003D
:10034000E3060100E7060100EB060100EF060100ED
:10035000F3060100F7060100FB060100FF0601009D
:1003600003070100070701000B0701000F07010049
:100370001307010072B6E848E84901600A6882F391
:100380000888E74801680F22120511430160BFF396
:100390004F8FBFF36F8FE348E3490160E3480321C8
:1003A000C02302689A4311430160DE480121C90756
:1003B0000160DF488047DF49DF4AE04B9A4204D0C2
:1003C0000868106004310432F8E7DD49DD4A002096
:1003D000914202D008600431FAE762B6DA48004779
:1003E000FFF7FEBFFEE7FEE7FFF7FEBFFFF7FEBF2A
:1003F000FFF7FEBFFEE7FFF7FEBFFEE70000D348B2
:100400000047D3480047D3480047D3480047D34864
:100410000047D3480047D3480047D3480047D34854
:100420000047D3480047D3480047D3480047D34844
:100430000047D3480047D3480047D3480047D34834
:100710000047D348004700BF08ED00E0000001009B
:1007200088ED00E000D007400000739410D007402F
:1007300095940100AC04020090090020A00C002058
:10074000A00C00205861002061890100FB530100CA
:100750000F54010023540100375401004B54010091
:100760005F54010073540100875401009B54010041
:10077000AF540100C3540100D7540100EB540100F1
:10078000FF54010013550100275501003B5501009E
:10079000E1030100E10301008569010071820100AC
:1007A000A1550100ED760100655D0100755D010058
:1007B0000D7401001D7401002D7401004D740100C1
:1007C0003D7401005D7401006D7401007D740100D1
:1007D0009D7401008D740100AD740100BD740100B1
:1007E000CD740100ED740100DD740100FD740100A1
:1007F0000D7501001D7501003D7501002D7501008D
:10080000E1030100E1030100E1030100E103010054
:10081000E1030100E103010081360100953601008A
:10082000A9360100BD360100D1360100E5360100D0
:10083000F93601000D37010021370100353701007D
:10084000493701005D37010071370100853701002C
:1008500099370100AD370100C1370100D5370100DC
:10086000E9370100FD37010011380100253801008A
:10087000393801004D380100613801007538010038
:10088000893801009D380100B1380100C5380100E8
:10089000D9380100ED380100013901001539010096
:1008A000293901003D390100513901006539010044
:1008B000793901008D390100A1390100B5390100F4
:1008C000C9390100DD390100F1390100053A0100A3
:1008D000193A01002D3A0100413A0100553A010050
:1008E000693A01007D3A0100913A0100A53A010000
:1008F000B93A0100CD3A0100E13A0100F53A0100B0
:10090000093B01001D3B0100313B0100453B01005B
:10091000593B01006D3B0100813B0100953B01000B
:10092000A93B0100BD3B0100D13B0100E53B0100BB
:10093000F93B01000D3C0100213C0100353C010068
:10094000493C01005D3C0100713C0100853C010017
:10095000993C0100AD3C0100C13C0100D53C0100C7
:10096000E93C0100FD3C0100113D0100253D010075
:10097000393D01004D3D0100613D0100753D010023
:10098000893D01009D3D0100B13D0100C53D0100D3
:10099000D93D0100ED3D0100617F0100717F010043
:1009A000817F0100917F0100A17F0100B17F0100E3
:1009B000C17F0100D17F0100E17F0100F17F0100D3
:1009C00001800100118001002180010031800100BF
:1009D0004180010051800100737C0100837C010093
:1009E000937C0100A37C01009F5E0100AF5E0100CB
:1009F0007B5601008B5601009B560100AB5601004F
:100A0000BB560100D5770100C56B0100D16B010019
:100A1000E103010077800100694F01007D4F010073
:100A2000914F0100317101003D710100013E010053
:100A30005F6501006F6501007F6501008F65010042
:100A40009F650100AF650100BF650100CF65010032
:100A5000E1030100E1030100754D0100697001002F
:100A600075700100000010B402464FEA82024FF296
:100A70007873C0F2010302EB0302126801F01F0356
:100A80004FF0010404FA03F34FF00004202901D2CF
:100A900013631BE0402901D2D36217E0602908D21A
:100AA000062801D0072801D153670FE04FF0010459
:100AB0000CE0802908D2062801D0072801D113674D
:100AC00004E04FF0010401E04FF00104204610BCA7
:100AD00070474DF8048D4FF00001082801D80146F9
:100AE00022E00F2820D80FF20808D8E800F000BF55
:100AF0001D1D1D1D1D1D1D1D1D090C0F1215181B73
:100B00004FF00C0110E04FF010010DE04FF0140118
:100B10000AE04FF0180107E04FF0200104E04FF029
:100B2000300101E04FF0400108465DF8048B70474A
:100B3000A1B39AB3082801D803462DE00C2804D8A5
:100B40004FF009004FF00C0326E0102804D84FF0B6
:100B50000A004FF010031FE0142804D84FF00B00D8
:100B60004FF0140318E0182804D84FF00C004FF091
:100B7000180311E0202804D84FF00D004FF0200397
:100B80000AE0302804D84FF00E004FF0300303E0A5
:100B90004FF00F004FF0400308601360704710B42F
:100BA00002464FEA82024FF29873C0F2010302EB51
:100BB000030213684FF000021C6804F07F04A14296
:100BC00008D8062802D24FF0400401E04FF080041C
:100BD000A14201D34FF00102B2B9186810F0005FD2
:100BE00012D05B6B4FEA03134FEA137303F101005A
:100BF00003464FEAC30318464FEA900000F1050090
:100C0000814201D84FF00102104610BC704710B469
:100C100001464FEA810108464FF29871C0F2010186
:100C200000EB010001684FF000024FF001030C6877
:100C300044F080440C600C6844F080540C600868F8
:100C400010F0004F0AD00C686FF3DF740C6005E001
:100C500002F10102086810F0006F05D144F640303F
:100C6000C0F24C008242F3D344F64030C0F24C0054
:100C7000824202D34FF0010311E04FF0000208E07E
:100C800002F10102086810F0807F02D04FF00003EB
:100C900005E044F64030C0F24C008242F0D31846E2
:100CA00010BC704710B401464FEA810108464FF26C
:100CB0009871C0F2010100EB010001684FF00002E1
:100CC0004FF001040B686FF31C730B600B686FF33C
:100CD0009E730B6008E002F10102086810F0807F4B
:100CE00002D14FF0000403E042F210708242F2D3CE
:100CF000204610BC704702464FEA820210464FF26F
:100D00009872C0F2010200EB02000268106810F451
:100D1000006F38D061B9D2F8002C4FEA82324FEA26
:100D2000927202F103004FF0010101FA00F22CE08F
:100D300001290CD1D2F8002C4FEAC2224FEA92725C
:100D400002F103004FF0010101FA00F21DE0022957
:100D50000CD1D2F8002C4FEA02224FEA927202F133
:100D600003004FF0010101FA00F20EE0D2F8002C6E
:100D70004FEA42124FEA927202F103004FF0010172
:100D800001FA00F201E04FF00802D0B27047F0B56E
:100D900081B005464FF008064FF4007728464FF023
:100DA0000001FFF7A8FF06EB0000B7FBF0F42846B0
:100DB0004FF00101FFF79FFF06EB0000B7FBF0F0DB
:100DC00004EB0004062D01D0072D15D128464FF065
:100DD0000201FFF790FF06EB0000B7FBF0F004EB19
:100DE000000428464FF00301FFF785FF06EB0000E3
:100DF000B7FBF0F004EB0004E0B201B0F0BD2DE968
:100E0000F04F85B004460D461646039320464FEA40
:100E100080004FF29871C0F2010100EB0100D0F8A0
:100E20000080CDF808804FF008098DF802904FF44B
:100E30000079CDF804904FF0000A4FF000004FF019
:100E4000000B16B14FF000013170062C2CBF0321AE
:100E500001218DF803104FF0000727E0C0B2A5EB89
:100E60000000C5B2F8B201462046FFF744FF9DF8E6
:100E7000028008EB0001DDF80480B8FBF1F00EB150
:100E8000FAB2327085420DD201FB05F05044DDF814
:100E9000088008F1800100EB0100DDF80C80C8F843
:100EA000000007E00AF5007A07F101079DF80380CA
:100EB0004745D3D9062C02D24FF4806001E04FF4AD
:100EC0000060824501D34FF0010B584605B0BDE8E4
:100ED000F08F2DE9F04F87B004468DF807101546C6
:100EE0009B46DDF840A020464FEA80004FF2987202
:100EF000C0F2010200EB020007684FF0000604ABED
:100F00000DF106029DF807102046FFF778FF012833
:100F100002D14FF001062BE16878402802D94FF04A
:100F2000010625E1049800F10809CDF814909DF818
:100F300007102046FFF733FE012802D14FF00106CB
:100F400016E1386810F4006F08D06879012805D1DF
:100F5000D7F8000C40F00040C7F8000C9DF80610D0
:100F60002046FFF7C8FE6A78824202D94FF0010698
:100F7000FEE003AA02A96878FFF7DAFDBAF1000FD4
:100F800071D068784FEAA000C0B202464FF000006E
:100F900031E0049C03464FEA830304F1080403EBA9
:100FA000040304464FEA8404544424784FEA04645A
:100FB00007464FEA870707F1010757443F784FEA92
:100FC000074747EA040407464FEA870707F1020785
:100FD00057443F784FEA072747EA040407464FEA99
:100FE000870707F1030757443F7847EA04041C606A
:100FF00000F10100C0B29042CBD310464FEA80000E
:10100000C0B214E020F0030200F00303C3F10303B5
:1010100003EB020202F03F02D2B2DDF81480424438
:1010200000EB0A031B78137000F10100C0B26A786C
:101030009042E7D3687812E020F0030200F0030347
:10104000C3F1030303EB020202F03F02D2B2DDF868
:10105000148042442B79137000F10100C0B29DF856
:101060000C209042E8D304984FF0000202600498EC
:101070004FF000024260049B029A18686FF313401D
:1010800002F00F024FEA024240EA0200186028789C
:1010900001281BD104982BF060424260049B5868E1
:1010A0006FF35F709DF8488008F007024FEA4272C4
:1010B00040EA02005860049A106840F40010106082
:1010C000049A106840F48000106023E0049B586884
:1010D0006FF39C4040F2FF720BEA02024FEA824239
:1010E00040EA02005860049B58686FF35F709DF8F7
:1010F000488008F007024FEA427240EA0200586056
:10110000049A10686FF355501060049A10686FF3DA
:1011100096501060A878012804D1049A106840F411
:1011200080101060049A10686FF31B601060E878FC
:10113000012804D1049A106840F000401060049B1C
:101140006A7918686FF39E7002F001024FEA8272AA
:1011500040EA02001860049B18686FF31B60DDF81A
:10116000448008F00F024FEA026240EA0200186071
:10117000304607B0BDE8F08F2DE9F04C83B004464F
:101180000E4617469A46DDF828B04FF0000501AB31
:101190000DF1030231462046FFF731FE012802D14E
:1011A0004FF0010546E031462046FFF7F8FC0128E4
:1011B00002D14FF001053DE001984FF000010160C0
:1011C00001984FF000014160012F0ED101982AF0E3
:1011D000604141600199086840F40010086001997D
:1011E00008686FF39650086016E0019A50686FF334
:1011F0009C4040F2FF710AEA01014FEA814140EA56
:1012000001005060019908686FF35550086001991A
:1012100008686FF396500860BBF10F0F0AD0019A6F
:1012200010686FF31B600BF00F014FEA016140EA99
:1012300001001060284603B0BDE8F08CF0B4014610
:101240004FEA81014FF29872C0F2010201EB0201F4
:101250000C6801464FEA81014FF27872C0F2010238
:1012600001EB02010B6803F18002062804D24FF45F
:1012700080774FF0400503E04FF400774FF0800592
:10128000616B41F0805161634FF000010AE00E464E
:101290004FEA860606EB02064FF0000CC6F800C0C7
:1012A00001F10101B942F2D303F508624FF00001E8
:1012B00009E00E464FEA860606EB02064FF0FF37BE
:1012C000376001F10101A942F3D34FF0FF311961F9
:1012D0004FF0FF3159614FF0FF3199614FF0FF310D
:1012E000996401464FEA81014FF29872C0F20102FF
:1012F00001EB0201096801F528624FF000010B467D
:101300004FEA830303EB02034FF000051D6001F178
:1013100001010629F3D301464FEA81014FF2987289
:10132000C0F2010201EB0201096801F52A624FF0E7
:1013300000010B464FEA830303EB02034FF0FF3536
:101340001D6001F101010429F3D301464FEA810137
:101350004FF29872C0F2010201EB0201096801F537
:101360002B624FF000010B464FEA830303EB0203AD
:101370004FF000051D6001F101010C29F3D34FEA84
:1013800080004FF29871C0F2010100EB010000688B
:1013900040F6287100EB01024FF0000108464FEAC9
:1013A000800000EB02004FF00003036001F1010137
:1013B0003629F3D3606B6FF31C706063F0BC704729
:1013C00030B585B0044620464FEA80004FF2787170
:1013D000C0F2010100EB010001680D6A20464FEAEE
:1013E000800040F6A042C2F2000200EB020000685A
:1013F00040F20402C0F2080200EA020005EA000519
:101400000D6205F0040058B34FF04C0014FB00F0DF
:1014100040F6C041C2F2000100EB0100006960B17A
:101420004FF04C0014FB00F040F6C041C2F2000146
:1014300000EB01000069804712E04FF000000290CD
:101440004FF0000001904FF00000009020464FF058
:1014500000034FF001024FF0000101F09EFD002853
:1014600005F4002098B34FF04C0014FB00F040F658
:10147000C041C2F2000100EB010000F1100000F1D8
:101480001000006880B14FF04C0014FB00F040F6F3
:10149000C041C2F2000100EB010000F1100000F1B8
:1014A00010000068804712E04FF0000002904FF0FB
:1014B000000001904FF00000009020464FF0000324
:1014C0004FF001024FF0040101F067FD002805B064
:1014D00030BD00B585B001464FEA81014FF2787208
:1014E000C0F2010201EB020109684FF400320A6206
:1014F0004FF04C0110FB01F140F6C042C2F2000275
:1015000001EB020101F1100101F10801096881B14B
:101510004FF04C0110FB01F040F6C041C2F2000157
:1015200000EB010000F1100000F1080000688047A6
:1015300011E04FF0000102914FF0000101914FF0D6
:10154000000100914FF000034FF001024FF0020143
:1015500001F023FD002805B000BD00B585B00146AF
:101560004FEA81014FF27872C0F2010201EB0201F1
:1015700009684FF480320A624FF04C0110FB01F110
:1015800040F6C042C2F2000201EB020101F110017B
:1015900001F10C01096881B14FF04C0110FB01F021
:1015A00040F6C041C2F2000100EB010000F1100062
:1015B00000F10C000068804711E04FF0000102913B
:1015C0004FF0000101914FF0000100914FF0000336
:1015D0004FF001024FF0030101F0DFFC002805B0DD
:1015E00000BD10B584B0044620464FEA80004FF29B
:1015F0007871C0F2010100EB0100016820464FEA5A
:10160000800040F62072C2F2000200EB02000A6A7B
:1016100002604FF0020008624FF04C0014FB00F033
:1016200040F6C041C2F2000100EB010000F11000E1
:1016300000F10400006880B14FF04C0014FB00F092
:1016400040F6C041C2F2000100EB010000F11000C1
:1016500000F104000068804712E04FF000000290A3
:101660004FF0000001904FF00000009020464FF036
:1016700000034FF001024FF0010101F08EFC002841
:1016800020464FEA800040F62071C2F2000100EBD4
:1016900001004FF00001016004B010BD10B584B02E
:1016A000044620464FEA80004FF27871C0F20101F3
:1016B00000EB0100016820464FEA800040F62072EE
:1016C000C2F2000200EB02000A6A02604FF48010CE
:1016D00008624FF04C0014FB00F040F6C041C2F22B
:1016E000000100EB010000F1100000F1140000689F
:1016F00080B14FF04C0014FB00F040F6C041C2F244
:10170000000100EB010000F1100000F1140000687E
:10171000804712E04FF0000002904FF0000001906F
:101720004FF00000009020464FF000034FF0010200
:101730004FF0050101F031FC002820464FEA8000FF
:1017400040F62071C2F2000100EB01004FF00001F1
:10175000016004B010BD30B585B0044620464FEAA4
:1017600080004FF27871C0F2010100EB01000068C7
:10177000D0F8085BD0F8001B01F4403105EA010500
:10178000C0F8085B05F4803098B34FF04C0014FBB0
:1017900000F040F6C041C2F2000100EB010000F190
:1017A000100000F13400006880B14FF04C0014FBD1
:1017B00000F040F6C041C2F2000100EB010000F170
:1017C000100000F134000068804712E04FF0000084
:1017D00002904FF0000001904FF000000090204672
:1017E0004FF000034FF001024FF00D0101F0D5FB67
:1017F000002805F4003098B34FF04C0014FB00F0C3
:1018000040F6C041C2F2000100EB010000F11000FF
:1018100000F13800006880B14FF04C0014FB00F07C
:1018200040F6C041C2F2000100EB010000F11000DF
:1018300000F138000068804712E04FF0000002908D
:101840004FF0000001904FF00000009020464FF054
:1018500000034FF001024FF00E0101F09EFB002843
:1018600005B030BD00B585B001464FEA81014FF2A9
:101870007872C0F2010201EB020109684FF0010227
:101880000A624FF04C0110FB01F140F6C042C2F277
:10189000000201EB020101F1100101F118010968D8
:1018A00081B14FF04C0110FB01F040F6C041C2F293
:1018B000000100EB010000F1100000F118000068C9
:1018C000804711E04FF0000102914FF000010191BB
:1018D0004FF0000100914FF000034FF001024FF074
:1018E000060101F05AFB002805B000BD30B585B0F7
:1018F000044620464FEA80004FF27871C0F20101A1
:1019000000EB01000068D0F8FC5AD0F8E01A01F4AE
:10191000502105EA0105C0F8FC5A05F4002098B3EF
:101920004FF04C0014FB00F040F6C041C2F2000141
:1019300000EB010000F1100000F12800006880B108
:101940004FF04C0014FB00F040F6C041C2F2000121
:1019500000EB010000F1100000F128000068804752
:1019600012E04FF0000002904FF0000001904FF0A5
:101970000000009020464FF000034FF001024FF0AE
:101980000A0101F00AFB002805F4802098B34FF00B
:101990004C0014FB00F040F6C041C2F2000100EB25
:1019A000010000F1100000F12C00006880B14FF040
:1019B0004C0014FB00F040F6C041C2F2000100EB05
:1019C000010000F1100000F12C000068804712E0D7
:1019D0004FF0000002904FF0000001904FF0000027
:1019E000009020464FF000034FF001024FF00B0132
:1019F00001F0D3FA002805F4803098B34FF04C0082
:101A000014FB00F040F6C041C2F2000100EB0100FF
:101A100000F1100000F13000006880B14FF04C0080
:101A200014FB00F040F6C041C2F2000100EB0100DF
:101A300000F1100000F130000068804712E04FF024
:101A4000000002904FF0000001904FF00000009065
:101A500020464FF000034FF001024FF00C0101F05F
:101A60009CFA002805B030BD2DE9F04C81B0064647
:101A700030464FEA80004FF29871C0F2010100EB4E
:101A80000100D0F800A030464FEA80004FF2787194
:101A9000C0F2010100EB01000468DAF8000000F078
:101AA0007F0000F10100276BA16A07EA0107C7F375
:101AB0000F07102888BF102083464FF00005B4E0C0
:101AC0004FF0010000FA05F000EA0700002800F0DE
:101AD000AA80DAF8000010F0005F7DD0072D7BD8D7
:101AE000052D26D14FF04C0016FB00F040F6C0410A
:101AF000C2F2000100EB010000F1100000F11C0037
:101B0000006880B14FF04C0016FB00F040F6C04179
:101B1000C2F2000100EB010000F1100000F11C0016
:101B20000068804705E0A06A6FF0200100EA01002C
:101B3000A062062D26D14FF04C0016FB00F040F6B7
:101B4000C041C2F2000100EB010000F1100000F101
:101B50002000006880B14FF04C0016FB00F040F60A
:101B6000C041C2F2000100EB010000F1100000F1E1
:101B700020000068804705E0A06A6FF0400100EA9D
:101B80000100A062072D49D14FF04C0016FB00F078
:101B900040F6C041C2F2000100EB010000F110006C
:101BA00000F12400006880B14FF04C0016FB00F0FB
:101BB00040F6C041C2F2000100EB010000F110004C
:101BC00000F124000068804728E0A06A6FF08001DF
:101BD00000EA0100A06221E04FF04C0016FB00F08B
:101BE00040F6C041C2F2000100EB0100006868B19C
:101BF0004FF04C0016FB00F040F6C041C2F200016D
:101C000000EB010001682846884707E04FF001001B
:101C100000FA05F1A06A20EA0100A0624FF001007D
:101C200000FA05F0206305F101055D45FFF448AFBA
:101C300001B0BDE8F08C2DE9F044074638464FEA84
:101C400080004FF29871C0F2010100EB01000168C1
:101C500038464FEA80004FF27872C0F2010200EB82
:101C600002000568086800F07F0000F101002E6B9B
:101C7000A96A06EA01066FF30F06202888BF202014
:101C800082464FF0100433E04FF0010000FA04F0F8
:101C900000EA060028B34FF04C0017FB00F040F6B6
:101CA000C041C2F2000100EB010000F10400006835
:101CB00078B14FF04C0017FB00F040F6C041C2F283
:101CC000000100EB010000F1040001682046884794
:101CD00007E04FF0010000FA04F1A86A20EA0100D1
:101CE000A8624FF0010000FA04F0286304F1010437
:101CF0005445C9D3BDE8F0842DE9F0440746384681
:101D00004FEA80004FF29871C0F2010100EB010030
:101D1000016838464FEA80004FF27872C0F2010243
:101D200000EB02000568086800F07F0000F1010088
:101D3000EE6A696A06EA0106C6F30F06302888BF14
:101D4000302082464FF020043AE0A4F120004FF00A
:101D5000010101FA00F000EA060038B34FF04C0030
:101D600017FB00F040F6C041C2F2000100EB010099
:101D700000F10800006878B14FF04C0017FB00F04C
:101D800040F6C041C2F2000100EB010000F1080082
:101D900001682046884709E0A4F120004FF00101C6
:101DA00001FA00F1686A20EA01006862A4F12000EB
:101DB0004FF0010101FA00F0E86204F10100C4B241
:101DC0005445C2D3BDE8F0842DE9F04407463846B7
:101DD0004FEA80004FF29871C0F2010100EB010060
:101DE000016838464FEA80004FF27872C0F2010273
:101DF00000EB02000568086800F07F0000F10100B8
:101E0000EE6A696A06EA01066FF30F06402888BF8A
:101E1000402082464FF0300439E0A4F120004FF01A
:101E2000010101FA00F000EA060038B34FF04C005F
:101E300017FB00F040F6C041C2F2000100EB0100C8
:101E400000F10C00006878B14FF04C0017FB00F077
:101E500040F6C041C2F2000100EB010000F10C00AD
:101E600001682046884709E0A4F120004FF00101F5
:101E700001FA00F1686A20EA01006862A4F120001A
:101E80004FF0010101FA00F0E86204F10104544549
:101E9000C3D3BDE8F0842DE9F04C81B0064630464E
:101EA0004FEA80004FF29871C0F2010100EB01008F
:101EB000D0F800A030464FEA80004FF27871C0F2AF
:101EC000010100EB01000468DAF8000000F07F0077
:101ED00000F10100276BA16A07EA0107202888BFEB
:101EE000202083464FF00005B6E04FF0010000FAD5
:101EF00005F000EA0700002800F0AC80DAF80000E6
:101F000010F0005F7FD0072D7DD8052D27D14FF031
:101F10004C0016FB00F040F6C041C2F2000100EB9D
:101F2000010000F1100000F11C00006880B14FF0CA
:101F30004C0016FB00F040F6C041C2F2000100EB7D
:101F4000010000F1100000F11C00006880477CE0F7
:101F5000A06A6FF0200100EA0100A06275E0062D82
:101F600027D14FF04C0016FB00F040F6C041C2F202
:101F7000000100EB010000F1100000F120000068FA
:101F800080B14FF04C0016FB00F040F6C041C2F2A9
:101F9000000100EB010000F1100000F120000068DA
:101FA000804752E0A06A6FF0400100EA0100A062A1
:101FB0004BE0072D49D14FF04C0016FB00F040F6E6
:101FC000C041C2F2000100EB010000F1100000F17D
:101FD0002400006880B14FF04C0016FB00F040F682
:101FE000C041C2F2000100EB010000F1100000F15D
:101FF00024000068804728E0A06A6FF0800100EAB2
:102000000100A06221E04FF04C0016FB00F040F60A
:10201000C041C2F2000100EB0100006868B14FF05E
:102020004C0016FB00F040F6C041C2F2000100EB8C
:10203000010001682846884707E04FF0010000FAD8
:1020400005F1A06A20EA0100A0624FF0010000FA49
:1020500005F0206305F101055D45FFF446AF01B0D1
:10206000BDE8F08C2DE9F044064630464FEA80008A
:102070004FF29871C0F2010100EB01000168304697
:102080004FEA80004FF27872C0F2010200EB0200CA
:102090000568086800F07F0000F10100EF6A696AD6
:1020A00007EA0107402888BF402082464FF02004FD
:1020B00039E0A4F120004FF0010101FA00F000EA3C
:1020C000070038B34FF04C0016FB00F040F6C0415B
:1020D000C2F2000100EB010000F10400006878B1D9
:1020E0004FF04C0016FB00F040F6C041C2F2000178
:1020F00000EB010000F1040001682046884709E078
:10210000A4F120004FF0010101FA00F1686A20EA11
:1021100001006862A4F120004FF0010101FA00F013
:10212000E86204F101045445C3D3BDE8F0842DE90D
:10213000F044064630464FEA80004FF29871C0F2F4
:10214000010100EB0100016830464FEA80004FF2C8
:102150007872C0F2010200EB02000568086800F026
:102160007F0000F101006F6FE96E07EA0107602848
:1021700088BF602082464FF040043AE0A4F140005E
:102180004FF0010101FA00F000EA070038B34FF008
:102190004C0016FB00F040F6C041C2F2000100EB1B
:1021A000010000F10800006878B14FF04C0016FB08
:1021B00000F040F6C041C2F2000100EB010000F166
:1021C000080001682046884709E0A4F140004FF06C
:1021D000010101FA00F1E86E20EA0100E866A4F1CD
:1021E00040004FF0010101FA00F0686704F10100BE
:1021F000C4B25445C2D3BDE8F0842DE9F04406468C
:1022000030464FEA80004FF29871C0F2010100EBB6
:102210000100016830464FEA80004FF27872C0F248
:10222000010200EB02000568086800F07F0000F181
:1022300001002F6FA96E07EA0107802828BF8020C0
:1022400082464FF0600439E0A4F160004FF00101D4
:1022500001FA00F000EA070038B34FF04C0016FB1B
:1022600000F040F6C041C2F2000100EB010000F1B5
:102270000C00006878B14FF04C0016FB00F040F6FF
:10228000C041C2F2000100EB010000F10C00016846
:102290002046884709E0A4F160004FF0010101FAEF
:1022A00000F1A86E20EA0100A866A4F160004FF0DA
:1022B000010101FA00F0286704F101045445C3D379
:1022C000BDE8F08400002DE9F04405460E4628469E
:1022D0004FEA80004FF29871C0F2010100EB01005B
:1022E000046828464FEA80004FF27871C0F201017D
:1022F00000EB0100D0F800A04FF00007206810F0BC
:10230000004F0CD12846FEF782FC10B14FF00107B8
:1023100005E0284600F066FA08B14FF0010727BB38
:10232000284600F033FA10B14FF001071DE02846AF
:10233000FEF76DFC10B14FF0010716E0206840F089
:10234000007020604FF0000005E000F101002168FE
:1023500011F0007F03D042F210718842F5D342F2AF
:102360001071884201D34FF00107002F40F0C18067
:10237000206840F4805020602846FEF75FFF4FF051
:102380000000CAF828004FF00000CAF82400062D0B
:1023900001D0072D07D14FF00000CAF86C004FF0B4
:1023A0000000CAF868004FF0FF30CAF830004FF064
:1023B000FF30CAF82C00062D01D0072D07D14FF0B1
:1023C000FF30CAF874004FF0FF30CAF8700040F2D6
:1023D0000700C0F21B00CAF820004FF45020CAF8D2
:1023E000FC0A4FF44030CAF8080B317F20686FF3C5
:1023F000CB2001F001014FEAC12140EA0100206039
:10240000206840F480302060317F206D6FF3DF70F2
:1024100001F001014FEAC17140EA01002065D4F8E2
:10242000000C6FF3CF30C4F8000C317F606B6FF39A
:102430000C3001F001014FEA013140EA0100606314
:10244000307F01284CD1717FD4F8000C6FF311401C
:1024500001F003014FEA014140EA0100C4F8000C19
:10246000B17FD4F8000C6FF3D44001F003014FEAC0
:10247000C14140EA0100C4F8000C062D01D0072D2F
:102480001AD1F17FD4F8000C6FF3975001F00301DB
:102490004FEA815140EA0100C4F8000C96F8201080
:1024A000D4F8000C6FF35A6001F003014FEA416168
:1024B00040EA0100C4F8000C06F10801284600F0CB
:1024C00031FA012802D14FF0010712E006F1240190
:1024D000284600F09DFA01280BD14FF0010708E0D3
:1024E00006F10801284600F0A9F9012801D14FF0B2
:1024F0000107002F54D12846FEF749FC316881427C
:1025000009D8062D02D24FF0400001E04FF08000C4
:102510003168814202D94FF0010741E03068A0F1F3
:10252000010120686FF3060001F07F0140EA01001D
:102530002060F079022803D0206840F40030206049
:102540003079012823D1307FF0B9206840F0005065
:1025500020607179606B6FF31B6001F00F014FEA2F
:10256000016140EA01006063B17920686FF3CF3008
:1025700001F001014FEAC13140EA010020604FF053
:10258000FF30CAF848000BE04FF0010708E0206870
:102590006FF35D702060B079012801D14FF0010721
:1025A000002F52D1206840F480202060F179284625
:1025B00000F087F810B14FF0010746E0F0790328EA
:1025C00025D02846FEF76EFB10B14FF001073CE026
:1025D00028464FEA80004FF29871C0F2010100EBEB
:1025E00001000068416B41F000514163D0F8E01AEE
:1025F0006FF3DF71C0F8E01AD0F8E01A6FF3C7117B
:10260000C0F8E01A416B6FF35D7141631DE028462D
:102610004FEA80004FF29871C0F2010100EB010017
:102620000068416B41F000514163D0F8E01A6FF34C
:10263000DF71C0F8E01AD0F8E01A6FF3C711C0F8E4
:10264000E01A416B6FF35D7141633846BDE8F08479
:1026500070B584B0054628464FEA80004FF2987165
:10266000C0F2010100EB010006684FF000044FF0DA
:10267000000002904FF0000001904FF00000009029
:1026800028464FF000034FF001024FF0100100F018
:1026900084FC10B14FF0010410E0306810F0004FDE
:1026A0000CD12846FEF7B3FA10B14FF0010405E053
:1026B000284600F097F808B14FF00104204604B016
:1026C00070BD2DE9F04581B007468A4638464FEA8D
:1026D00080004FF29871C0F2010100EB0100046824
:1026E00025684FEAC5154FEAD5754FF000062DB99C
:1026F0003846FEF78CFA08B14FF00106B6BB5046DB
:10270000042833D80FF20408D8E800F00310193079
:102710002C0060686FF3C300606060686FF30C307A
:10272000606020686FF3D75020601FE0606840F061
:102730000800606060686FF30C30606016E06068ED
:102740006FF3C3006060606840F480506060206890
:102750006FF351402060D4F8000C6FF3CF30C4F811
:10276000000C03E0206840F0004020604EB9BAF150
:10277000030F06D02DB93846FEF794FA08B14FF092
:102780000106304601B0BDE8F085000010B40146F6
:102790004FEA810108464FF29871C0F2010100EB47
:1027A000010001684FF000024FF00004086810F4C7
:1027B000801F14D00B686FF3DF730B6005E002F12C
:1027C0000102086810F4801F03D042F210708242A8
:1027D000F5D342F21070824201D34FF0010420463B
:1027E00010BC704710B401464FEA810108464FF211
:1027F0009871C0F2010100EB010001684FF0000286
:102800004FF00004086810F0004F14D10B6843F03B
:1028100000430B6005E002F10102086810F4801F1C
:1028200003D142F210708242F5D342F2107082421C
:1028300001D34FF00104204610BC70472DE9F0444D
:1028400082460D4650464FEA80004FF29871C0F222
:10285000010100EB0100046826684FEAC6164FEA42
:10286000D6764FF000072EB95046FEF7D0F908B1E2
:102870004FF00107002F52D1286838B1686828B19D
:10288000A86818B1E86808B1286910B94FF00107C5
:1028900045E02868A0F1010160686FF3020001F0D3
:1028A000070140EA01006060A868A0F101016068CA
:1028B0006FF3124001F007014FEA014140EA0100C5
:1028C00060606868A0F1010160686FF3D54001F0B5
:1028D00007014FEAC14140EA01006060E868A0F1E9
:1028E000010160686FF31F6001F0FF014FEA0161B1
:1028F00040EA010060602869A0F1010160686FF39F
:10290000975001F003014FEA815140EA01006060F5
:102910002EB95046FEF7C6F908B14FF00107384608
:10292000BDE8F0842DE9F04482460D4650464FEA5A
:1029300080004FF29871C0F2010100EB01000468C1
:1029400026684FEAC6164FEAD6764FF000072EB932
:102950005046FEF75CF908B14FF00107002F54D143
:10296000286838B1686828B1A86818B1E86808B163
:10297000286910B94FF0010747E02868A0F101016C
:10298000206D6FF38F2001F03F014FEA812140EA73
:1029900001002065A868A0F10101206D6FF304001B
:1029A00001F01F0140EA010020656868A0F1010103
:1029B000206D6FF3491001F01F014FEA411140EA09
:1029C00001002065E868A0F10101206D6FF35E5001
:1029D00040F2FF3201EA02014FEA415140EA0100B0
:1029E00020652869A0F10101206D6FF3144001F00A
:1029F0001F014FEA014140EA010020652EB950460F
:102A0000FEF750F908B14FF001073846BDE8F084F1
:102A10002DE9F04482460D4650464FEA80004FF2C1
:102A20009871C0F2010100EB0100046826684FEACA
:102A3000C6164FEAD6764FF000072EB95046FEF77D
:102A4000E6F808B14FF00107002F5CD1286838B1D3
:102A5000686828B1A86818B1E86808B1286910B991
:102A60004FF0010748E02968D4F8040C6FF38E207A
:102A700001F01F014FEA812140EA0100C4F8040C73
:102A8000A868A0F10101D4F8040C6FF3020001F072
:102A9000070140EA0100C4F8040C6868A0F10101D4
:102AA000D4F8040C6FF3471001F007014FEA41110D
:102AB00040EA0100C4F8040CE868A0F10101D4F870
:102AC000040C6FF31D5040F2FF3201EA02014FEA9D
:102AD000015140EA0100C4F8040C2869A0F1010189
:102AE000D4F8040C6FF3124001F007014FEA0141E2
:102AF00040EA0100C4F8040C2EB95046FEF7D2F8A3
:102B000008B14FF001073846BDE8F0842DE9F044E4
:102B100007468A4638464FEA80004FF29871C0F265
:102B2000010100EB0100066834684FEAC4144FEA63
:102B3000D4744FF000052CB93846FEF768F808B198
:102B40004FF0010585B930686FF310400AF00101BC
:102B50004FEA014140EA010030602CB93846FEF7E7
:102B6000A1F808B14FF001052846BDE8F084000047
:102B70002DE9F04D82B004468DF8071017469B46AC
:102B800020464FEA80004FF29872C0F2010200EB3B
:102B90000200026820464FEA80004FF27873C0F2CC
:102BA000010300EB0300D0F800A04FF00006156809
:102BB0004FEAC5154FEAD57539462046FDF7EFFFB8
:102BC00010B14FF0010606E02DB92046FEF71FF8C0
:102BD00008B14FF0010636BB9DF80780B8F1000F31
:102BE00010D138464FEA80000AF5086200EB020077
:102BF0004FEA8B4240F20003C1F6FC7302EA030283
:102C0000026009E038464FEA80000AF5086200EBEE
:102C100002002BF0604202602DB92046FEF742F818
:102C200008B14FF00106304602B0BDE8F08D00005B
:102C3000F0B583B004460D4616461F462946204689
:102C4000FDF711FF10B14FF0010021E04FF00F0030
:102C500000903B46324629462046FEF78DFA40B9A1
:102C60004FF0000000903B46324629462046FEF7D2
:102C700083FA18B929462046FDF7F5FE40B94FF012
:102C8000040000903B46324629462046FEF774FA7F
:102C900003B0F0BD2DE9F04486B004460D4616465B
:102CA0001F46DDF830A04FF0000005AB0DF1130218
:102CB00029462046FEF7A3F8012802D14FF0010073
:102CC0002CE029462046FDF76AFF012802D14FF08B
:102CD000010023E0059800684FEA00104FEA1070E9
:102CE00030B1082804D0092802D04FF0020015E0C6
:102CF00029462046FDF7B7FE10B14FF001000DE068
:102D00004FF0000002904FF00C000190CDF800A0B1
:102D10003B46324629462046FEF7DBF806B0BDE8C2
:102D2000F084F0B583B004460D4616461F464FF0BA
:102D3000000001AB0DF1030229462046FEF75FF8C3
:102D4000012802D14FF001001CE029462046FDF782
:102D500026FF012802D14FF0010013E0019800681E
:102D60004FEA00104FEA107030B1082804D009284B
:102D700002D04FF0020005E03B463246294620468D
:102D8000FFF756FF03B0F0BD2DE9F04C83B00446C9
:102D90008A46174620464FEA80004FF27871C0F20B
:102DA000010100EB010006684FF0000501AB0DF1D9
:102DB00003025FFA8AF001462046FEF720F8012858
:102DC00002D14FF001050AE0019800F1080B5146CD
:102DD0002046FDF7E4FE012801D14FF00105002D4A
:102DE00040F0AF8001980068019800684FEA003019
:102DF0004FEA1070FDF76DFE82469DF803102046E5
:102E0000FDF779FF824505D99DF803102046FDF7AF
:102E100072FF824687F848A00198006838600198E0
:102E2000006810F4001F05D00198406820F0604051
:102E3000786006E0019840684FEAC0004FEA5050C1
:102E400078604FEAAA00C0B201464FF000005AE095
:102E50004FEA800207F1080302EB0302019C0346DC
:102E60004FEA830304F1080403EB04031B6803F037
:102E70007F434FEA1363DBB2137007F1080202F1DC
:102E800001024FEA800303EB0202019C03464FEA72
:102E9000830304F1080403EB04031B6803F47F03BA
:102EA0004FEA1343DBB2137007F1080202F102028A
:102EB0004FEA800303EB0202019C03464FEA8303BF
:102EC00004F1080403EB04031B6803F47F434FEA97
:102ED0001323DBB2137007F1080202F103024FEA79
:102EE000800303EB0202019C03464FEA830304F1D3
:102EF000080403EB04031B6803F0FF03DBB2137049
:102F000000F10100C0B28842A2D34FEA8100C0B2F2
:102F100014E020F0030100F00302C2F1030202EB0F
:102F2000010101F03F01C9B207F1080200EB020202
:102F300059440978117000F10100C0B25045E8D33E
:102F4000B068284603B0BDE8F08C00000000000027
:102F5000000000000000000010B44FF0000306283D
:102F600002D34FF0010315E0032902D94FF001030A
:102F700010E04FF04C0410FB04F040F6C044C2F2E5
:102F8000000400EB04000C464FEA8404214601EBE8
:102F900000000260184610BC70472DE9F04F83B066
:102FA00005460C461646019328464FEA80004FF22C
:102FB0009871C0F2010100EB0100D0F800A0284692
:102FC0004FEA80004FF27871C0F2010100EB01007E
:102FD0000768DAF800B04FEACB1B4FEADB7B4FF013
:102FE00000098DF80390BBF1000F07D12846FDF7CB
:102FF0000EFE18B14FF001098DF803909DF8038083
:10300000B8F1000F40F0B5822046102800F2A682E9
:103010000FF20408D8E810F04E004E009B009B0011
:10302000F400F40041018E018E018E01AD01AD016D
:10303000AD01DC01DC011100FF01EEB9B86ADDF879
:10304000048040EA0800B862786ADDF8308040EA1F
:1030500008007862062D02D0072D40F07F82F86EBE
:10306000DDF8348040EA0800F866B86EDDF8388094
:1030700040EA0800B86671E2B86ADDF8048020EA28
:103080000800B862786ADDF8308020EA08007862CB
:10309000062D02D0072D40F06182F86EDDF83480F5
:1030A00020EA0800F866B86EDDF8388020EA0800EB
:1030B000B86653E22EBB20464FEA80004FF2F4710F
:1030C000C0F2010100EB010228464FEA800040F601
:1030D000A041C2F2000100EB01010868126840EA59
:1030E0000200086020464FEA80004FF2B871C0F23B
:1030F000010100EB01017868096840EA010078608D
:103100002CE220464FEA80004FF2B871C0F2010174
:1031100000EB01017868096820EA01007860204628
:103120004FEA80004FF2F471C0F2010100EB01029E
:1031300028464FEA800040F6A041C2F2000100EBB1
:1031400001010868126820EA0200086006E25EBB1E
:10315000DAF8000040F40010CAF8000020464FEAF8
:1031600080004FF2F471C0F2010100EB0102284629
:103170004FEA800040F6A041C2F2000100EB0101DD
:103180000868126840EA0200086020464FEA8000A2
:103190004FF2B871C0F2010100EB010178680968D3
:1031A00040EA01007860D9E1DAF800006FF3555089
:1031B000CAF8000020464FEA80004FF2B871C0F212
:1031C000010100EB01017868096820EA01007860DC
:1031D00020464FEA80004FF2F471C0F2010100EB8B
:1031E000010228464FEA800040F6A041C2F20001E9
:1031F00000EB01010868126820EA02000860ADE1F6
:103200002EBB20464FEA80004FF2F471C0F201015C
:1032100000EB010228464FEA800040F6A041C2F2CE
:10322000000100EB01010868126840EA0200086032
:1032300020464FEA80004FF2B871C0F2010100EB66
:103240000101786B096840EA0100786386E1204655
:103250004FEA80004FF2B871C0F2010100EB0101AA
:10326000786B096820EA0100786320464FEA800005
:103270004FF2F471C0F2010100EB010228464FEA5F
:10328000800040F6A041C2F2000100EB0101086895
:10329000126820EA0200086060E12EBB20464FEA77
:1032A00080004FF2F471C0F2010100EB01022846E8
:1032B0004FEA800040F6A041C2F2000100EB01019C
:1032C0000868126840EA0200086020464FEA800061
:1032D0004FF2B871C0F2010100EB010138680968D2
:1032E00040EA0100386039E120464FEA80004FF2A1
:1032F000B871C0F2010100EB01013868096820EAE9
:103300000100386020464FEA80004FF2F471C0F2AD
:10331000010100EB010228464FEA800040F6A0417F
:10332000C2F2000100EB01010868126820EA020005
:10333000086013E176B920464FEA80004FF2B87179
:10334000C0F2010100EB0101B86A096840EA01001E
:10335000B86203E120464FEA80004FF2B871C0F234
:10336000010100EB0101B86A096820EA0100B862B6
:10337000F4E0DAF8340040F00050CAF83400DAF82B
:10338000E00A6FF3DF70CAF8E00A86B920464FEA18
:1033900080004FF2B871C0F2010100EB0101D7F8D3
:1033A000E00A096840EA0100C7F8E00AD6E02046D2
:1033B0004FEA80004FF2B871C0F2010100EB010149
:1033C000D7F8E00A096820EA0100C7F8E00AC5E07A
:1033D00086B920464FEA80004FF2B871C0F2010171
:1033E00000EB0101D7F8000B096840EA0100C7F8BB
:1033F000000BB3E020464FEA80004FF2B871C0F2F4
:10340000010100EB0101D7F8000B096820EA010077
:10341000C7F8000BA2E0002E4ED128464FEA8000EC
:1034200040F6A041C2F2000100EB010040F20701AA
:10343000C0F21B010160B86A40F0FF30B862786AE0
:1034400040F0FF307862062D01D0072D07D1F86ECD
:1034500040F0FF30F866B86E40F0FF30B86678682C
:1034600040F44C407860786B40F040407863DAF884
:10347000340040F00050CAF83400DAF8E00A6FF384
:10348000DF70CAF8E00AD7F8E00A40F45020C7F825
:10349000E00ADAF8000040F08060CAF80000DAF8CC
:1034A000000040F40010CAF80000D7F8000B40F408
:1034B0004030C7F8000B51E0B86A00F00000B86275
:1034C000786A00F000007862062D01D0072D07D140
:1034D000F86E00F00000F866B86E00F00000B86604
:1034E00078686FF44C4100EA01007860786B20F056
:1034F00040407863DAF8340040F00050CAF83400F5
:10350000DAF8E00A6FF3DF70CAF8E00AD7F8E00AE9
:103510006FF4502100EA0100C7F8E00ADAF8000071
:103520006FF39A60CAF80000DAF800006FF35550A4
:10353000CAF80000D7F8000B6FF4403100EA010030
:10354000C7F8000B28464FEA800040F6A041C2F2BF
:10355000000100EB01004FF000010160BBF1000F22
:1035600007D12846FDF79EFB18B14FF001098DF8F1
:1035700003909DF8030003B0BDE8F08F10B403463C
:103580004FEA83034FF27874C0F2010403EB0403A3
:103590001B684FF00004202912D242B94FF00100FD
:1035A00000FA01F1986A40EA0100986263E04FF086
:1035B000010000FA01F1986A20EA010098625AE0DD
:1035C000402916D252B9A1F120004FF0010101FAB1
:1035D00000F1586A40EA010058624CE0A1F1200075
:1035E0004FF0010101FA00F1586A20EA0100586227
:1035F00041E060291DD2062801D0072816D152B912
:10360000A1F140004FF0010101FA00F1D86E40EA4B
:103610000100D8662FE0A1F140004FF0010101FA4E
:1036200000F1D86E20EA0100D86624E04FF00104D2
:1036300021E080291DD2062801D0072816D152B9D1
:10364000A1F160004FF0010101FA00F1986E40EA2B
:10365000010098660FE0A1F160004FF0010101FA4E
:1036600000F1986E20EA0100986604E04FF0010432
:1036700001E04FF00104204610BC7047000000003C
:1036800000B581B04FF00000FDF79AFEBFF34F8FF9
:1036900001B000BD00B581B04FF00000FDF719FF8B
:1036A000BFF34F8F01B000BD00B581B04FF00000F7
:1036B000FDF753FFBFF34F8F01B000BD00B581B0E0
:1036C0004FF00000FDF78DFFBFF34F8F01B000BD3D
:1036D00000B581B04FF00000FDF7E0FFBFF34F8F62
:1036E00001B000BD00B581B04FF00000FEF733F827
:1036F000BFF34F8F01B000BD00B581B04FF00000A7
:10370000FEF7B0F8BFF34F8F01B000BD00B581B038
:103710004FF00000FEF7EAF8BFF34F8F01B000BD95
:1037200000B581B04FF00000FEF79EF9BFF34F8F58
:1037300001B000BD00B581B04FF00000FEF77BFA8C
:10374000BFF34F8F01B000BD00B581B04FF0000056
:10375000FEF7D2FABFF34F8F01B000BD00B581B0C4
:103760004FF00000FEF730FBBFF34F8F01B000BDFC
:1037700000B581B04FF00100FDF722FEBFF34F8F7F
:1037800001B000BD00B581B04FF00100FDF7A1FE12
:10379000BFF34F8F01B000BD00B581B04FF0010005
:1037A000FDF7DBFEBFF34F8F01B000BD00B581B068
:1037B0004FF00100FDF715FFBFF34F8F01B000BDC3
:1037C00000B581B04FF00100FDF768FFBFF34F8FE8
:1037D00001B000BD00B581B04FF00100FDF7BBFFA7
:1037E000BFF34F8F01B000BD00B581B04FF00100B5
:1037F000FEF738F8BFF34F8F01B000BD00B581B0C0
:103800004FF00100FEF772F8BFF34F8F01B000BD1B
:1038100000B581B04FF00100FEF726F9BFF34F8FDE
:1038200001B000BD00B581B04FF00100FEF703FA12
:10383000BFF34F8F01B000BD00B581B04FF0010064
:10384000FEF75AFABFF34F8F01B000BD00B581B04B
:103850004FF00100FEF7B8FABFF34F8F01B000BD83
:1038600000B581B04FF00200FDF7AAFDBFF34F8F06
:1038700001B000BD00B581B04FF00200FDF729FE98
:10388000BFF34F8F01B000BD00B581B04FF0020013
:10389000FDF763FEBFF34F8F01B000BD00B581B0EF
:1038A0004FF00200FDF79DFEBFF34F8F01B000BD4A
:1038B00000B581B04FF00200FDF7F0FEBFF34F8F6F
:1038C00001B000BD00B581B04FF00200FDF743FF2D
:1038D000BFF34F8F01B000BD00B581B04FF00200C3
:1038E000FDF7C0FFBFF34F8F01B000BD00B581B041
:1038F0004FF00200FDF7FAFFBFF34F8F01B000BD9C
:1039000000B581B04FF00200FEF7AEF8BFF34F8F65
:1039100001B000BD00B581B04FF00200FEF78BF999
:10392000BFF34F8F01B000BD00B581B04FF0020072
:10393000FEF7E2F9BFF34F8F01B000BD00B581B0D3
:103940004FF00200FEF740FABFF34F8F01B000BD09
:1039500000B581B04FF00300FDF732FDBFF34F8F8C
:1039600001B000BD00B581B04FF00300FDF7B1FD1F
:10397000BFF34F8F01B000BD00B581B04FF0030021
:10398000FDF7EBFDBFF34F8F01B000BD00B581B077
:103990004FF00300FDF725FEBFF34F8F01B000BDD0
:1039A00000B581B04FF00300FDF778FEBFF34F8FF5
:1039B00001B000BD00B581B04FF00300FDF7CBFEB4
:1039C000BFF34F8F01B000BD00B581B04FF00300D1
:1039D000FDF748FFBFF34F8F01B000BD00B581B0C8
:1039E0004FF00300FDF782FFBFF34F8F01B000BD22
:1039F00000B581B04FF00300FEF736F8BFF34F8FEC
:103A000001B000BD00B581B04FF00300FEF713F91F
:103A1000BFF34F8F01B000BD00B581B04FF0030080
:103A2000FEF76AF9BFF34F8F01B000BD00B581B05A
:103A30004FF00300FEF7C8F9BFF34F8F01B000BD90
:103A400000B581B04FF00400FDF7BAFCBFF34F8F13
:103A500001B000BD00B581B04FF00400FDF739FDA5
:103A6000BFF34F8F01B000BD00B581B04FF004002F
:103A7000FDF773FDBFF34F8F01B000BD00B581B0FE
:103A80004FF00400FDF7ADFDBFF34F8F01B000BD57
:103A900000B581B04FF00400FDF700FEBFF34F8F7B
:103AA00001B000BD00B581B04FF00400FDF753FE3A
:103AB000BFF34F8F01B000BD00B581B04FF00400DF
:103AC000FDF7D0FEBFF34F8F01B000BD00B581B050
:103AD0004FF00400FDF70AFFBFF34F8F01B000BDA8
:103AE00000B581B04FF00400FDF7BEFFBFF34F8F6C
:103AF00001B000BD00B581B04FF00400FEF79BF8A7
:103B0000BFF34F8F01B000BD00B581B04FF004008E
:103B1000FEF7F2F8BFF34F8F01B000BD00B581B0E2
:103B20004FF00400FEF750F9BFF34F8F01B000BD16
:103B300000B581B04FF00500FDF742FCBFF34F8F99
:103B400001B000BD00B581B04FF00500FDF7C1FC2C
:103B5000BFF34F8F01B000BD00B581B04FF005003D
:103B6000FDF7FBFCBFF34F8F01B000BD00B581B086
:103B70004FF00500FDF735FDBFF34F8F01B000BDDD
:103B800000B581B04FF00500FDF788FDBFF34F8F02
:103B900001B000BD00B581B04FF00500FDF7DBFDC1
:103BA000BFF34F8F01B000BD00B581B04FF00500ED
:103BB000FDF758FEBFF34F8F01B000BD00B581B0D7
:103BC0004FF00500FDF792FEBFF34F8F01B000BD2F
:103BD00000B581B04FF00500FDF746FFBFF34F8FF2
:103BE00001B000BD00B581B04FF00500FEF723F82D
:103BF000BFF34F8F01B000BD00B581B04FF005009D
:103C0000FEF77AF8BFF34F8F01B000BD00B581B069
:103C10004FF00500FEF7D8F8BFF34F8F01B000BD9D
:103C200000B581B04FF00600FDF7CAFBBFF34F8F20
:103C300001B000BD00B581B04FF00600FDF749FCB2
:103C4000BFF34F8F01B000BD00B581B04FF006004B
:103C5000FDF783FCBFF34F8F01B000BD00B581B00D
:103C60004FF00600FDF7BDFCBFF34F8F01B000BD64
:103C700000B581B04FF00600FDF710FDBFF34F8F88
:103C800001B000BD00B581B04FF00600FDF763FD47
:103C9000BFF34F8F01B000BD00B581B04FF00600FB
:103CA000FDF7E0FDBFF34F8F01B000BD00B581B05F
:103CB0004FF00600FDF71AFEBFF34F8F01B000BDB5
:103CC00000B581B04FF00600FEF7E5F8BFF34F8F67
:103CD00001B000BD00B581B04FF00600FEF7C2F99B
:103CE000BFF34F8F01B000BD00B581B04FF00600AB
:103CF000FEF71DFABFF34F8F01B000BD00B581B0D4
:103D00004FF00600FEF779FABFF34F8F01B000BD08
:103D100000B581B04FF00700FDF752FBBFF34F8FA6
:103D200001B000BD00B581B04FF00700FDF7D1FB39
:103D3000BFF34F8F01B000BD00B581B04FF0070059
:103D4000FDF70BFCBFF34F8F01B000BD00B581B094
:103D50004FF00700FDF745FCBFF34F8F01B000BDEA
:103D600000B581B04FF00700FDF798FCBFF34F8F0F
:103D700001B000BD00B581B04FF00700FDF7EBFCCE
:103D8000BFF34F8F01B000BD00B581B04FF0070009
:103D9000FDF768FDBFF34F8F01B000BD00B581B0E6
:103DA0004FF00700FDF7A2FDBFF34F8F01B000BD3C
:103DB00000B581B04FF00700FEF76DF8BFF34F8FED
:103DC00001B000BD00B581B04FF00700FEF74AF921
:103DD000BFF34F8F01B000BD00B581B04FF00700B9
:103DE000FEF7A5F9BFF34F8F01B000BD00B581B05C
:103DF0004FF00700FEF701FABFF34F8F01B000BD8F
:103E00002DE9004144F21408C4F20608D8F8000075
:103E100010F4802F2FD044F21408C4F20608D8F80A
:103E2000000010F0004F07D04FF0B64044F21408E5
:103E3000C4F20608C8F8000044F21408C4F20608E8
:103E4000D8F8000040F0004044F21408C4F206081C
:103E5000C8F8000040F64078C2F20008D8F8000028
:103E600038B140F64078C2F20008D8F80000804728
:103E700001E000F0B0FB44F21C08C4F20608D8F8D8
:103E8000000010F4802F31D044F21C08C4F2060860
:103E9000D8F8000010F0004F07D04FF0B64044F2C1
:103EA0001C08C4F20608C8F8000044F21C08C4F25A
:103EB0000608D8F8000040F0004044F21C08C4F2A4
:103EC0000608C8F8000040F64070C2F2000000F199
:103ED0000400006840B140F64070C2F2000000F1FA
:103EE00004000068804701E000F0A1FBBFF34F8FA2
:103EF000BDE800812DE9004144F21C08C4F2060827
:103F0000D8F8001011F0004F07D04FF0B64144F23E
:103F10001C08C4F20608C8F8001044F21C08C4F2D9
:103F20000608D8F800106FF4802201EA02016FF051
:103F3000020201EA02014FEA400040F0010041EABA
:103F4000000141F0004044F21C08C4F20608C8F821
:103F500000004FF0030000F087FEBDE800812DE96E
:103F6000104181B04FF0000444F23008C4F206085A
:103F7000D8F8001011F0004F07D04FF0B64144F2CE
:103F80003008C4F20608C8F8001044F23008C4F241
:103F90000608D8F8001041F0807144F23008C4F2ED
:103FA0000608C8F8001044F23008C4F20608D8F831
:103FB000001041F0004144F23008C4F20608C8F88D
:103FC000001044F22808C4F20608D8F8001011F0D6
:103FD000004F07D04FF0B64144F22808C4F206085B
:103FE000C8F8001044F22808C4F20608D8F80010F7
:103FF00041F4405144F22808C4F20608C8F8001001
:1040000044F22808C4F20608D8F8001041F4007100
:1040100044F22808C4F20608C8F8001044F2280840
:10402000C4F20608D8F800106FF3410100F0010255
:104030004FEA420241EA020144F22808C4F20608AB
:10404000C8F8001044F22808C4F20608D8F8001096
:1040500041F0010144F22808C4F20608C8F8001033
:1040600044F22808C4F20608D8F8001041F00041D4
:1040700044F22808C4F20608C8F800104FF0050002
:1040800000F0F2FD10B14FF0010431E04FF0B64006
:1040900044F22808C4F20608C8F8000044F22808D0
:1040A000C4F20608D8F8001041F0007144F2280864
:1040B000C4F20608C8F8001044F22808C4F2060842
:1040C000D8F800106FF3492144F22808C4F206081A
:1040D000C8F8001044F22808C4F20608D8F8001006
:1040E00041F0004144F22808C4F20608C8F8001064
:1040F000204601B0BDE810812DE9104181B044F2A5
:104100001808C4F20608D8F8003013F0004F07D0A2
:104110004FF0B64344F21808C4F20608C8F800305D
:1041200044F21808C4F20608D8F800306FF382038E
:1041300000F001044FEA840443EA040344F218083F
:10414000C4F20608C8F8003044F21808C4F20608A1
:10415000D8F800306FF3000302F0010043EA0003D7
:1041600044F21808C4F20608C8F8003044F21808EF
:10417000C4F20608D8F8003043F0020344F21808ED
:10418000C4F20608C8F8003044F21808C4F2060861
:10419000D8F8003043F0004344F21808C4F206088F
:1041A000C8F8003044F21408C4F20608D8F8000039
:1041B00010F0004F07D04FF0B64044F21408C4F29C
:1041C0000608C8F8000044F21408C4F20608D8F83B
:1041D00000306FF4802003EA00036FF0020003EA6E
:1041E00000034FEA410040F0010043EA000343F0BE
:1041F000004044F21408C4F20608C8F800004FF06A
:10420000040000F031FD01B0BDE810812DE910413E
:1042100081B04FF0000401283BD14FF0030000F0C3
:1042200023FD08B14FF00104002C40F0AD8044F2B2
:104230000C08C4F20608D8F8000010F0004F07D0B0
:104240004FF0B64044F20C08C4F20608C8F800006B
:1042500044F20C08C4F20608D8F800006FF4E0211C
:1042600000EA010040F4803044F20C08C4F2060871
:10427000C8F8000044F20C08C4F20608D8F80000A0
:1042800040F0004044F20C08C4F20608C8F80000F0
:104290007AE002283AD14FF0040000F0E5FC08B1C2
:1042A0004FF00104002C6FD144F20C08C4F2060850
:1042B000D8F8000010F0004F07D04FF0B64044F29D
:1042C0000C08C4F20608C8F8000044F20C08C4F256
:1042D0000608D8F800006FF4E02100EA010040F47D
:1042E000003044F20C08C4F20608C8F8000044F29A
:1042F0000C08C4F20608D8F8000040F0004044F270
:104300000C08C4F20608C8F800003DE0032839D1C3
:104310004FF0050000F0A8FC08B14FF001049CBB71
:1043200044F20C08C4F20608D8F8000010F0004F60
:1043300007D04FF0B64044F20C08C4F20608C8F8A3
:10434000000044F20C08C4F20608D8F800006FF42C
:10435000E02100EA010040F4403044F20C08C4F2CD
:104360000608C8F8000044F20C08C4F20608D8F8A1
:10437000000040F0004044F20C08C4F20608C8F8FF
:10438000000001E04FF00104204601B0BDE81081BB
:1043900000004DF8048D44F22808C4F20608D8F84D
:1043A000000010F0004F07D04FF0B64044F228084C
:1043B000C4F20608C8F8000044F22808C4F206084F
:1043C000D8F800006FF3000044F22808C4F2060891
:1043D000C8F8000044F22808C4F20608D8F8000023
:1043E0006FF3596044F22808C4F20608C8F80000C8
:1043F00044F22808C4F20608D8F8000040F0004053
:1044000044F22808C4F20608C8F800005DF8048BDE
:1044100070474DF8048D44F22C08C4F20608D8F811
:10442000001011F0004F07D04FF0B64144F22C08B5
:10443000C4F20608C8F80010427844F22C08C4F20E
:104440000608D8F800106FF3124102F007024FEA95
:10445000024241EA020144F22C08C4F20608C8F8FC
:104460000010027844F22C08C4F20608D8F80010B4
:104470006FF3010102F0030241EA020144F22C0849
:10448000C4F20608C8F80010426844F22C08C4F2CE
:104490000608D8F800106FF30F2102F0FF024FEA70
:1044A000022241EA020144F22C08C4F20608C8F8CC
:1044B0000010427A44F22C08C4F20608D8F8001022
:1044C0006FF3041102F001024FEA021241EA020105
:1044D00044F22C08C4F20608C8F80010017A44F22D
:1044E0002C08C4F20608D8F800006FF3451001F05C
:1044F00001014FEA411140EA010044F22C08C4F2E4
:104500000608C8F8000044F22C08C4F20608D8F8DF
:10451000000040F0004044F22C08C4F20608C8F83D
:1045200000005DF8048B70474DF8048D44F21408C8
:10453000C4F20608D8F8000010F0004F07D04FF082
:10454000B64044F21408C4F20608C8F8000044F269
:104550001408C4F20608D8F800006FF4802100EABD
:10456000010020F0010040F0004044F21408C4F2C1
:104570000608C8F8000044F21808C4F20608D8F883
:10458000000010F0004F07D04FF0B64044F218087A
:10459000C4F20608C8F8000044F21808C4F206087D
:1045A000D8F800006FF3410044F21808C4F206087E
:1045B000C8F8000044F21808C4F20608D8F8000051
:1045C00040F0004044F21808C4F20608C8F80000A1
:1045D0005DF8048B70474DF8048D44F21408C4F262
:1045E0000608D8F8000010F0004F07D04FF0B64092
:1045F00044F21408C4F20608C8F8000044F2140893
:10460000C4F20608D8F800006FF4802100EA010027
:104610006FF4007100EA010040F0004044F2140819
:10462000C4F20608C8F800005DF8048B70474DF826
:10463000048D44F21C08C4F20608D8F8000010F0FB
:10464000004F07D04FF0B64044F21C08C4F20608F1
:10465000C8F8000044F21C08C4F20608D8F80000AC
:104660006FF4802100EA01006FF4007100EA01009C
:1046700040F0004044F21C08C4F20608C8F80000EC
:104680005DF8048B70474DF8048D4FEA90024FEAB5
:1046900082024FF63403C0F2010302EB03021368F7
:1046A0000246543A31D2283217D214320AD2043296
:1046B00067D0043265D0043263D0043261D0043252
:1046C0005FD00BE1003A5CD0043A5AD0043A58D09B
:1046D000043A56D0043A54D000E1143A0AD20432D3
:1046E0004FD004324DD004324BD0043249D0043282
:1046F00047D0F3E0003A44D0043A42D0043A40D0E4
:10470000043A3ED0043A3CD0E8E0283A17D21432BA
:104710000AD2043235D0043233D0043231D00432DC
:104720002FD004322DD0D9E0003A2AD0043A28D034
:10473000043A26D0043A24D0043A22D0CEE00C3AEF
:104740000BD2023200F29B8065D0B2F1FF322ED044
:10475000053216D0043214D0C0E02C3A08D204320C
:104760000FD010320DD014320BD0043209D0B5E086
:10477000003A06D0043A04D0043A02D0043A40F099
:10478000AD80186810F0004F02D04FF0B6401860AE
:104790001A686FF30B2201F00F014FEA012142EA80
:1047A00001021A60196841F00041196096E044F274
:1047B0000C08C4F20608D8F8000010F0004F07D02B
:1047C0004FF0B64044F20C08C4F20608C8F80000E6
:1047D00044F20C08C4F20608D8F800206FF47060A8
:1047E00002EA00024FEA012040EA020044F20C080B
:1047F000C4F20608C8F8000044F20C08C4F2060827
:10480000D8F8001041F0004144F20C08C4F2060848
:10481000C8F8001062E044F20C08C4F20608D8F8A8
:10482000000010F0004F07D04FF0B64044F20C08E3
:10483000C4F20608C8F8000044F20C08C4F20608E6
:10484000D8F800206FF0F00002EA00024FEA0110F1
:1048500040EA020044F20C08C4F20608C8F800005E
:1048600044F20C08C4F20608D8F8001041F00041E8
:1048700044F20C08C4F20608C8F800102EE044F216
:104880000C08C4F20608D8F8000010F0004F07D05A
:104890004FF0B64044F20C08C4F20608C8F8000015
:1048A00044F20C08C4F20608D8F8002022F00F02E7
:1048B00041EA020044F20C08C4F20608C8F80000FD
:1048C00044F20C08C4F20608D8F8001041F0004188
:1048D00044F20C08C4F20608C8F800105DF8048B16
:1048E000704710B44FEA90024FEA82024FF6340349
:1048F000C0F2010302EB030212684FF0000304460A
:10490000543C3AD2283418D214340BD204346ED02A
:1049100004346CD004346AD0043468D0043400F019
:1049200050819CE1003C62D0043C60D0043C5ED0ED
:10493000043C5CD0043C5AD091E1143C0FD20434C6
:1049400000F0B080043400F0AD80043400F0AA80A0
:10495000043400F0A780043400F0A4807FE1003C20
:1049600000F0A080043C00F09D80043C00F09A80A0
:10497000043C3CD0043C3AD071E1283C17D21434BA
:104980000AD2043433D0043431D004342FD0043468
:104990002DD004342BD062E1003C28D0043C26D03A
:1049A000043C24D0043C22D0043C20D057E1343CC9
:1049B0000DD2103400F0B780143400F002810434BA
:1049C00000F0FF80083412D0043410D047E1003CDE
:1049D00000F0F780043C00F0F480043C00F0F1802B
:1049E000043C00F0EE80043C00F0EB8037E11068FE
:1049F00010F0004F02D04FF0B640106001290AD1EC
:104A000014686FF3061401F007014FEA011144EA3C
:104A10000104146041E002290AD114686FF30614FE
:104A200001F007014FEA011144EA0104146034E087
:104A300003290AD114686FF3061401F007014FEA45
:104A4000011144EA0104146027E004290AD1146822
:104A50006FF3061401F007014FEA011144EA010463
:104A600014601AE005290AD114686FF3061401F0E6
:104A700007014FEA011144EA010414600DE051B945
:104A800014686FF3061401F007014FEA011144EABC
:104A90000104146001E04FF00103116841F000418E
:104AA0001160DEE0106810F0004F02D04FF0B64009
:104AB000106003290AD114686FF3061401F007018E
:104AC0004FEA011144EA0104146027E004290AD1E5
:104AD00014686FF3061401F007014FEA011144EA6C
:104AE000010414601AE005290AD114686FF3061452
:104AF00001F007014FEA011144EA010414600DE0DE
:104B000051B914686FF3061401F007014FEA01115F
:104B100044EA0104146001E04FF00103116841F020
:104B2000004111609DE0106810F0004F02D04FF07E
:104B3000B640106003290AD114686FF3061401F01F
:104B400007014FEA011144EA0104146034E004292A
:104B50000AD114686FF3061401F007014FEA01113E
:104B600044EA0104146027E005290AD114686FF3B0
:104B7000061401F007014FEA011144EA0104146030
:104B80001AE006290AD114686FF3061401F0070130
:104B90004FEA011144EA010414600DE051B91468B0
:104BA0006FF3061401F007014FEA011144EA010412
:104BB000146001E04FF00103116841F00041116001
:104BC0004FE0106810F0004F02D04FF0B640106078
:104BD00001290AD114686FF3061401F007014FEAA6
:104BE000011144EA0104146034E002290AD1146876
:104BF0006FF3061401F007014FEA011144EA0104C2
:104C0000146027E003290AD114686FF3061401F039
:104C100007014FEA011144EA010414601AE0042973
:104C20000AD114686FF3061401F007014FEA01116D
:104C300044EA010414600DE051B914686FF30614DE
:104C400001F007014FEA011144EA0104146001E098
:104C50004FF00103116841F00041116001E04FF095
:104C60000103184610BC70474DF8048D4FF0000149
:104C70004FF000020346052B75D80FF20808D8E85C
:104C800003F000BF7204060507080EE022E036E0DC
:104C90004AE05EE048F2A060C0F20100814202D921
:104CA0004FF0010261E001F101014DF20408C4F28C
:104CB0000708D8F8000010F0040FEBD055E048F2D8
:104CC000A060C0F20100814202D94FF001024CE025
:104CD00001F1010144F21C08C4F20608D8F80000F2
:104CE00010F4803FEBD040E044F64030C0F24C007E
:104CF000814202D94FF0010237E001F1010149F28E
:104D00000008C4F20708D8F8000010F4007FEBD0C8
:104D10002BE048F2A060C0F20100814202D94FF0BE
:104D2000010222E001F1010144F21408C4F2060874
:104D3000D8F8000010F4803FEBD016E048F2A060F5
:104D4000C0F20100814202D94FF001020DE001F1F1
:104D5000010144F22808C4F20608D8F8000010F453
:104D6000803FEBD001E04FF0010210465DF8048B6C
:104D7000704700002DE9304143F21C08C4F20708D7
:104D8000D8F8005005F0030543F21808C4F20708EC
:104D9000D8F8000005EA000543F21C08C4F2070831
:104DA000C8F800504FF000044FF0010000FA04F082
:104DB00000EA050040B320464FEA800040F6487103
:104DC000C2F2000100EB0100006858B120464FEA32
:104DD000800040F64871C2F2000100EB010000685B
:104DE000804711E04FF0010000FA04F143F2180887
:104DF000C4F20708D8F8000020EA010043F21808BE
:104E0000C4F20708C8F8000004F10104022CCBD357
:104E1000BFF34F8FBDE83081000000002DE9304125
:104E2000054628464FEA80004FF62011C0F20101E6
:104E300000EB010000684FF61411C0F2010101F10E
:104E400008018468096804EA0104C16804EA0104ED
:104E5000C4604FF61418C0F20108D8F8000000EA48
:104E6000040008B328464FEA40004FEA800040F6AD
:104E70005071C2F2000100EB0100006868B12846E1
:104E80004FEA40004FEA800040F65071C2F2000144
:104E900000EB01000068804706E028464FF0010261
:104EA0004FF0000100F032F84FF61410C0F201008C
:104EB00000F10400006800EA040028B340F65070D6
:104EC000C2F2000000F1040128464FEA40004FEA18
:104ED000800000EB0100006878B140F65070C2F22B
:104EE000000000F1040128464FEA40004FEA80002C
:104EF00000EB01000068804706E028464FF0010201
:104F00004FF0010100F002F8BDE8308110B4034613
:104F10004FEA830318464FF62013C0F2010300EB5B
:104F2000030003687AB90C464FEA840420464FF622
:104F30001411C0F2010100EB01009C68006844EA12
:104F400000049C600EE00C464FEA840420464FF6B5
:104F50001411C0F2010100EB01009C68006824EA12
:104F600000049C6010BC704700B581B04FF0000099
:104F7000FFF754FFBFF34F8F01B000BD00B581B004
:104F80004FF00100FFF74AFFBFF34F8F01B000BDA4
:104F900000B581B04FF00200FFF740FFBFF34F8F25
:104FA00001B000BD2DE9104181B04FF00104BFF305
:104FB0004F8F4EF60C58CEF20008D8F8000000F4DF
:104FC000E06040F20001C0F2FA5140EA010040F016
:104FD00004004EF60C58CEF20008C8F80000BFF3EB
:104FE0004F8F00E000BF002CFCD101B0BDE8108164
:104FF0004DF8048D4FF00101002800F09B80427AAB
:1050000042F21008C4F20308D8F800106FF3000150
:1050100002F0010241EA020142F21008C4F2030860
:10502000C8F80010027A42F21008C4F20308D8F857
:1050300000106FF3820102F001024FEA820241EA9E
:10504000020142F21008C4F20308C8F8001042F24C
:105050001008C4F20308D8F8001011F0010F15D1A0
:10506000426842F20C08C4F20308D8F800106FF34B
:105070000F014FF6FF7302EA030241EA020142F216
:105080000C08C4F20308C8F8001006E0416842F2B8
:105090000C08C4F20308C8F80010C17A71B942F2D2
:1050A0001008C4F20308D8F8001041F0C00142F221
:1050B0001008C4F20308C8F800100FE042F210080C
:1050C000C4F20308D8F800106FF3871141F0800193
:1050D00042F21008C4F20308C8F80010827A42F2C3
:1050E0001008C4F20308D8F800106FF3051102F09D
:1050F00003024FEA021241EA020142F21008C4F22E
:105100000308C8F8001042F21008C4F20308D8F8E7
:10511000001041F0020142F21008C4F20308C8F87E
:105120000010006842F20808C4F20308C8F8000042
:105130004FF0000108465DF8048B70472DE93001FF
:105140004FF00004012A13D142F21008C4F2030800
:10515000D8F8005045F0020542F21008C4F20308E6
:10516000C8F8005042F20808C4F20308C8F800303A
:1051700042F21008C4F20308D8F800506FF341055A
:1051800042F21008C4F20308C8F8005027E004EB0C
:10519000000204F1010303EB00031B784FEA032331
:1051A000127843EA020204F1020303EB00031B78C6
:1051B0004FEA034343EA020204F1030303EB000353
:1051C0001B784FEA036343EA020542F20808C4F27F
:1051D0000308C8F8005004F10404A1F104010429F3
:1051E000D5D20CE004EB0002127842F20808C4F2B7
:1051F000030888F80020A1F1010104F1010400294D
:10520000F0D842F20808C4F20308D8F80000BDE85C
:10521000300170472DE9304148F21C08C4F2000803
:10522000D8F8005048F20C08C4F20008D8F8000082
:1052300005EA00054FF0000420464FEA80004FF6D3
:105240003811C0F2010100EB0100006800EA05001E
:10525000002840D04FEA044048F28001C8F2000123
:1052600040EA010048F21408C4F20008C8F800003F
:1052700020464FEA40004FEA800040F66871C2F2D3
:10528000000100EB0100006868B120464FEA4000D1
:105290004FEA800040F66871C2F2000100EB0100A5
:1052A0000068804717E020464FEA80004FF638112B
:1052B000C0F2010100EB010148F20C08C4F2000841
:1052C000D8F80000096820EA010048F20C08C4F28E
:1052D0000008C8F8000004F10104102CACD3BDE8AC
:1052E00030812DE9704181B048F22008C4F20008F5
:1052F000D8F8002001464FEA81014FF63813C0F27A
:10530000010301EB0301096801EA0201002971D0E0
:105310004FEA006148F20002C0F2800241EA020155
:1053200040EA010148F21408C4F20008C8F800106D
:1053300040F66871C2F2000101F1040201464FEA31
:1053400041014FEA810101EB0201096871B140F6A8
:105350006871C2F2000101F104014FEA40004FEA16
:10536000800000EB01000068804743E04FF000013F
:105370004FF000024FF000044FF000034FF0000127
:1053800001464FEA411148F20022C4F2000201EB4B
:10539000020189694FF0020221EA020104464FEA44
:1053A000441448F20025C4F2000504EB0504A16191
:1053B00002EA010410E005464FEA451548F20026CE
:1053C000C4F2000605EB0605A961642B02D94FF073
:1053D00001010FE003F1010305464FEA451548F2CC
:1053E0000026C4F2000605EB0605AD6902EA0505D4
:1053F000A542E0D101B0BDE8708100B581B04FF0A9
:105400000000FFF76EFFBFF34F8F01B000BD00B586
:1054100081B04FF00100FFF764FFBFF34F8F01B081
:1054200000BD00B581B04FF00200FFF75AFFBFF397
:105430004F8F01B000BD00B581B04FF00300FFF702
:1054400050FFBFF34F8F01B000BD00B581B04FF0EA
:105450000400FFF746FFBFF34F8F01B000BD00B55A
:1054600081B04FF00500FFF73CFFBFF34F8F01B055
:1054700000BD00B581B04FF00600FFF732FFBFF36B
:105480004F8F01B000BD00B581B04FF00700FFF7AE
:1054900028FFBFF34F8F01B000BD00B581B04FF0C2
:1054A0000800FFF71EFFBFF34F8F01B000BD00B52E
:1054B00081B04FF00900FFF714FFBFF34F8F01B029
:1054C00000BD00B581B04FF00A00FFF70AFFBFF33F
:1054D0004F8F01B000BD00B581B04FF00B00FFF75A
:1054E00000FFBFF34F8F01B000BD00B581B04FF09A
:1054F0000C00FFF7F6FEBFF34F8F01B000BD00B503
:1055000081B04FF00D00FFF7ECFEBFF34F8F01B0FD
:1055100000BD00B581B04FF00E00FFF7E2FEBFF313
:105520004F8F01B000BD00B581B04FF00F00FFF705
:10553000D8FEBFF34F8F01B000BD00B581B0FFF7BB
:1055400069FEBFF34F8F01B000BD2DE9104181B05E
:1055500041F20004C4F206044FF0000000F017F816
:10556000A06800F0100068B140F6E878C2F20008C8
:10557000D8F8000030B140F6E878C2F20008D8F858
:1055800000008047BFF34F8F01B0BDE8108141F2AA
:105590000002C4F20602916841F080719160704788
:1055A00000B581B0FFF7D1FF01B000BD2DE9F04596
:1055B00081B0064630464FEA80004FF68821C0F29F
:1055C000010100EB0100056830464FEA80004FF60C
:1055D0007421C0F2010100EB0100D0F800A0D5F861
:1055E00090704FF000044FF0010000FA04F000EA60
:1055F000070088B340F6EC78C2F20008D8F8000043
:1056000050B140F6EC78C2F20008D8F80020E0B2C1
:105610000146304690471FE020464FEA80000AF1DD
:10562000100100EB01004FF0B641016020464FEA47
:10563000800005F1100100EB010108686FF31340D1
:10564000086020464FEA800005F1100100EB0101DF
:10565000086840F4004008604FF0010000FA04F0D0
:1056600000EA0700C5F8900004F10104202CBAD329
:10567000BFF34F8F01B0BDE8F08500B581B04FF0AA
:105680000000FFF793FF01B000BD00B581B04FF0FF
:105690000100FFF78BFF01B000BD00B581B04FF0F6
:1056A0000200FFF783FF01B000BD00B581B04FF0ED
:1056B0000300FFF77BFF01B000BD00B581B04FF0E4
:1056C0000400FFF773FF01B000BD30B403464FEA9A
:1056D00083034FF68824C0F2010403EB04031B6824
:1056E00004464FEA840420464FF67424C0F20104B5
:1056F00000EB040000680C464FEA840403F1100537
:1057000004EB0504246814F4004F09D00C464FEA5A
:10571000840400F1100004EB00004FF0B644046074
:105720000C464FEA8404204603F1100400EB040009
:1057300004686FF30A2402F007024FEA022244EAE7
:10574000020404604FEA8101084603F1100100EBF6
:105750000100016841F40041016030BC70472DE94F
:10576000704181B0044620464FEA80004FF6083170
:10577000C0F2010100EB0100056820464FEA8000FD
:105780004FF60031C0F2010100EB01000068C66D68
:10579000C16906EA0106C6654FF6C428C0F20108D1
:1057A000D8F8000000EA060030B320464FEAC001F6
:1057B000A1EB00004FEA40004FEA800040F6F07194
:1057C000C2F2000100EB0100006888B120464FEAF8
:1057D000C001A1EB00004FEA40004FEA800040F614
:1057E000F071C2F2000100EB01000068804703E0A5
:1057F000E8696FF30000E8614FF6C420C0F20100D1
:1058000000F10400006800EA060050B340F6F070B2
:10581000C2F2000000F1040120464FEAC002A2EBF0
:1058200000004FEA40004FEA800000EB01000068F2
:1058300098B140F6F070C2F2000000F10401204679
:105840004FEAC002A2EB00004FEA40004FEA80009E
:1058500000EB01000068804703E0E8696FF3410056
:10586000E8614FF6C420C0F2010000F108000068B2
:1058700000EA060050B340F6F070C2F2000000F1FA
:10588000080120464FEAC002A2EB00004FEA4000A8
:105890004FEA800000EB0100006898B140F6F0701C
:1058A000C2F2000000F1080120464FEAC002A2EB5C
:1058B00000004FEA40004FEA800000EB0100006862
:1058C000804703E0E8696FF38200E8614FF6C42087
:1058D000C0F2010000F10C00006800EA060050B3BD
:1058E00040F6F070C2F2000000F10C0120464FEAD1
:1058F000C002A2EB00004FEA40004FEA800000EB3C
:105900000100006898B140F6F070C2F2000000F1AA
:105910000C0120464FEAC002A2EB00004FEA400013
:105920004FEA800000EB01000068804703E0E8696F
:105930006FF3C300E8614FF6C420C0F2010000F12C
:105940001000006800EA060050B340F6F070C2F2A2
:10595000000000F1100120464FEAC002A2EB000057
:105960004FEA40004FEA800000EB0100006898B168
:1059700040F6F070C2F2000000F1100120464FEA3C
:10598000C002A2EB00004FEA40004FEA800000EBAB
:1059900001000068804703E0E8696FF30410E861E4
:1059A0004FF6C420C0F2010000F11400006800EAC4
:1059B000060050B340F6F070C2F2000000F114018E
:1059C00020464FEAC002A2EB00004FEA40004FEA37
:1059D000800000EB0100006898B140F6F070C2F260
:1059E000000000F1140120464FEAC002A2EB0000C3
:1059F0004FEA40004FEA800000EB0100006880475A
:105A000003E0E8696FF34510E8614FF6C420C0F287
:105A1000010000F11800006800EA060050B340F6EB
:105A2000F070C2F2000000F1180120464FEAC002F7
:105A3000A2EB00004FEA40004FEA800000EB0100BB
:105A4000006898B140F6F070C2F2000000F1180151
:105A500020464FEAC002A2EB00004FEA40004FEAA6
:105A6000800000EB01000068804703E0E8696FF305
:105A70009650E8614FF6C420C0F2010000F11C000E
:105A8000006800EA060050B340F6F070C2F2000071
:105A900000F11C0120464FEAC002A2EB00004FEAD1
:105AA00040004FEA800000EB0100006898B140F62A
:105AB000F070C2F2000000F11C0120464FEAC00263
:105AC000A2EB00004FEA40004FEA800000EB01002B
:105AD0000068804703E0E8696FF3D750E8614FF64C
:105AE000C420C0F2010000F12000006800EA0600B6
:105AF00050B340F6F070C2F2000000F120012046E1
:105B00004FEAC002A2EB00004FEA40004FEA8000DB
:105B100000EB0100006898B140F6F070C2F200009E
:105B200000F1200120464FEAC002A2EB00004FEA3C
:105B300040004FEA800000EB01000068804703E06E
:105B4000E8696FF31860E8614FF6C420C0F2010005
:105B500000F12400006800EA060050B340F6F0703F
:105B6000C2F2000000F1240120464FEAC002A2EB7D
:105B700000004FEA40004FEA800000EB010000689F
:105B800098B140F6F070C2F2000000F12401204606
:105B90004FEAC002A2EB00004FEA40004FEA80004B
:105BA00000EB01000068804703E0E8696FF359608B
:105BB000E8614FF6C420C0F2010000F1280000683F
:105BC00000EA060050B340F6F070C2F2000000F1A7
:105BD000280120464FEAC002A2EB00004FEA400035
:105BE0004FEA800000EB0100006898B140F6F070C9
:105BF000C2F2000000F1280120464FEAC002A2EBE9
:105C000000004FEA40004FEA800000EB010000680E
:105C1000804703E0E8696FF39A60E8614FF6C420BB
:105C2000C0F2010000F12C00006800EA060050B349
:105C300040F6F070C2F2000000F12C0120464FEA5D
:105C4000C002A2EB00004FEA40004FEA800000EBE8
:105C50000100006898B140F6F070C2F2000000F157
:105C60002C0120464FEAC002A2EB00004FEA4000A0
:105C70004FEA800000EB01000068804703E0E8691C
:105C80006FF3DB60E8614FF6C420C0F2010000F161
:105C90003000006800EA060050B340F6F070C2F22F
:105CA000000000F1300120464FEAC002A2EB0000E4
:105CB0004FEA40004FEA800000EB0100006898B115
:105CC00040F6F070C2F2000000F1300120464FEAC9
:105CD000C002A2EB00004FEA40004FEA800000EB58
:105CE00001000068804703E0E8696FF39E70E86197
:105CF0004FF6C420C0F2010000F13400006800EA51
:105D0000060050B340F6F070C2F2000000F134011A
:105D100020464FEAC002A2EB00004FEA40004FEAE3
:105D2000800000EB0100006898B140F6F070C2F20C
:105D3000000000F1340120464FEAC002A2EB00004F
:105D40004FEA40004FEA800000EB01000068804706
:105D500003E0E8696FF3DF70E861BFF34F8F01B0D4
:105D6000BDE8708100B581B04FF00000FFF7F7FC8F
:105D700001B000BD00B581B04FF00100FFF7EFFCAE
:105D800001B000BD2DE9F044064630464FEA8000E0
:105D90004FF64831C0F2010100EB0100D0F800A03D
:105DA0004FF000042146304600F089F8074630469F
:105DB0004FEA800004EB00004FEA800041F26001EE
:105DC000C2F2000100EB0100006807EA000720466C
:105DD0004FEA800100EB01004FEA80000AF1080160
:105DE00000EB0100C7604FF0000528464FEA800035
:105DF0004FF65031C0F2010100EB0100006800EAEB
:105E00000700F8B330464FEA800004EB00004FEA89
:105E1000800005EB00004FEA800041F28001C2F2F1
:105E2000000100EB0100006898B130464FEA8000A5
:105E300004EB00004FEA800005EB00004FEA800011
:105E400041F28001C2F2000100EB010000688047CE
:105E500018E028464FEA80004FF66431C0F2010195
:105E600000EB010220464FEA800100EB01004FEAFF
:105E700080000AF1080100EB0101C868126820EAFD
:105E80000200C86005F10105042DAED304F1010044
:105E9000C4B2042C86D3BFF34F8FBDE8F08400B5A5
:105EA00081B04FF00000FFF76DFF01B000BD00B5FD
:105EB00081B04FF00100FFF765FF01B000BD024661
:105EC0004FEA820210464FF64832C0F2010200EB60
:105ED000020003680A464FEA820002EB00024FEA22
:105EE0008202104603F1080100EB0100C26810466F
:105EF0007047002810DB4FEA50114FEA81014EF243
:105F00000012CEF2000201EB020100F01F004FF080
:105F1000010202FA00F00860704700B581B0002865
:105F200014DB4FEA50114FEA81014EF28012CEF29B
:105F3000000201EB020100F01F004FF0010202FA23
:105F400000F00860BFF34F8FBFF36F8F01B000BD4B
:105F5000002810DB4FEA50114FEA81014EF28022F7
:105F6000CEF2000201EB020100F01F004FF001022F
:105F700002FA00F00860704700280CDB4EF2004285
:105F8000CEF2000200EB02004FEA011101F0FF0126
:105F9000C9B201700FE000F00F00A0F104004EF64E
:105FA0001852CEF2000200EB02004FEA011101F09C
:105FB000FF01C9B2017070472DE9104181B04FF067
:105FC0000004A0F10101B1F1807F02D34FF0010480
:105FD0001DE0A0F101004EF21408CEF20008C8F84E
:105FE00000004FF00F014FF0FF30FFF7C5FF4FF0FB
:105FF00000004EF21808CEF20008C8F800004FF07A
:1060000007004EF21008CEF20008C8F80000204643
:1060100001B0BDE8108100002DE9F04405464FF0C5
:1060200000044FF0000028464FEA80004FF6883108
:10603000C0F2010100EB0100076828464FEA80002A
:106040004FF68031C0F2010100EB0100D0F800A052
:106050004FF69030C0F2010000F144000668B86BC2
:1060600006EA00064FF000044FF0010000FA04F0C9
:1060700000EA0600002842D020464FEA80000AF1DC
:106080003C0100EB0100006810F0100F37D02046F3
:106090004FEA800007F13C0100EB010000686FF05F
:1060A000200100EA010021464FEA810107F13C028C
:1060B00001EB0201086005EB051004EB00004FEA5C
:1060C000800041F20011C2F2000100EB0100006803
:1060D00070B105EB051004EB00004FEA800041F2BF
:1060E0000011C2F2000100EB01000068804706E0E9
:1060F000E0B2014628464FF0010200F07CFA04F1BC
:106100000104072CB0D9BFF34F8FBDE8F08400B570
:1061100081B04FF0000101464FEA81014FF688320D
:10612000C0F2010201EB02010A684FF69031C0F2A1
:10613000010101F140010968D2F8903001EA030140
:106140004FF69033C0F2010303F140031B6803EAEA
:10615000010353B3D2F890106FF0300301EA03014A
:10616000C2F8901041F20011C2F2000101F14002A8
:1061700000EB00114FEA810101EB0201096871B1E6
:1061800041F20011C2F2000101F1400100EB0010E8
:106190004FEA800000EB01000068804705E04FF007
:1061A00001024FF0100100F026FABFF34F8F01B04B
:1061B00000BD70B504464FF0000020464FEA800055
:1061C0004FF68831C0F2010100EB010005684FF67F
:1061D0009030C0F2010000F144000668A86B06EAA6
:1061E00000064FF69030C0F2010000F13000006868
:1061F00000EA060048B3A86B6FF4805100EA010082
:10620000A86341F20010C2F2000000F1300104EB7B
:1062100004104FEA800000EB0100006870B141F209
:106220000010C2F2000000F1300104EB04104FEA4C
:10623000800000EB01000068804706E020464FF038
:1062400001024FF00C0100F0D6F94FF69030C0F289
:10625000010000F13400006800EA060048B3A86BB2
:106260006FF4005100EA0100A86341F20010C2F28D
:10627000000000F1340104EB04104FEA800000EB51
:106280000100006870B141F20010C2F2000000F19C
:10629000340104EB04104FEA800000EB01000068B9
:1062A000804706E020464FF001024FF00D0100F05C
:1062B000A2F94FF69030C0F2010000F138000068FA
:1062C00000EA060048B3A86B6FF4804100EA0100C1
:1062D000A86341F20010C2F2000000F1380104EBA3
:1062E00004104FEA800000EB0100006870B141F239
:1062F0000010C2F2000000F1380104EB04104FEA74
:10630000800000EB01000068804706E020464FF067
:1063100001024FF00E0100F06EF94FF69030C0F21E
:10632000010000F13C00006800EA060048B3A86BD9
:106330006FF4004100EA0100A86341F20010C2F2CC
:10634000000000F13C0104EB04104FEA800000EB78
:106350000100006870B141F20010C2F2000000F1CB
:106360003C0104EB04104FEA800000EB01000068E0
:10637000804706E020464FF001024FF00F0100F089
:106380003AF9BFF34F8F70BD70B504464FF000006F
:1063900020464FEA80004FF68831C0F2010100EB41
:1063A000010005684FF69030C0F2010000F1440092
:1063B0000668A86B06EA00064FF69030C0F20100AE
:1063C00000F12000006800EA060048B3A86B6FF4F3
:1063D000807100EA0100A86341F20010C2F20000DF
:1063E00000F1200104EB04104FEA800000EB0100F3
:1063F000006870B141F20010C2F2000000F120010B
:1064000004EB04104FEA800000EB010000688047B5
:1064100006E020464FF001024FF0080100F0EBF8D3
:106420004FF69030C0F2010000F12400006800EA4D
:10643000060048B3A86B6FF4007100EA0100A8637E
:1064400041F20010C2F2000000F1240104EB04103C
:106450004FEA800000EB0100006870B141F20010CB
:10646000C2F2000000F1240104EB04104FEA8000A6
:1064700000EB01000068804706E020464FF0010273
:106480004FF0090100F0B7F84FF69030C0F201006C
:1064900000F12800006800EA060048B3A86B6FF41A
:1064A000806100EA0100A86341F20010C2F200001E
:1064B00000F1280104EB04104FEA800000EB01001A
:1064C000006870B141F20010C2F2000000F1280132
:1064D00004EB04104FEA800000EB010000688047E5
:1064E00006E020464FF001024FF00A0100F083F869
:1064F0004FF69030C0F2010000F12C00006800EA75
:10650000060048B3A86B6FF4006100EA0100A863BD
:1065100041F20010C2F2000000F12C0104EB041063
:106520004FEA800000EB0100006870B141F20010FA
:10653000C2F2000000F12C0104EB04104FEA8000CD
:1065400000EB01000068804706E020464FF00102A2
:106550004FF00B0100F04FF8BFF34F8F70BD00B547
:1065600081B04FF00000FFF757FD01B000BD00B54E
:1065700081B04FF00000FFF7CAFD01B000BD00B5CB
:1065800081B04FF00000FFF714FE01B000BD00B570
:1065900081B04FF00000FFF7F7FE01B000BD00B57D
:1065A00081B04FF00100FFF737FD01B000BD00B52D
:1065B00081B04FF00100FFF7AAFD01B000BD00B5AA
:1065C00081B04FF00100FFF7F4FD01B000BD00B550
:1065D00081B04FF00100FFF7D7FE01B000BD000011
:1065E00000000000000000000000000000000000AB
:1065F0000000000000002DE9700103464FEA83030C
:1066000018464FF68033C0F2010300EB0300036825
:10661000002A14BF002001200446112900F2AE8197
:106620000FF20408D8E801F00914233241505F6EDC
:106630007D88939EA9B4BFCAD5E2D96B6FF30411CC
:1066400004F001044FEA041441EA0401D96395E11E
:1066500003F13C0000F1040529686FF3041104F014
:1066600001034FEA031341EA0301296086E103F1C4
:106670003C0000F1080529686FF3041104F00103E0
:106680004FEA031341EA0301296077E103F13C007B
:1066900000F10C0529686FF3041104F001034FEABF
:1066A000031341EA0301296068E103F13C0000F1B2
:1066B000100529686FF3041104F001034FEA031376
:1066C00041EA0301296059E103F13C0000F114059E
:1066D00029686FF3041104F001034FEA031341EA40
:1066E000030129604AE103F13C0000F11805296823
:1066F0006FF3041104F001034FEA031341EA0301AD
:1067000029603BE103F13C0000F11C0529686FF3AF
:10671000041104F001034FEA031341EA0301296065
:106720002CE1596B6FF3104104F001044FEA04446B
:1067300041EA0401596321E1596B6FF3514104F0BF
:1067400001044FEA444441EA0401596316E1596BDC
:106750006FF3924104F001044FEA844441EA0401DA
:1067600059630BE1596B6FF3D34104F001044FEA15
:10677000C44441EA0401596300E1596B6FF31451B9
:1067800004F001044FEA045441EA04015963F5E0BE
:10679000596B6FF3555104F001044FEA445441EA38
:1067A00004015963EAE0596B6FF3965104F0010458
:1067B0004FEA845441EA04015963DFE0596B6FF3F7
:1067C000D75104F001044FEAC45441EA040159636B
:1067D000D4E0D3F88C106FF30C3104F001044FEACD
:1067E000043441EA0401C3F88C10C7E0D96B6FF39D
:1067F000041104F001054FEA051541EA0501D963CA
:1068000003F13C0000F1040631686FF3041104F059
:1068100001054FEA051541EA0501316003F13C002D
:1068200000F1080631686FF3041104F001054FEA26
:10683000051541EA0501316003F13C0000F10C0649
:1068400031686FF3041104F001054FEA051541EAC0
:106850000501316003F13C0000F1100631686FF36F
:10686000041104F001054FEA051541EA0501316004
:1068700003F13C0000F1140631686FF3041104F0D9
:1068800001054FEA051541EA0501316003F13C00BD
:1068900000F1180631686FF3041104F001054FEAA6
:1068A000051541EA0501316003F13C0000F11C06C9
:1068B00031686FF3041104F001054FEA051541EA50
:1068C00005013160596B6FF3104104F001054FEA87
:1068D000054541EA05015963596B6FF3514104F0D5
:1068E00001054FEA454541EA05015963596B6FF3CC
:1068F000924104F001054FEA854541EA05015963DB
:10690000596B6FF3D34104F001054FEAC54541EAE5
:1069100005015963596B6FF3145104F001054FEAF7
:10692000055541EA05015963596B6FF3555104F060
:1069300001054FEA455541EA05015963596B6FF36B
:10694000965104F001054FEA855541EA0501596366
:10695000596B6FF3D75104F001054FEAC55541EA71
:1069600005015963D3F88C106FF30C3104F0010466
:106970004FEA043441EA0401C3F88C10BDE8700109
:10698000704700002DE9104181B04DF21008C4F2AB
:106990000708D8F8004040F69018C2F20008D8F86E
:1069A000000004EA00044DF20008C4F20708D8F819
:1069B000000010F0004F09D040F20000C9F273400F
:1069C0004DF20008C4F20708C8F800004DF21008A4
:1069D000C4F20708C8F800404DF20008C4F20708E6
:1069E000D8F8000040F000404DF20008C4F207085B
:1069F000C8F800004FF6D838C0F20108D8F80000F7
:106A000000EA0400A0B141F28818C2F20008D8F8E8
:106A1000000038B141F28818C2F20008D8F800002E
:106A2000804705E04FF001014FF0000000F026F82C
:106A30004FF6D830C0F2010000F10400006800EA0F
:106A40000400B0B141F28810C2F2000000F104006D
:106A5000006840B141F28810C2F2000000F1040069
:106A60000068804705E04FF001014FF0010000F0A1
:106A700005F8BFF34F8F01B0BDE810814DF8048DCC
:106A80004DF20008C4F20708D8F8002012F0004FB9
:106A900009D040F20002C9F273424DF20008C4F27C
:106AA0000708C8F8002051BB02464FEA820211468F
:106AB0004FF6E432C0F2010201EB02014DF2100880
:106AC000C4F20708D8F80020096842EA01024DF232
:106AD0001008C4F20708C8F800204FEA80004FF6FB
:106AE000D831C0F2010100EB010140F69012C2F270
:106AF00000021068096840EA0100106029E00246BF
:106B00004FEA820211464FF6D832C0F2010201EB81
:106B1000020140F69013C2F200031A68096822EAE3
:106B200001021A604FEA80004FF6E431C0F2010121
:106B300000EB01014DF21008C4F20708D8F800007C
:106B4000096820EA01004DF21008C4F20708C8F8ED
:106B500000004DF20008C4F20708D8F8000040F029
:106B600000404DF20008C4F20708C8F800005DF8C4
:106B7000048B70474FF0010220280CD202464FEAE6
:106B8000820210464CF20002C4F2070200EB02003F
:106B900001604FF00002104670474FF001022028BC
:106BA0000ED269B102464FEA820210464CF2000250
:106BB000C4F2070200EB0200006808604FF0000218
:106BC0001046704700B581B000F008F801B000BD74
:106BD00000B581B000F002F801B000BD2DE9104110
:106BE00081B04FF0000049F21808C4F20708D8F845
:106BF000000010F0004F09D040F20000C9F6670015
:106C000049F21808C4F20708C8F8000049F2000861
:106C1000C4F20708D8F8004041F2A018C2F20008F8
:106C2000D8F8000004EA00044FF6F030C0F201008A
:106C300000F10400006800EA040030B34FF0FF30B8
:106C400049F21008C4F20708C8F8000041F2901099
:106C5000C2F2000000F10400006840B141F290105F
:106C6000C2F2000000F10400006880470DE049F224
:106C70000408C4F20708D8F800006FF3041049F2C2
:106C80000408C4F20708C8F800004FF6F038C0F254
:106C90000108D8F8000000EA0400E0B141F29018C1
:106CA000C2F20008D8F8000038B141F29018C2F2E0
:106CB0000008D8F8000080470DE049F20408C4F24B
:106CC0000708D8F800006FF3C30049F20408C4F2C3
:106CD0000708C8F800004FF6F030C0F2010000F1DC
:106CE0000800006800EA040080B349F20008C4F21A
:106CF0000708D8F8000041F27F4100EA010040F4A3
:106D0000006049F20008C4F20708C8F8000041F228
:106D10009010C2F2000000F10800006840B141F29A
:106D20009010C2F2000000F10800006880470DE0FA
:106D300049F20408C4F20708D8F800006FF34510C0
:106D400049F20408C4F20708C8F800004FF6F03012
:106D5000C0F2010000F10C00006800EA040080B3FA
:106D600049F20008C4F20708D8F8000041F27F4158
:106D700000EA010040F4005049F20008C4F207089C
:106D8000C8F8000041F29010C2F2000000F10C00BF
:106D9000006840B141F29010C2F2000000F10C0016
:106DA000006880470DE049F20408C4F20708D8F8EB
:106DB00000006FF3861049F20408C4F20708C8F80F
:106DC000000049F21808C4F20708D8F8000040F0A3
:106DD000004049F21808C4F20708C8F80000BFF3E1
:106DE0004F8F01B0BDE810810000000000000000DE
:106DF00000000000000000002DE9104181B048F2C1
:106E00004008C4F20408D8F8004041F2C018C2F2A9
:106E10000008D8F8000004EA000448F24008C4F270
:106E20000408C8F800404FF61840C0F2010000F115
:106E30000400006800EA0400F0B141F2A410C2F2BC
:106E4000000000F10400006840B141F2A410C2F259
:106E5000000000F10400006880470DE048F20408DB
:106E6000C4F20408D8F800006FF3186048F2040870
:106E7000C4F20408C8F800004FF61840C0F2010040
:106E800000F10800006800EA0400F0B141F2A4102B
:106E9000C2F2000000F10800006840B141F2A41005
:106EA000C2F2000000F10800006880470DE048F2DF
:106EB0000408C4F20408D8F800006FF3596048F2DF
:106EC0000408C4F20408C8F800004FF61840C0F2E5
:106ED000010000F10C00006800EA0400F0B141F28A
:106EE000A410C2F2000000F10C00006840B141F2B1
:106EF000A410C2F2000000F10C00006880470DE011
:106F000048F20408C4F20408D8F800006FF39A604D
:106F100048F20408C4F20408C8F800004FF618400C
:106F2000C0F2010000F11000006800EA0400F0B1B6
:106F300041F2A410C2F2000000F11000006840B15C
:106F400041F2A410C2F2000000F110000068804776
:106F50000DE048F20408C4F20408D8F800006FF30A
:106F6000DB6048F20408C4F20408C8F800004FF6D9
:106F70001840C0F2010000F11400006800EA0400AB
:106F8000F0B141F2A410C2F2000000F11400006858
:106F900040B141F2A410C2F2000000F114000068F8
:106FA00080470DE048F20408C4F20408D8F8000055
:106FB0006FF31C7048F20408C4F20408C8F800001B
:106FC0004FF61840C0F2010000F11800006800EA16
:106FD0000400F0B141F2A410C2F2000000F1180068
:106FE000006840B141F2A410C2F2000000F11800A4
:106FF000006880470DE048F20408C4F20408D8F89D
:1070000000006FF35D7048F20408C4F20408C8F889
:1070100000004FF61848C0F20108D8F8000000EA56
:107020000400E0B141F2A418C2F20008D8F8000050
:1070300038B141F2A418C2F20008D8F80000804725
:107040000DE048F20408C4F20408D8F800006FF319
:10705000104048F20408C4F20408C8F80000BFF366
:107060004F8F01B0BDE8108100B581B0FFF7C4FEBD
:1070700001B000BD00B581B0FFF7BEFE01B000BD9C
:1070800000000000000000002DE900414FF0010069
:107090004FF20C08C4F20708C8F8000041F2C41807
:1070A000C2F20008D8F8000030B141F2C418C2F2B0
:1070B0000008D8F800008047BFF34F8FBDE800817B
:1070C0002DE9104181B04FF000044FF0010000FAAB
:1070D00004F04FF21C08C4F20708D8F8001000EAC8
:1070E0000100E0B14FF21C08C4F20708C8F8000024
:1070F00020464FEA800041F2C811C2F2000100EBC5
:107100000100006858B120464FEA800041F2C811E2
:10711000C2F2000100EB01000168E0B2884704F10F
:107120000104112CD1D3BFF34F8F01B0BDE8108102
:1071300000B581B0FFF7A8FF01B000BD00B581B078
:10714000FFF7BEFF01B000BD2DE9004101464FEA47
:1071500081014FF6CC42C0F2010201EB0201096845
:1071600002464FEA82024FF6BC43C0F2010302EB33
:1071700003021268136A4FF6DC48C0F20108D8F81F
:10718000002002EA0302E2B100EB80024FEA820231
:1071900041F20C23C2F2000302EB0302126862B157
:1071A00000EB80004FEA800041F20C21C2F20001A6
:1071B00000EB01000068804703E0C8696FF300003E
:1071C000C861BFF34F8FBDE8008100B581B00146B3
:1071D0004FEA81014FF6CC42C0F2010201EB0201FD
:1071E000096802464FEA82024FF6BC43C0F201032F
:1071F00002EB03021268136A4A6A02F001024FF6B8
:10720000DC42C0F2010202F10402126802EA030247
:1072100002B341F20C22C2F2000202F1040300EBBD
:1072200080024FEA820202EB0302126872B141F25D
:107230000C21C2F2000101F1040100EB80004FEAD1
:10724000800000EB01000068804703E0C8696FF32D
:107250004100C861BFF34F8F01B000BD00B581B0E0
:1072600001464FEA81014FF6CC42C0F2010201EB28
:107270000201096802464FEA82024FF6BC43C0F29F
:10728000010302EB03021268136A4FF6DC42C0F2FC
:10729000010202F11002126802EA030202B341F293
:1072A0000C22C2F2000202F1100300EB80024FEA4E
:1072B000820202EB0302126872B141F20C21C2F2A7
:1072C000000101F1100100EB80004FEA800000EBAB
:1072D00001000068804703E0C8696FF30410C861CB
:1072E000BFF34F8F01B000BD00B581B001464FEA3A
:1072F00081014FF6CC42C0F2010201EB02010968A4
:1073000002464FEA82024FF6BC43C0F2010302EB91
:1073100003021268136ACA6A02F001024FF6DC42E5
:10732000C0F2010202F10802126802EA030202B38B
:1073300041F20C22C2F2000202F1080300EB8002CB
:107340004FEA820202EB0302126872B141F20C2191
:10735000C2F2000101F1080100EB80004FEA800059
:1073600000EB01000068804703E0C8696FF382000A
:10737000C861BFF34F8F01B000BD00B581B00146B9
:107380004FEA81014FF6CC42C0F2010201EB02014B
:10739000096802464FEA82024FF6BC43C0F201037D
:1073A00002EB03021268136A8A6A02F001024FF6C6
:1073B000DC42C0F2010202F10C02126802EA03028E
:1073C00002B341F20C22C2F2000202F10C0300EB04
:1073D00080024FEA820202EB0302126872B141F2AC
:1073E0000C21C2F2000101F10C0100EB80004FEA18
:1073F000800000EB01000068804703E0C8696FF37C
:10740000C300C861BFF34F8F01B000BD00B581B0AC
:107410004FF00000FFF798FE01B000BD00B581B04D
:107420004FF00000FFF7D1FE01B000BD00B581B004
:107430004FF00000FFF712FF01B000BD00B581B0B2
:107440004FF00000FFF750FF01B000BD00B581B064
:107450004FF00000FFF791FF01B000BD00B581B013
:107460004FF00100FFF770FE01B000BD00B581B024
:107470004FF00100FFF7A9FE01B000BD00B581B0DB
:107480004FF00100FFF7EAFE01B000BD00B581B08A
:107490004FF00100FFF728FF01B000BD00B581B03B
:1074A0004FF00100FFF769FF01B000BD00B581B0EA
:1074B0004FF00200FFF748FE01B000BD00B581B0FB
:1074C0004FF00200FFF781FE01B000BD00B581B0B2
:1074D0004FF00200FFF7C2FE01B000BD00B581B061
:1074E0004FF00200FFF700FF01B000BD00B581B012
:1074F0004FF00200FFF741FF01B000BD00B581B0C1
:107500004FF00300FFF720FE01B000BD00B581B0D1
:107510004FF00300FFF759FE01B000BD00B581B088
:107520004FF00300FFF79AFE01B000BD00B581B037
:107530004FF00300FFF7D8FE01B000BD00B581B0E9
:107540004FF00300FFF719FF01B000BD10B4024671
:107550004FEA820210464FF6CC42C0F2010200EB25
:1075600002000268002957D0087813686FF355535A
:1075700000F001044FEA445443EA04031360C8686E
:10758000D3686FF30F034FF6FF7400EA040043EA79
:107590000003D3604868A0F1010013686FF314433F
:1075A00000F01F044FEA044443EA04031360087A1E
:1075B00013686FF3861300F001044FEA841443EA62
:1075C00004031360487A13686FF3C71300F00104D3
:1075D0004FEAC41443EA04031360887A13686FF314
:1075E000092300F003044FEA042443EA0403136070
:1075F000086913696FF3010300F0030043EA000315
:107600001361486911696FF3114100F003034FEAF8
:10761000034341EA0301116110BC704701464FEA80
:10762000810108464FF6CC41C0F2010100EB010098
:107630000268916841F001019160704701464FEA8C
:10764000810108464FF6CC41C0F2010100EB010078
:10765000026891686FF300019160704710B40246B0
:107660004FEA820210464FF6CC42C0F2010200EB14
:1076700002000468A2686FF3114201F003034FEAAD
:10768000034342EA0302A26010BC704702464FEA7D
:10769000820210464FF6BC42C0F2010200EB02002B
:1076A00002681166704701464FEA810108464FF6AD
:1076B000BC41C0F2010100EB01000168086E704797
:1076C00002464FEA820210464FF6BC42C0F2010267
:1076D00000EB020002684FF0010000FA01F092692D
:1076E00000EA020020FA01F1C8B270472DE900411A
:1076F00041F25C28C2F20008D8F8000030B141F233
:107700005C28C2F20008D8F800008047BFF34F8F12
:10771000BDE8008110B54FF0000420464FEA80001C
:1077200040F22401C4F2040100EB010000684FEABA
:1077300000404FEAD07021464FEA810140F2240216
:10774000C4F2040201EB020109684FEA81414FEAE9
:10775000D17100EA010021464FEA810140F2240282
:10776000C4F2040201EB020319686FF3CF3100F099
:1077700001024FEAC23241EA0201196018B3204601
:107780004FEA800041F26021C2F2000100EB0100EB
:10779000006858B120464FEA800041F26021C2F2F1
:1077A000000100EB0100006880470CE020464FEA32
:1077B000800040F22401C4F2040100EB01010868DA
:1077C0006FF34D30086004F10104042CA5D3BFF31E
:1077D0004F8F10BD00B581B0FFF79CFF01B000BD19
:1077E00001EB000003464FEA8303184641F2602193
:1077F000C2F2000100EB01000260704710B40246C3
:107800004FEA820240F22403C4F2040302EB0304B1
:107810000B7822686FF38A2203F001034FEA832377
:1078200042EA030222600A78002A58D102464FEA4F
:10783000820240F21403C4F2040302EB03024B6819
:10784000136002464FEA820240F22403C4F20403AA
:1078500002EB03040B7A22686FF3CB2203F00103DF
:107860004FEAC32342EA0302226002464FEA820241
:1078700040F22403C4F2040302EB03034C7A1A68B7
:107880006FF3010204F0030442EA04021A600246A4
:107890004FEA820240F22403C4F2040302EB030421
:1078A0004B7B22686FF3861203F001034FEA8313C8
:1078B00042EA030222604FEA800040F22402C4F24E
:1078C000040200EB0202097B10686FF3850001F0EF
:1078D0000F014FEA810140EA010010607FE002469B
:1078E0004FEA820240F21403C4F2040302EB0302E3
:1078F0004B68136002464FEA820240F22403C4F24E
:10790000040302EB03040B7A22686FF3CB2203F02B
:1079100001034FEAC32342EA0302226002464FEA10
:10792000820240F22403C4F2040302EB03034C7A04
:107930001A686FF3010204F0030442EA04021A60B9
:1079400002464FEA820240F22403C4F2040302EB2F
:1079500003048B7A22686FF3092203F003034FEAD2
:10796000032342EA0302226002464FEA820240F207
:107970002403C4F2040302EB0304CB7A22686FF3FE
:10798000C71203F001034FEAC31342EA0302226065
:1079900002464FEA820240F22403C4F2040302EBDF
:1079A00003044B7B22686FF3861203F001034FEA56
:1079B000831342EA030222604FEA800040F224026D
:1079C000C4F2040200EB0202097B10686FF3850029
:1079D00001F00F014FEA810140EA0100106010BC84
:1079E000704701464FEA8101084640F22401C4F283
:1079F000040100EB0102116841F4804111607047FD
:107A000001464FEA8101084640F22401C4F2040114
:107A100000EB010211686FF38E311160704710B4F2
:107A200002464FEA8202104640F22402C4F20402E7
:107A300000EB020422686FF34D3201F001034FEABC
:107A4000433342EA0302226010BC704701464FEA0A
:107A5000910001464FEA810108464FF61851C0F2E5
:107A6000010100EB01000168086810F0004F02D02E
:107A70004FF0B64008600A686FF355520A600A6812
:107A800042F400120A600A6842F000420A6070473D
:107A900001464FEA910001464FEA810108464FF640
:107AA0001851C0F2010100EB01000168086810F0F4
:107AB000004F02D04FF0B64008600A686FF3010231
:107AC00042F001020A600A6842F400120A600A6881
:107AD00042F000420A60704701464FEA91000146B9
:107AE0004FEA810108464FF61851C0F2010100EB40
:107AF00001000168086810F0004F02D04FF0B64056
:107B000008600A686FF301020A600A686FF3555251
:107B10000A600A6842F000420A607047F0B581B01E
:107B2000074638464FEA80004FF6EC51C0F201019B
:107B300000EB01000668356905F03F05F06805EACD
:107B4000000535614FF0000420464FEA80004FF6F3
:107B5000F451C0F2010100EB0100006800EA0500E9
:107B600050B3C7EBC70004EB00004FEA800041F2BE
:107B70007021C2F2000100EB0100006870B1C7EB98
:107B8000C70004EB00004FEA800041F27021C2F20E
:107B9000000100EB0100006880470DE020464FEA3D
:107BA00080004FF6F451C0F2010100EB0101F068D2
:107BB000096820EA0100F06004F10104052CC3D932
:107BC000BFF34F8F01B0F0BD10B501464FEA810100
:107BD0004FF61462C0F2010201EB0201096802468D
:107BE0004FEA82024FF6EC53C0F2010302EB0302AC
:107BF00012684FF6F453C0F2010303F11C031B6833
:107C0000146903EA04034FF6F454C0F2010404F1CA
:107C10001804246804EA030444B34FF6F453C0F292
:107C2000010303F118031B68136141F27022C2F2D1
:107C3000000202F11803C0EBC0024FEA820202EB1D
:107C40000302126872B141F27021C2F2000101F127
:107C50001801C0EBC0004FEA800000EB0100006893
:107C6000804703E0C8686FF30820C860BFF34F8FF8
:107C700010BD00B581B04FF00000FFF74FFF01B01D
:107C800000BD00B581B04FF00000FFF79DFF01B0CF
:107C900000BD00B581B04FF00100FFF73FFF01B01C
:107CA00000BD00B581B04FF00100FFF78DFF01B0BE
:107CB00000BD0000000000002DE9F04406464FF032
:107CC00000044FF000054FF0000030464FEA8000FE
:107CD0004FF62C61C0F2010100EB0100D0F800A0CA
:107CE00030464FEA80004FF61C61C0F2010100EB04
:107CF000010007684FF63C60C0F2010000F12C0063
:107D00000568786905EA00054FF000044FF00100AE
:107D100000FA04F000EA050000284AD020464FEAA5
:107D200080000AF1180100EB0100006810F0100F4C
:107D30003FD020464FEA800007F1180100EB010018
:107D400000686FF0200100EA010021464FEA81013E
:107D500007F1180201EB020108604FF00B0016FB5F
:107D600000F004EB00004FEA800041F2A821C2F2CB
:107D7000000100EB0100006880B14FF00B0016FB22
:107D800000F004EB00004FEA800041F2A821C2F2AB
:107D9000000100EB0100006880470AE020464FEA3E
:107DA00080000AF1180100EB010108686FF304106C
:107DB000086004F10104072CA8D9BFF34F8FBDE878
:107DC000F08410B54FF0000201464FEA81014FF6F2
:107DD0002C62C0F2010201EB0201096802464FEA7F
:107DE00082024FF61C63C0F2010302EB0302136828
:107DF000DA6E6FF0100402EA0402DA6641F2A82299
:107E0000C2F2000202F128034FF00B0210FB02F253
:107E10004FEA820202EB0302126882B141F2A8210A
:107E2000C2F2000101F128014FF00B0210FB02F039
:107E30004FEA800000EB01000068804703E0886E95
:107E40006FF386108866BFF34F8F10BD10B54FF0EB
:107E5000000201464FEA81014FF62C62C0F2010296
:107E600001EB0201096802464FEA82024FF61C63E9
:107E7000C0F2010302EB030213685A696FF4007445
:107E800002EA04025A6141F2A822C2F2000202F19F
:107E900024034FF00B0210FB02F24FEA820202EBC6
:107EA0000302126882B141F2A821C2F2000101F17D
:107EB00024014FF00B0210FB02F04FEA800000EBB0
:107EC00001000068804703E008696FF349200861FA
:107ED000BFF34F8F10BD10B54FF0000201464FEABF
:107EE00081014FF62C62C0F2010201EB0201096828
:107EF00002464FEA82024FF61C63C0F2010302EB16
:107F0000030213685A696FF4807402EA04025A612A
:107F100041F2A822C2F2000202F120034FF00B024C
:107F200010FB02F24FEA820202EB0302126882B1F6
:107F300041F2A821C2F2000101F120014FF00B0231
:107F400010FB02F04FEA800000EB01000068804760
:107F500003E008696FF308200861BFF34F8F10BD7D
:107F600000B581B04FF00000FFF7A6FE01B000BDE4
:107F700000B581B04FF00000FFF723FF01B000BD56
:107F800000B581B04FF00000FFF760FF01B000BD09
:107F900000B581B04FF00000FFF79DFF01B000BDBC
:107FA00000B581B04FF00100FFF786FE01B000BDC3
:107FB00000B581B04FF00100FFF703FF01B000BD35
:107FC00000B581B04FF00100FFF740FF01B000BDE8
:107FD00000B581B04FF00100FFF77DFF01B000BD9B
:107FE00000B581B04FF00200FFF766FE01B000BDA2
:107FF00000B581B04FF00200FFF7E3FE01B000BD15
:1080000000B581B04FF00200FFF720FF01B000BDC6
:1080100000B581B04FF00200FFF75DFF01B000BD79
:1080200000B581B04FF00300FFF746FE01B000BD80
:1080300000B581B04FF00300FFF7C3FE01B000BDF3
:1080400000B581B04FF00300FFF700FF01B000BDA5
:1080500000B581B04FF00300FFF73DFF01B000BD58
:108060000000000000000000000000000000000010
:108070000000000000002DE9104181B04FF66C6057
:10808000C0F2010000F11000046844F25408C4F288
:108090000308D8F8000004EA000444F25C08C4F2C3
:1080A0000308D8F8000004EA000444F25808C4F2B7
:1080B0000308C8F8004004F0010010B341F258383A
:1080C000C2F20008D8F8000038B141F25838C2F2C4
:1080D0000008D8F80000804713E044F25C08C4F2BE
:1080E0000308D8F800004FF66C68C0F20108D8F811
:1080F000001020EA010044F25C08C4F20308C8F84A
:1081000000004FEA540000F0010028B341F258305B
:10811000C2F2000000F10400006840B141F25830A2
:10812000C2F2000000F104000068804714E04FF63E
:108130006C60C0F2010000F1040144F25C08C4F27A
:108140000308D8F80000096820EA010044F25C083E
:10815000C4F20308C8F800004FEA940000F00100E0
:1081600028B341F25830C2F2000000F10800006864
:1081700040B141F25830C2F2000000F1080000683E
:10818000804714E04FF66C60C0F2010000F1080176
:1081900044F25C08C4F20308D8F80000096820EA39
:1081A000010044F25C08C4F20308C8F800004FEA7A
:1081B000D40000F0010028B341F25830C2F20000B0
:1081C00000F10C00006840B141F25830C2F20000EA
:1081D00000F10C000068804714E04FF66C60C0F2BC
:1081E000010000F10C0144F25C08C4F20308D8F865
:1081F0000000096820EA010044F25C08C4F20308A8
:10820000C8F80000BFF34F8F01B0BDE81081000037
:108210000000034642F20002C4F20502EFF31080B0
:10822000014601B972B64AF2C410CBF2D9005061CE
:1082300043F60F30C1F61E205061D36001B962B61B
:1082400042F20002C4F205024FF000014FF00000BC
:1082500007E0B1F5801F02D34FF0010005E001F106
:108260000101936813F0807FF3D070470000000095
:108270002DE9104181B0EFF31080044604B972B6C5
:1082800041F26838C2F20008D8F8000030B141F27B
:108290006838C2F20008D8F800008047BFF34F8F5B
:1082A00007B40F480F49104A0160026007BC42F250
:1082B0000808C4F20508D8F800004FF68068C0F23C
:1082C0000108D8F8001040EA010042F20808C4F2A0
:1082D0000508C8F8000004B962B601B0BDE8108115
:1082E00014200540C4A1D9B00F3B1E1A00B583B0BD
:1082F0004FF071008DF8040001A800F101004FF06B
:108300000101017001A800F102004FF0FF010170AE
:1083100001A800F103004FF00101017001F093F892
:10832000012806D101A84FF0040101F01EFF01F061
:108330009FF803B000BD4DF8048D4FF0000047F6E4
:10834000F478C0F20208D8F800104AF65522CAF6AE
:108350005522914201D14FF001005DF8048B704726
:108360002DE9104181B04FF48028D8F800104FF06B
:108370000418D8F800404FF480204EF60858CEF28A
:108380000008C8F80000084680F30888084680F313
:108390000988BFF34F8FA047FEE700B581B04FF0CB
:1083A00004014FF06400FCF79CFA4FF000014FF01D
:1083B0006400FCF768F94FF06400FFF747FB4FF0EB
:1083C0006400FFF765FB4FF004014FF0B400FCF7C9
:1083D00088FA4FF004014FF0C000FCF782FA4FF02A
:1083E000B400FFF755FB4FF0C000FFF751FB4FF013
:1083F00002024FF000014FF00400FDF766F94FF064
:1084000002024FF001014FF00400FDF75EF94FF05A
:1084100002024FF002014FF00400FDF756F94FF051
:1084200004024FF005014FF00100FDF74EF94FF641
:10843000A061C0F201014FF00000FFF787F84FF094
:1084400001014FF00000FFF709F94FF00000FFF7BE
:10845000E5F801B000BD00B581B04FF06400FFF752
:10846000F5FA4FF00000FFF7E9F84FF06400FFF76E
:1084700033FB4FF000014FF06400FCF732FA01B01B
:1084800000BD00B581B04FF004014FF0B000FCF723
:1084900028FA4FF000014FF0B000FCF7F4F84FF06D
:1084A000B000FFF7F5FA4FF0D000FFF7F1FA4FF008
:1084B00003024FF00D014FF00000FDF706F94FF0F9
:1084C00003024FF00C014FF00000FDF7FEF801B081
:1084D00000BD00B581B04FF0B000FFF7B7FA4FF024
:1084E000D000FFF7B3FA4FF0B000FFF7F5FA4FF006
:1084F000D000FFF7F1FA01B000BD2DE9004141F2D3
:108500006C38C2F20008D8F800003C2808D241F2CA
:108510006C31C2F20001086800F10100086007E058
:108520004FF0000041F26C38C2F20008C8F80000B9
:1085300041F26C38C2F20008D8F800104FF00A007F
:10854000B1FBF0F04FF00A0808FB00F0A1EB0000CF
:1085500008B900F09FFBBDE800812DE9004100F063
:10856000A4FD41F27438C2F20008D8F80000B0F55A
:10857000FA6F08D241F27431C2F20001086800F1CA
:108580000100086007E04FF0000041F27438C2F2C9
:108590000008C8F80000BDE8008100B581B047F2CE
:1085A0000010C0F20200FDF707FD10B14FF001000E
:1085B00001E04FF0000001B000BD2DE900414FF097
:1085C00000004EF21408CEF20008C8F800004FF088
:1085D00000004EF21808CEF20008C8F800004FF074
:1085E00000004EF21008CEF20008C8F800004FF06C
:1085F00000014FF0FF30FDF7BFFCBDE800812DE921
:1086000000414FF0000042F20808C4F20508D8F813
:10861000001040F27132C0F2070201EA020140F29A
:108620004102C0F20402914237D04AF2C411CBF2A7
:10863000D90142F21408C4F20508C8F8001043F644
:108640000F31C1F61E2142F21408C4F20508C8F821
:10865000001040F24101C0F2040142F20808C4F2E5
:108660000508C8F8001047F20071C0F2010142F29B
:108670000C08C4F20508C8F8001004E0B0F5801F2B
:1086800012D200F1010042F20808C4F20508D8F83D
:10869000001011F0807FF1D006E047F20070C0F2C8
:1086A0000100FFF7B6FD002800F0F4FABDE80081F4
:1086B00000B581B04FF6FF70C0F20100FFF7A9FDD1
:1086C000002800F0E7FA01B000BD4DF8048D40F23B
:1086D0000808C4F20208D8F8001021F00F0140F297
:1086E0000808C4F20208C8F8001040F20808C4F2F2
:1086F0000208D8F8001041EA000140F20808C4F26C
:108700000208C8F800105DF8048B704710B54FF0F0
:1087100000044FF000014FF08500FBF7B4FF4FF06D
:1087200001014FF08600FBF7AEFF4FF001014FF063
:108730008700FBF7A8FF4FF000024FF001014FF058
:108740000000FBF7D9FC18B14FF0010420463AE0D5
:1087500040F6A010C2F20000FBF75BFE4FF00100F4
:10876000FBF7FDFB4FF00400FFF7AFFF4FF00300F6
:10877000FBF74CFD0028F9D14FF0A000FFF7ACF952
:108780004FF004014FF0A000FCF7ABF84FF00101EF
:108790004FF0A000FBF777FF4FF0A000FFF778F94C
:1087A0004FF004014FF03000FCF79BF8012803D193
:1087B0004FF00104204606E04FF000014FF030007A
:1087C000FBF761FF204610BD00B581B04FF00100FE
:1087D000FBF790FB4FF00100FBF718FDA8B94FF035
:1087E00001014FF08500FBF74EFF4FF001014FF004
:1087F0008600FBF748FF4FF003014FF08700FBF7BF
:1088000042FF4FF00100FFF760FF4FF000014FF013
:108810003000FCF766F8002801B000BD00B581B05B
:108820004FF004014FF00800FCF75BF84FF0000137
:108830004FF00800FBF727FF4FF00800FFF728F97B
:108840004FF0B500FDF755FB4FF69061C0F2010106
:108850004FF00000FEF7D2FF48F2FB42C0F20102E7
:108860004FF000014FF00000FEF7BAFF4FF001019A
:108870004FF00000FFF7D3F84FF00000FFF7B1F81A
:1088800001B000BD00B581B04FF00000FFF7B8F8AF
:108890004FF000014FF00000FFF7C1F84FF0080063
:1088A000FFF71AF94FF0B500FDF737FB4FF0000165
:1088B0004FF00800FCF715F801B000BD00B581B01D
:1088C000FFF76BFD01B000BD00B581B0FFF7C3FD40
:1088D00001B000BD00B581B04FF09400FFF7B6F8CD
:1088E0004FF09400FFF7F8F801B000BD00B581B07B
:1088F000FFF785FEFFF70AFFFFF74FFEFFF78EFF3A
:1089000000F0FEF9FFF7BDFD00F0B2F9FFF7D6FF6A
:1089100002F0C9FA00F089FD06F0FCFCFFF7E6FC66
:1089200001B000BD00B581B0FFF7D3FD4FF0C80026
:10893000FFF7D2F8FFF7CEFF00F0DAFAFFF73DFEBF
:10894000FFF7B6FEFFF79EFFFFF7BEFFFFF73CFF06
:10895000FBF71FFDFBF7E8FD00F09CF901B000BD3F
:108960002DE9104181B04FF000044FF0000041F2BA
:10897000D838C2F2000888F800004FF0C800FFF7AE
:1089800087F8FFF7B3FF40F68418C2F20008D8F862
:10899000000045F2AA51C5F2AA5188423BD0FFF728
:1089A000CAFC012837D140F68418C2F20008D8F872
:1089B000000045F2AA51C5F2AA51884207D14FF0F2
:1089C000FF3040F68418C2F20008C8F800004FF0EB
:1089D000010041F27038C2F2000888F8000005E09A
:1089E00001F08CFF042801D14FF0010441F2D83886
:1089F000C2F2000898F800001428F1D94FF00000E6
:108A000041F27038C2F2000888F800001CB9FFF784
:108A100089FFFFF7A5FC40F68418C2F20008D8F8D9
:108A2000000045F2AA51C5F2AA51884207D14FF081
:108A3000FF3040F68418C2F20008C8F8000000F0C9
:108A40004BFCFCE72DE9004182B04FF000000090A4
:108A50004FF00000019001A9684600F03CF9009831
:108A600041F27838C2F20008C8F8000041F27838C4
:108A7000C2F20008D8F8000041F27838C2F20008CB
:108A8000D8F800100968016041F27838C2F2000895
:108A9000D8F8000041F27838C2F20008D8F8001087
:108AA0004968416041F27838C2F20008D8F8000005
:108AB00041F27838C2F20008D8F800108968816065
:108AC00041F27838C2F20008D8F8000041F2783854
:108AD000C2F20008D8F80010C968C16002B0BDE851
:108AE00000812DE9104181B0044672B641F2783818
:108AF000C2F20008D8F80000026841F28031C2F2E8
:108B0000000120469047044662B6204601B0BDE809
:108B100010812DE9F04585B004464FF00005174659
:108B200002F00F0010B14FF0010553E04FEA1110B1
:108B30004FEA0010064601F00F0A72B6AEB141F2DC
:108B40007838C2F20008D8F80000D0F808C041F226
:108B50008038C2F20008D8F8043022463146384640
:108B6000E047012801D14FF0010595BB07EB06074F
:108B7000BAF1000F2DD04FF00000504509D26946E0
:108B800000EB010100EB060202EB040212780A700E
:108B900005E0694600EB01014FF0FF020A7000F1A9
:108BA00001001028E9D341F27838C2F20008D8F861
:108BB0000000846841F28038C2F20008D8F804301E
:108BC0006A4638464FF01001A047012801D14FF006
:108BD000010562B6284605B0BDE8F0854FF00002F9
:108BE000002811D3B0F5001F0ED201EB0003A3F152
:108BF0000103002B08D301EB0003A3F10103B3F53C
:108C0000001F01D24FF00102B0F1807F12D3B0F10A
:108C1000817F0FD201EB0003A3F10103B3F1807F49
:108C200008D301EB0003A3F10103B3F1817F01D26B
:108C30004FF00102B0F1007F18D347F6FF73C0F286
:108C40000023984212D801EB0003A3F10103B3F112
:108C5000007F0BD301EB0000A0F1010047F6FF718C
:108C6000C0F20021884201D84FF00102104670473F
:108C70004DF8048D4FF0000040F20008C4F20208E5
:108C8000D8F8001011F0010F01D04FF001005DF88D
:108C9000048B70472DE9104181B0EFF3108004463A
:108CA00004B972B64BF2D610CAF2C40042F21408EC
:108CB000C4F20508C8F8000040F67B40C1F60D601C
:108CC00042F21408C4F20508C8F8000004B962B6FC
:108CD00001B0BDE810814DF8048D4FF6B868C0F2C0
:108CE0000108D8F8002002604FF6B868C0F2010809
:108CF000D8F8040008604FF001005DF8048B70475D
:108D00002DE9304192B04FF000044FF0000504AA65
:108D10004FF6C065C0F201050BCD0BC20BCD0BC2E7
:108D20000BCD0BC20BCD0BC295E8030082E803000C
:108D30004FF03000FEF78AFE4FF03000FEF7A8FE3D
:108D400040F60408C2F20008B8F8000040F2011131
:108D500088420CD140F60608C2F20008B8F80000BC
:108D60004FF6FE61884202D14FF4DE6518E040F60E
:108D70000408C2F20008B8F8000040F2022188425C
:108D80000CD140F60608C2F20008B8F800004FF611
:108D9000FD51884202D140F2F16501E04FF4DE65F9
:108DA00004A94FF00100F9F78EFA10B14FF0010459
:108DB0009AE02B464FF000024FF000014FF0010007
:108DC000F9F7AFFF012801D14FF0010440F2DF7342
:108DD0004FF000024FF002014FF00100F9F7A1FF40
:108DE000012801D14FF001044FF001014FF00100C3
:108DF000F9F78CFE40F2FF734FF000024FF00001D4
:108E00004FF00100F9F7B4FE40F2FF734FF0020299
:108E10004FF000014FF00100F9F7AAFE48F62D725D
:108E2000C0F201024FF000014FF00100FAF794F890
:108E30004FF0000002904FF0000001904FF0000052
:108E400000904FF000034FF001024FF010014FF07F
:108E50000100FAF7A2F84FF0000002904FF0000076
:108E600001904FF0000000904FF000034FF000021F
:108E70004FF00A014FF00100FAF78FF84FF00000B1
:108E800002904FF0000001904FF0000000904FF072
:108E900000034FF000024FF00B014FF00100FAF712
:108EA0007CF84FF000024FF000014FF00100FAF79C
:108EB00065FB012801D14FF001044FF000024FF093
:108EC00002014FF00100FAF759FB012801D14FF0E0
:108ED00001044CB94FF001014FF04B00FDF74CF885
:108EE0004FF04B00FDF705F8204612B0BDE8308189
:108EF00000B581B04FF00100F9F7AAFB4FF0000177
:108F00004FF04B00FDF738F84FF04B00FDF705F838
:108F10004FF04B00FDF71CF84FF03000FEF796FDC8
:108F20004FF03000FEF7D8FD01B000BD2DE9004143
:108F300084B008B1022809D141F28C32C2F2000299
:108F400001464FF00100F9F71FFF0028684600F0C6
:108F50002AF841F27038C2F2000898F8000098B17F
:108F60009DF8040002280FD101A800F1010000784B
:108F7000102809D101A800F102000078032803D1CC
:108F80004FF0040001F0C5FC684601F0D9F84FF03D
:108F9000010041F28838C2F2000888F8000004B0ED
:108FA000BDE80081FEE72DE9004141F28C38C2F2B4
:108FB000000898F84810016041F28C38C2F20008AD
:108FC000D8F80410C160026841F29431C2F2000185
:108FD00000F1040006F044FBBDE800812DE970417A
:108FE00085B004464FF002024FF000054FF0000636
:108FF0004FF6F860C0F2010002AB05881D8045887D
:109000005D8080889880082902D94FF0080000E030
:1090100008468DF8090040F60408C2F20008B8F8C6
:10902000000040F2011188420CD140F60608C2F25D
:109030000008B8F800004FF6FE61884202D14FF4F4
:10904000DF6518E040F60408C2F20008B8F8000036
:1090500040F2022188420CD140F60608C2F2000814
:10906000B8F800004FF6FD51884202D140F2F96590
:1090700001E04FF4DF654AF6AA260BE000942B4688
:1090800002AA4FF001014FF00100F9F703FE02467A
:10909000A6F10106022A01D1002EEFD1012A01D149
:1090A000FFF780FF05B0BDE870814DF8048D41F2F7
:1090B000DA31C2F20001088800F1010080B20880B4
:1090C00041F2DE31C2F20001088800F1010080B2F5
:1090D000088041F2DC31C2F20001088800F1010091
:1090E00080B208804FF0010041F2E238C2F200087D
:1090F00088F8000041F2D838C2F2000898F8000061
:10910000142809D841F2D831C2F20001087800F1E0
:109110000100C0B2087007E04FF0640041F2D83897
:10912000C2F2000888F8000041F2DA38C2F2000802
:10913000B8F8000000F0010038B94FF0010041F22A
:10914000E138C2F2000888F8000041F2DA38C2F2D1
:109150000008B8F800104FF0050091FBF0F000EBAC
:109160008000A1EB000038B94FF0010041F2E03877
:10917000C2F2000888F8000041F2DA38C2F20008B2
:10918000B8F8000000F101014FF00A0091FBF0F087
:109190004FF00A0808FB00F0A1EB000038B94FF0CF
:1091A000010041F2E338C2F2000888F8000041F201
:1091B000DA38C2F20008B8F8000000F102014FF0FE
:1091C000640091FBF0F04FF0640808FB00F0A1EBA5
:1091D000000038B94FF0010041F2E438C2F2000853
:1091E00088F8000041F2DA38C2F20008B8F800004E
:1091F000662807D34FF0000041F2DA38C2F20008C7
:10920000A8F8000041F2DE38C2F20008B8F8000009
:109210004FF6FE71884207D34FF0000041F2DE386E
:10922000C2F20008A8F8000041F2DC38C2F20008DF
:10923000B8F800104FF4FA7091FBF0F04FF4FA78A0
:1092400008FB00F0A1EB000038B94FF0010041F23B
:10925000E538C2F2000888F8000041F2DC38C2F2BA
:109260000008B8F80000B0F5FA7F07D34FF000000F
:1092700041F2DC38C2F20008A8F800005DF8048B67
:1092800070474DF8048D41F2DE38C2F20008B8F89C
:1092900000005DF8048B70474DF8048D41F2DE3814
:1092A000C2F20008B8F80010B1F57E4F08D34FF0B5
:1092B000000041F2DE38C2F20008A8F8000008E021
:1092C00041F2DE32C2F20002118801EB000188B2E5
:1092D00010805DF8048B70472DE9004141F2E238BF
:1092E000C2F2000898F8000068B100F08FFD05F0A8
:1092F000EEFE05F0E3FC4FF0000041F2E238C2F26E
:10930000000888F8000041F2E138C2F2000898F83D
:10931000000038B14FF0000041F2E138C2F200081D
:1093200088F8000041F2E038C2F2000898F8000026
:1093300070B101F016FE08B101F0DBFB01F0ADFCED
:109340004FF0000041F2E038C2F2000888F8000057
:1093500041F2E338C2F2000898F8000098B14FF0EB
:10936000030002F085FB08B102F02DFB01F004FEC2
:1093700008B101F063FC4FF0000041F2E338C2F2A3
:10938000000888F8000041F2E438C2F2000898F8BA
:109390000000D8B104F009FA012805D14FF000000F
:1093A00004F0F8F903F0A8FD04F015FA012805D13E
:1093B0004FF0000004F004FA03F0CDFE4FF000007F
:1093C00041F2E438C2F2000888F8000041F2E538C2
:1093D000C2F2000898F8000048B106F09FF84FF07C
:1093E000000041F2E538C2F2000888F8000041F2BE
:1093F000DE38C2F20008B8F800004FF6FF7188426C
:1094000009D241F2DE31C2F20001088800F1010008
:1094100080B2088007E04FF0000041F2DE38C2F26F
:109420000008A8F80000BDE8008100B581B04FF049
:109430009400FEF72DFB4FF60070C0F20100FBF721
:10944000D7FD01B000BD00B583B001A94FF0010008
:10945000FDF7A3FB01984AF6CC21CAF6CC2188423D
:1094600002D14FF0010001E04FF0000003B000BD59
:1094700000B581B04FF0000001464FF00100FDF74C
:1094800079FB012802D14FF0010001E04FF000000C
:1094900001B000BD2DE9F00140F20002C1F6FE72FC
:1094A0006FF060454FF0005340F2FF76C2F20006C5
:1094B00040F68414C2F2000440F68F17C2F200078F
:1094C00040F69010C2F200004FF6FF71C2F20101A7
:1094D00005E04FF0000CC2F800C002F10402AA42FD
:1094E000F7D304E04FF000021A6003F10403B34223
:1094F000F8D34EF20808C4F20708D8F8002012F496
:10950000806F0DD104E04FF00002226004F10404EA
:10951000BC42F8D304E04FF00002026000F1040006
:109520008842F8D3BDE8F00170474DF8048D032858
:1095300022D238B94FF47A7141F2EC38C2F2000805
:10954000C8F80010012808D141F2EC31C2F2000144
:1095500001F104014FF47A720A6002280CD141F241
:10956000EC30C2F2000000F1080041F2E838C2F22B
:10957000000898F8001001605DF8048B70474DF802
:10958000048D032818D228B941F2EC38C2F2000841
:10959000C8F80010012806D141F2EC32C2F20002F4
:1095A00002F104021160022806D141F2EC30C2F24D
:1095B000000000F1080001605DF8048B704703288B
:1095C0000CD201464FEA8101084641F2EC31C2F269
:1095D000000100EB01004FF000010160704703281B
:1095E00002D34FF0000035E001464FEA810141F21D
:1095F000EC32C2F2000201EB0201096811B94FF02E
:10960000000027E001464FEA810141F2EC32C2F24C
:10961000000201EB0201096801290DD14FEA800027
:1096200041F2EC31C2F2000100EB01004FF0000109
:1096300001604FF0FF300DE04FEA800041F2EC3165
:10964000C2F2000100EB01010868A0F1010008600E
:109650004FF001007047032802D34FF0000026E0CE
:1096600001464FEA810141F2EC32C2F2000201EB05
:109670000201096800290DD94FEA800041F2EC315E
:10968000C2F2000100EB01004FF0000101604FF059
:1096900001000CE04FEA800041F2EC31C2F200011F
:1096A00000EB01004FF0000101604FF00000704737
:1096B0002DE9104181B04FF0000041F2FE38C2F2B6
:1096C000000888F800004FF0000041F2FD38C2F2B7
:1096D000000888F800004FF0000041F2FC38C2F2A8
:1096E000000888F800004FF0000041F2FB38C2F299
:1096F000000888F800004FF0000041F2FA38C2F28A
:10970000000888F800004FF0000041F2F938C2F27A
:10971000000888F800004FF0000041F2F838C2F26B
:10972000000888F800004FF000042046FFF747FFCC
:1097300004F10100C4B2032CF7D301B0BDE81081DD
:109740002DE9704181B0082907D8037803F00F0391
:109750009BB21C464FF0010304E000F101031C78AA
:109760004FF00203072C39D8C4B341F20048C2F2CB
:109770000008A8F800404FF000040EE041F2104548
:10978000C2F2000504EB050504EB030606EB000638
:1097900036782E7004F10104A4B2A1F10105AC42A7
:1097A000ECDBA1EB030080B241F20248C2F20008F8
:1097B000A8F8000041F20448C2F20008D8F80440BA
:1097C000134641F20048C2F20008B8F8001041F216
:1097D0001040C2F200004FF00002A04701B0BDE807
:1097E00070812DE93041027802F00F0292B24FEA07
:1097F000022292B2144600F10102127844EA0202F7
:1098000094B2082C02D24FF0FF3059E040F6FF72BC
:10981000944206D34FF0020000F0A9F96FF0010066
:109820004EE041F20048C2F20008A8F800404FF0B4
:1098300000020EE041F21043C2F2000302EB030308
:1098400002F1020505EB00052D781D7002F1010201
:1098500092B2A1F102039A42ECDBA1F1020080B2C4
:1098600041F20248C2F20008A8F800004FF00000E0
:1098700000F07DF94FF0000041F2F938C2F2000823
:1098800088F800004FF0010041F2FD38C2F20008F4
:1098900088F800004FF00000FFF747FE4FF000008F
:1098A00041F2F838C2F2000888F8000041F204489A
:1098B000C2F20008D8F80010204688474FF0010097
:1098C000BDE830812DE9F0410646A1F10100C0B2AA
:1098D0000546307800F00F00C0B207464FF0000494
:1098E0004FF00000FFF7B7FE002802DC4FF0FF301A
:1098F000B8E041F2F832C2F20002107800F1010043
:10990000C0B2107041F2F838C2F2000898F80000B6
:109910000F2807D94FF0000041F2F838C2F20008D2
:1099200088F8000041F2F838C2F2000898F8000008
:10993000B84217D041F20448C2F20008D8F80440F7
:1099400041F20248C2F20008B8F8001041F210409B
:10995000C2F200004FF001034FF00402A0476FF085
:1099600001007FE04FF0000016E041F20248C2F231
:109970000008B8F8001000EB010141F21042C2F2F9
:10998000000201EB020100F1010202EB0602127873
:109990000A7000F1010080B2A842E6D341F202420F
:1099A000C2F20002108800EB050080B2108041F284
:1099B0000248C2F20008B8F8000041F20048C2F2C2
:1099C0000008B8F8001088421FD34FF0000041F2A1
:1099D000FD38C2F2000888F8000041F20448C2F2E3
:1099E0000008D8F8044041F20048C2F20008B8F874
:1099F000001041F21040C2F200004FF001034FF09E
:109A00000002A0474FF000002CE0002C1CD941F2CE
:109A1000F932C2F20002107800F10100C0B21070F9
:109A200041F2F938C2F2000898F80000A0420BD3C6
:109A30004FF0000000F09BF84FF0000041F2F938C1
:109A4000C2F2000888F800004FF0010041F2FD3832
:109A5000C2F2000888F800004FF00000FFF765FD33
:109A60004FF00100BDE8F0812DE9704181B004465E
:109A70001546207800F00F00C0B206464FF00100F6
:109A8000FFF7E9FD002802DC4FF0FF306CE0022D0B
:109A900002D14FF0FF3067E04FF0000041F2FC3898
:109AA000C2F2000888F80000032E0BD341F20448EC
:109AB000C2F20008D8F808204FF0050090476FF078
:109AC000010051E0022E0BD141F20448C2F200081D
:109AD000D8F808204FF0080090476FF0020043E0EC
:109AE000012E0ED14FF0010041F2FC38C2F2000805
:109AF00088F800004FF00100FFF717FD4FF001005C
:109B000032E004F10100007842F21048C2F200088D
:109B100088F8000004F1020000787F280CD804F1D6
:109B20000200007800F10100C0B241F2E838C2F250
:109B3000000888F8000007E04FF07F0041F2E838A5
:109B4000C2F2000888F800004FF0000041F2FB3834
:109B5000C2F2000888F800004FF001014FF0020047
:109B6000FFF70DFD4FF0000001B0BDE870812DE959
:109B7000004182B04FF60C78C0F20108D8F800100E
:109B80004FF60C78C0F20108D8F804200091019239
:109B900000F00F0040F03000C0B28DF800006846C1
:109BA00000F101004FF000010170684600F1020071
:109BB0004FF00001017068464FF0080100F003FB10
:109BC00002B0BDE800812DE9704183B04FF61C78EA
:109BD000C0F20108D8F800204FF61C78C0F2010846
:109BE000D8F80430009201934FF00802C9B3082955
:109BF00037D2CBB203F00F03DBB28DF800304FF059
:109C000001044FF000030BE003EB04056E4605EB87
:109C1000060503EB000636782E7003F101039BB2B4
:109C20008B42F1D301EB040081B24FF000004FF6FC
:109C30001473C0F2010300EB03031B78994207D8A9
:109C40004FF61471C0F2010100EB0100027804E04C
:109C500000F1010080B20828E9D31146684600F0FF
:109C6000B2FA03B0BDE870812DE9004182B04FF631
:109C70002478C0F20108D8F800204FF62478C0F20A
:109C80000108D8F8043000920193082902D3B1F5F5
:109C9000805F02D34FF0000033E04FEA2122D2B2BE
:109CA00002F00F0242F01002D2B28DF800206A4694
:109CB00002F1010201F0FF01C9B211704FF0000280
:109CC000694601F1020102EB010102EB00031B787E
:109CD0000B7002F101018AB2062AF1D368464FF0F7
:109CE000080100F070FA4FF0010041F2FC38C2F2B6
:109CF000000888F800004FF00100FFF716FC4FF055
:109D0000060002B0BDE800812DE9104183B00C4689
:109D10004FF62C78C0F20108D8F800104FF62C78D6
:109D2000C0F20108D8F804300091019302F00F014D
:109D300041F02001C9B28DF800104FF000010BE096
:109D40006A4602F1010201EB020201EB00031B78FB
:109D5000137001F1010189B2A1420DD20729EFD39D
:109D60000AE0684600F1010001EB00004FF000023C
:109D7000027001F1010081B20729F2D368464FF069
:109D8000080100F020FA072C02D94FF0070000E08C
:109D9000204603B0BDE810812DE9104181B00C468A
:109DA000082C30D3B4F5805F2DD24FF000010CE0C9
:109DB00042F21842C2F2000201EB020201EB000380
:109DC0001B78137001F1010189B2A142F0D34FF069
:109DD000000141F2FA38C2F2000888F8001021466A
:109DE000FFF742FFC0B2014642F21448C2F2000837
:109DF000A8F80010A4EB010080B242F21248C2F2AF
:109E00000008A8F8000001B0BDE810812DE910415C
:109E100081B04FF00000FFF7E2FB002816DAFFF7F1
:109E200047FC41F20448C2F20008D8F8044041F26D
:109E30000248C2F20008B8F8001041F21040C2F225
:109E400000004FF001034FF00302A0474FF0010064
:109E5000FFF7C5FB00280ADAFFF72AFC41F20448A5
:109E6000C2F20008D8F808104FF0020088474FF0FF
:109E70000200FFF7B4FB002880F2878041F2FA313C
:109E8000C2F20001087800F10100C0B2087041F28E
:109E9000FA38C2F2000898F800000F2807D94FF0EE
:109EA000000041F2FA38C2F2000888F8000041F2DE
:109EB000FA38C2F2000898F8002042F21248C2F2C2
:109EC0000008B8F8001042F21448C2F20008B8F8CE
:109ED000000042F21843C2F2000300EB0300FFF758
:109EE00013FFC0B2014642F21442C2F200021088CF
:109EF00000EB010080B2108042F21242C2F2000276
:109F00001088A0EB010080B2108042F21248C2F229
:109F10000008B8F80000002835D942F21048C2F213
:109F2000000898F80000002828D941F2FB31C2F25D
:109F30000001087800F10100C0B2087041F2FB385E
:109F4000C2F2000898F8000042F21048C2F200087D
:109F500098F80010884204D24FF00200FFF7E5FAAB
:109F600013E04FF0010041F2FC38C2F2000888F81B
:109F700000004FF00100FFF7D8FA06E04FF00200B2
:109F8000FFF7D3FA01E0FFF793FB01B0BDE81081C2
:109F90002DE9F0410D46164610B94FF0010401E0DD
:109FA0004FF0020428784FEA2010C0B20146013970
:109FB00006D33CD00239C0F0818000F09F80BDE024
:109FC00041F2FE38C2F2000898F80000022801D1E0
:109FD000012C08D041F2FE38C2F2000898F80000C7
:109FE000002840F0AB80FFF763FB41F2FE38C2F27D
:109FF000000898F80000022813D141F20448C2F288
:10A000000008D8F80470234641F20248C2F2000862
:10A01000B8F8001041F21040C2F200004FF0060202
:10A02000B847224631462846FFF78AFB86E041F2D0
:10A03000FE38C2F2000898F80000022807D041F26A
:10A04000FE38C2F2000898F80000002876D1FFF729
:10A050002FFB41F2FE38C2F2000898F800000228F7
:10A0600014D141F20448C2F20008D8F8044041F289
:10A070000248C2F20008B8F8001041F21040C2F2E3
:10A0800000004FF001034FF00602A047314628467A
:10A09000FFF7A7FB002808DD4FF0020041F2FE3871
:10A0A000C2F2000888F8000048E04FF0000041F2DA
:10A0B000FE38C2F2000888F800003FE041F2FE38A6
:10A0C000C2F2000898F80000022837D141F2FD38AA
:10A0D000C2F2000898F8000080B331462846FFF726
:10A0E000F1FB00282ADCFFF7E3FA4FF0000041F211
:10A0F000FE38C2F2000888F800001FE041F2FE3886
:10A10000C2F2000898F80000012817D141F2FC388B
:10A11000C2F2000898F8000080B122463146284675
:10A12000FFF7A2FC002809DAFFF7C2FA4FF000009F
:10A1300041F2FE38C2F2000888F80000BDE8F08164
:10A1400000B581B0C16840F2DF72914202D14FF098
:10A15000010301E04FF0000301780A4600F1040119
:10A160001846FFF715FF01B000BD2DE9004189B188
:10A17000B1F5805F0ED2072902D8FFF724FD09E070
:10A180004FF0010241F2FE38C2F2000888F80020C8
:10A19000FFF702FEBDE8008107B4009818B10198EE
:10A1A00008B1029810B94FF0FF300AE041F20442C2
:10A1B000C2F2000200A890E80B0082E80B004FF00A
:10A1C000000003B0704700B581B0FEF707FF01B093
:10A1D00000BD30B581B0044600F090FB05464FF05D
:10A1E000010000F096FB022D05D14FF001014FF068
:10A1F000030001F061FCE07900F14000C0B2E071C1
:10A2000004F1070000F102004FF00001017004F1B9
:10A21000070000F103004FF03201017004F1070064
:10A2200000F104004FF00101017004F1070000F19A
:10A2300005004FF0F40101704FF00600A0804FF0D0
:10A24000000001B030BD10B504464FF0040000F02E
:10A2500060FB4FF0000000F09AFEE07900F1400052
:10A26000C0B2E07104F1070000F102004FF00001FC
:10A27000017004F1070000F103004FF0320101709A
:10A2800004F1070000F104004FF00101017004F136
:10A29000070000F105004FF0F40101704FF00600D7
:10A2A000A0804FF0000010BD10B504464FF0010132
:10A2B0004FF0030001F000FC4FF00200A080E079B5
:10A2C00000F14000C0B2E0714FF0000010BD10B5C9
:10A2D00004464FF0000004F1070000F1030001F014
:10A2E00053FD38B9E17901F14001C9B2E1714FF094
:10A2F0000B01A18010BD10B504464FF0000004F121
:10A30000070000F1030001F050FD38B9E17901F1D7
:10A310004001C9B2E1714FF00E01A18010BD10B52E
:10A3200004464FF0000004F1070000F1030001F0C3
:10A330004DFD38B9E17901F14001C9B2E1714FF049
:10A340000501A18010BD10B504464FF0000004F1D6
:10A35000070000F1030001F045FD38B9E17901F192
:10A360004001C9B2E1714FF00F01A18010BD10B5DD
:10A3700004464FF0000004F1070000F1030001F073
:10A3800042FD38B9E17901F14001C9B2E1714FF004
:10A390000401A18010BD10B504464FF0000004F187
:10A3A000070000F1030001F0BBFD38B9E17901F1CC
:10A3B0004001C9B2E1714FF00601A18010BD4FF01C
:10A3C000000200F1070101F102010978032906D01A
:10A3D000022904D0012902D04FF0310207E04FF0EA
:10A3E00002018180C17901F14001C9B2C1711046F9
:10A3F00070474FF0000200F1070101F102010978F6
:10A40000032906D0022904D0012902D04FF03102DD
:10A4100007E04FF002018180C17901F14001C9B22A
:10A42000C1711046704710B504464FF0000000F0AF
:10A43000AEFDE07900F14000C0B2E0714FF00200E3
:10A44000A0804FF0000010BDC17901F14001C9B2F8
:10A45000C1714FF0020181804FF000007047C17957
:10A4600001F14001C9B2C1714FF0020181804FF08A
:10A47000000070474FF000014FF000010A464FEA1C
:10A480008203A3EB02024FEA820240F6AC13C2F24F
:10A49000000302EB03021278904204D001F10101A3
:10A4A000C9B20629EAD3062901D34FF0FF010846B5
:10A4B000704770B50E464FF0FF044FF0000506F1EF
:10A4C0000701002964D0FFF7D5FF044606F1070015
:10A4D00000F1010000784FEAE01000F00100C0B286
:10A4E0000146FF2C52D0012914D121464FEA8100A8
:10A4F000A0EB01014FEA8101084640F6AC11C2F21F
:10A50000000100EB0100007920B14FF0010000F0E4
:10A5100024FE03E04FF0000000F01FFE21464FEA4A
:10A520008100A0EB01014FEA8101084640F6AC1121
:10A53000C2F2000100EB01004088B188884202D9D4
:10A540004FF0130524E021464FEA8100A0EB010102
:10A550004FEA8101084640F6AC11C2F2000100EB5F
:10A5600001008068A0B121464FEA8100A0EB010103
:10A570004FEA8101084640F6AC11C2F2000100EB3F
:10A580000100816830468847054601E04FF011051B
:10A59000284670BD00B581B04FF0000100F1070200
:10A5A00042B18288022A05D3C27901461046FFF7DC
:10A5B00080FF0146084601B000BD10B44FF0000313
:10A5C0004FF000030AE01C464FEA041404EB0104B8
:10A5D0002468A04204D003F10103DBB29342F2D31A
:10A5E000934201D34FF0FF03184610BC70472DE98A
:10A5F000F04C81B08B4614464FF0FF054FF000073A
:10A600004FF000014FF00006BBF804A01A462146A7
:10A61000FFF7D3FF054600F071F9074600F084F913
:10A620000146FF2D0BD140F65420C2F200008442B7
:10A6300002D14FF0310653E04FF0120650E02846A9
:10A640004FEA001000EB0400C088504507D82846A8
:10A650004FEA001000EB04000089504502D24FF091
:10A6600013063DE028464FEA001000EB0400007995
:10A6700000EA0700B8B940F63420C2F20000844274
:10A6800002D14FF07E062BE040F61420C2F200000B
:10A69000844205D040F6F410C2F2000084421FD17B
:10A6A0004FF022061CE028464FEA001000EB0400A1
:10A6B0004079012804D1012902D04FF033060FE080
:10A6C00028464FEA001000EB0400C06840B128465D
:10A6D0004FEA001000EB0400C16858468847064660
:10A6E000304601B0BDE8F08C00B581B04FF00003FA
:10A6F0004FF0000100F107028AB100F1070101F1FA
:10A700000101097801F07F0340F63422C2F2000211
:10A71000014618464FF00203FFF769FF014608465D
:10A7200001B000BD00B581B04FF000034FF0000153
:10A7300000F107028AB100F1070101F10101097876
:10A7400001F07F0340F6B422C2F20002014618462F
:10A750004FF00203FFF74BFF0146084601B000BD72
:10A760004FF000014FF0000100F1070169B100F165
:10A77000070101F1010109784FEA012100F1070009
:10A7800000F10200007841EA00014FF03101084673
:10A79000704700B581B04FF000034FF0000100F1A9
:10A7A00007028AB100F1070101F10101097801F006
:10A7B0007F0340F61422C2F20002014618464FF011
:10A7C0000203FFF714FF0146084601B000BD00B5C3
:10A7D00081B04FF000034FF0000100F107028AB191
:10A7E00000F1070101F10101097801F07F0340F652
:10A7F000D422C2F20002014618464FF00103FFF7CF
:10A80000F6FE0146084601B000BD00B581B04FF02C
:10A8100000034FF0000100F107028AB100F10701C7
:10A8200001F10101097801F07F0340F6F412C2F250
:10A830000002014618464FF00203FFF7D8FE01461A
:10A84000084601B000BD0000000030B44FF0000425
:10A850004FF0000411E023464FEA830503EB0503A4
:10A860004FEA830303EB01031B88834202D14FF0BD
:10A87000000006E004F101039CB29442EBD34FF0D8
:10A88000010030BC7047884202D04FF0010001E067
:10A890004FF00000704700000000F0B581B00646A0
:10A8A0000D4617464FF000004FF0000400F03CF852
:10A8B00001464FF000001CE002464FEA820302EB23
:10A8C00003024FEA820202EB0502128896420DD182
:10A8D00089B94FEA800100EB01004FEA800000EBEC
:10A8E0000500C07838B14FF0010404E000F1010028
:10A8F000C0B2B842E0D3204601B0F0BD4DF8048D9F
:10A9000040F6E428C2F2000898F800005DF8048BD5
:10A9100070474DF8048D40F6E428C2F2000888F82C
:10A9200000005DF8048B70474DF8048D43F2284811
:10A93000C2F2000898F800005DF8048B70474DF8EB
:10A94000048D43F22848C2F2000888F800005DF840
:10A95000048B70474DF8048D43F22C48C2F2000876
:10A96000D8F800005DF8048B70474DF8048D43F271
:10A970002C48C2F20008C8F800005DF8048B70474C
:10A980004DF8048D43F23048C2F20008D8F80000B8
:10A990005DF8048B70474DF8048D43F23048C2F2E5
:10A9A0000008C8F800005DF8048B70474DF8048D6E
:10A9B00043F23448C2F2000898F800005DF8048BB6
:10A9C00070474DF8048D43F23448C2F2000888F80D
:10A9D00000005DF8048B70474DF8048D43F2384851
:10A9E000C2F20008D8F800005DF8048B70474DF8FB
:10A9F000048D43F23848C2F20008C8F800005DF840
:10AA0000048B70474DF8048D43F23C48C2F20008B5
:10AA100098F800005DF8048B70474DF8048D43F200
:10AA20003C48C2F2000888F800005DF8048B7047CB
:10AA30004DF8048D43F23D48C2F2000898F800003A
:10AA40005DF8048B70474DF8048D43F23D48C2F227
:10AA5000000888F800005DF8048B70474DF8048DFD
:10AA600040F6E528C2F2000898F800005DF8048B73
:10AA700070474DF8048D40F6E528C2F2000888F8CA
:10AA800000005DF8048B70474DF8048D43F23E489A
:10AA9000C2F2000898F800005DF8048B70474DF88A
:10AAA000048D43F23E48C2F2000888F800005DF8C9
:10AAB000048B70474DF8048D43F24048C2F2000801
:10AAC000B8F800005DF8048B70474DF8048D43F230
:10AAD0004048C2F20008A8F800005DF8048B7047F7
:10AAE0004FF000028088884201D24FF013021046D6
:10AAF00070472DE9F0414FF00C074FF000044FF084
:10AB0000000543F24846C2F200064FF0000474E02C
:10AB100020464FEA8001A1EB00004FEA800040F69A
:10AB2000E821C2F2000100EB01000078F1798842CF
:10AB300060D120464FEA8001A1EB00004FEA80007F
:10AB400040F6E821C2F2000100EB010041883046E6
:10AB5000FFF7C6FF054606F1070000F10100007887
:10AB60004FEAE01000F00100C0B2002D47D10128EB
:10AB700017D120464FEA8001A1EB00004FEA800088
:10AB800040F6E821C2F2000100EB0100007940B17B
:10AB90004FF0010043F24248C2F2000888F800007A
:10ABA00007E04FF0000043F24248C2F2000888F884
:10ABB000000020464FEA8001A1EB00004FEA800030
:10ABC00040F6E821C2F2000100EB01008068B0B15C
:10ABD00020464FEA8001A1EB00004FEA800040F6DA
:10ABE000E821C2F2000100EB01008168304688478D
:10ABF000054604E004F10100C4B2BC4288D3BC4263
:10AC000001D34FF0110555B943F24248C2F2000892
:10AC100098F80020B188304600F079FA03E0294620
:10AC2000304600F050FA4FF0000043F24348C2F2C1
:10AC3000000888F800002846BDE8F0812DE9304181
:10AC40004FF0000443F65845C2F200052846FFF7CE
:10AC5000A1FC0446112C03D0122C01D0312C01D1BF
:10AC60004FF0FF0454B943F24548C2F2000898F887
:10AC70000020A988284600F04AFA03E02146284629
:10AC800000F021FA4FF0000043F24448C2F20008FD
:10AC900088F800002046BDE8308100B581B043F25D
:10ACA0001840C2F2000000F0BAFD43F21840C2F2B0
:10ACB000000000F1040002F0DAFC43F21840C2F296
:10ACC000000000F1060003F0D2F843F21840C2F28F
:10ACD000000000F1080002F0FBFC43F21840C2F251
:10ACE000000000F10A0001F0ADFE43F21840C2F28C
:10ACF000000000F10C0002F01CFD01B000BD4DF899
:10AD0000048D4FF0000143F21848C2F20008A8F881
:10AD10000010A0F1020080B243F22648C2F20008FF
:10AD2000A8F800005DF8048B70472DE9F041054656
:10AD30000C4616461F464FF0000000F076F926B18B
:10AD40004FF0000000F023F962E0012F30D14FF006
:10AD5000000043F24848C2F20008C8F8000043F27D
:10AD60004848C2F20008A8F804404FF0010043F23E
:10AD70004848C2F2000888F806004FF000000CE0D6
:10AD800043F24F41C2F2000100EB010100EB05026A
:10AD900012780A7000F1010080B2A042F0D34FF0A7
:10ADA000010043F24348C2F2000888F800002FE097
:10ADB0004FF0000043F65848C2F20008C8F80000FF
:10ADC00043F65848C2F20008A8F804404FF00000CB
:10ADD00043F65848C2F2000888F806004FF0000019
:10ADE0000CE043F65F41C2F2000100EB010100EB11
:10ADF000050212780A7000F1010080B2A042F0D37F
:10AE00004FF0010043F24448C2F2000888F8000005
:10AE1000BDE8F08100B581B04FF0000000F0B7F858
:10AE200001B000BD2DE9004182B04FF050008DF817
:10AE30000000684600F101004FF002010170684611
:10AE400000F102004FF000010170684600F10300BC
:10AE50004FF032010170684600F104004FF001012B
:10AE60000170684600F105004FF0F401017040F6F2
:10AE70008418C2F20008D8F8000045F2AA51C5F2C1
:10AE8000AA5188420CD14FF00200FFF742FD4FF06B
:10AE9000000000F07CF868464FF00601FFF765F906
:10AEA00002B0BDE800812DE9004184B04FF0000000
:10AEB00043F24348C2F2000888F800004FF0000057
:10AEC00043F24448C2F2000888F800004FF0000046
:10AED00043F24248C2F2000888F800004FF0000038
:10AEE00043F24548C2F2000888F800004FF0000025
:10AEF00043F21848C2F20008A8F804004FF000001E
:10AF000043F21848C2F20008A8F806004FF000000B
:10AF100043F21848C2F20008A8F808004FF00000F9
:10AF200043F21848C2F20008A8F80A0001F0CBFB6F
:10AF3000FFF778FF4AF6FF40C0F2010001904AF6A1
:10AF40002B50C0F2010002904AF61560C0F20100D9
:10AF5000039001A890E80700FFF71EF904B0BDE8D0
:10AF600000814DF8048D43F24348C2F2000898F87E
:10AF700000005DF8048B70474DF8048D43F244489F
:10AF8000C2F2000898F800005DF8048B70474DF895
:10AF9000048D0146062945D80FF20408D8E801F0CF
:10AFA000040D161F28313A004FF47A7043F2184806
:10AFB000C2F20008A8F8000034E04FF0040043F2A9
:10AFC0001848C2F2000888F802002BE04FF0100089
:10AFD00043F21848C2F20008A8F8040022E04FF437
:10AFE000B47043F21848C2F20008A8F8060019E04D
:10AFF0004FF4B47043F21848C2F20008A8F80800F1
:10B0000010E04FF4FA6043F21848C2F20008A8F8C2
:10B010000A0007E04FF4B47043F21848C2F2000887
:10B02000A8F80C005DF8048B70474DF8048D0146BC
:10B03000062945D80FF20408D8E801F0040D161FC0
:10B0400028313A004FF0000043F21848C2F20008DD
:10B05000A8F8000034E04FF0000043F21848C2F2B4
:10B06000000888F802002BE04FF0000043F2184877
:10B07000C2F20008A8F8040022E04FF0000043F2FA
:10B080001848C2F20008A8F8060019E04FF00000C6
:10B0900043F21848C2F20008A8F8080010E04FF088
:10B0A000000043F21848C2F20008A8F80A0007E0BE
:10B0B0004FF0000043F21848C2F20008A8F80C0054
:10B0C0005DF8048B704730B581B004460D46782D8D
:10B0D00003D04FF00000FFF75AFFFF2D15D004F109
:10B0E000070000F10200057004F1070000F1010003
:10B0F000E17901704FF07F00E0714FF00300A08014
:10B10000A18804F10700FFF730F801B030BD70B539
:10B1100004460D4616464FF00000FFF738FF26B9EB
:10B12000294604F10700FFF720F870BD4DF8048DA3
:10B1300040F6E628C2F2000898F800005DF8048B9B
:10B1400070474DF8048D40F6E628C2F2000888F8F2
:10B1500000005DF8048B704700004DF8048D43F249
:10B160004548C2F2000888F800005DF8048B70477B
:10B1700099281CD84FF0000103464FF0010213E05C
:10B1800003F00F0002FB00F0C0B201EB0000C1B2FF
:10B190004FEA820002EB00024FEA4202D0B2C2B292
:10B1A0004FEA2310C0B20346002BE9D801E04FF06C
:10B1B000FF0108467047884202D04FF0010001E0CD
:10B1C0004FF0000070472DE9F04B84B083464FF0FC
:10B1D00002004FF000054FF000044FF000064FF062
:10B1E00000070BF1070000F1010000784FEA002092
:10B1F00080B206460BF1070000F10200007846EA33
:10B20000000086B24FF0000412E020464FEA8001B1
:10B2100000EB01004FEA80004FF63471C0F20101EB
:10B2200000EB01000088864204D004F10100C4B2A2
:10B23000022CEAD3022C6CD020464FEA800100EBAE
:10B2400001004FEA80004FF63471C0F2010100EBBB
:10B250000100D0F80C80D0F81090CDF80880CDF81F
:10B260000C9020464FEA800100EB01004FEA80007D
:10B270004FF63471C0F2010100EB0100B0F8048018
:10B28000ADF806804FF000004FF0000739E002985B
:10B2900007EB00000078133804D00F380CD01138B9
:10B2A00020D02BE0BDF80610BBF80400FFF783FFA9
:10B2B00020B34FF0130521E0FFF720FB21464FEAB2
:10B2C000810201EB02014FEA81014FF63472C0F2B4
:10B2D000010201EB0201897801EA000070B94FF028
:10B2E00022050BE04FF63471C0F2010130464FF0F9
:10B2F0000202FFF7D2FA08B14FF0330507F101005F
:10B30000C7B2039800F0FF00874204D2002DBED0E0
:10B3100001E04FF03105284604B0BDE8F08B70B570
:10B3200005464FF002004FF000004FF000044FF0D0
:10B33000000605F1070000F1010000784FEA002047
:10B3400080B2064605F1070000F10200007846EAE7
:10B35000000086B22846FFF736FFF0BB4FF000042E
:10B3600039E021464FEA810201EB02014FEA8101F7
:10B370004FF63472C0F2010201EB020109888E42DD
:10B3800026D120464FEA800100EB01004FEA800001
:10B390004FF63471C0F2010100EB0100816805F144
:10B3A000070000F10300884721464FEA810201EBC4
:10B3B00002014FEA81014FF63472C0F2010201EB43
:10B3C0000201C988A980E97901F14001C9B2E97196
:10B3D00004F10101CCB2022CC3D370BD70B584B0AE
:10B3E00004464FF000004FF0000001A900EB0101FE
:10B3F00000EB040212780A7000F10100C0B20A28C2
:10B40000F3D32078FFF7B4FE064604F1010000787C
:10B41000FFF7AEFE054604F102000078FFF7A8FE34
:10B42000632E05D80C2D03D815B11F2800D810B9EC
:10B430004FF0310007E001A94FF0020002F0EAFEF0
:10B4400008B14FF0720004B070BD70B582B0044610
:10B450004FF000004FF0000001A900EB010100EBEC
:10B46000040212780A7000F10100C0B20428F3D37C
:10B470002078FFF77DFE064604F101000078FFF713
:10B4800077FE054604F102000078FFF771FE632E97
:10B4900005D80C2D03D815B11F2800D810B94FF0CE
:10B4A000310007E001A94FF0020002F0DCFE08B114
:10B4B0004FF0720002B070BD2DE9F04B84B007462A
:10B4C0004FF001004FF000064FF0000407F10700B5
:10B4D00000F10100007800F07F00C0B283464FF019
:10B4E000000454E020464FEA800100EB01004FEADF
:10B4F00080004FF66471C0F2010100EB0100D0F84A
:10B500000C80D0F81090CDF80880CDF80C90204633
:10B510004FEA800100EB01004FEA80004FF66471B2
:10B52000C0F2010100EB0100B0F80480ADF8068024
:10B530004FF000054FF000051FE0029805EB0000FA
:10B54000007812380AD0013814D1BDF80610B88836
:10B55000FFF799F970B14FF013060BE04FF66471E5
:10B56000C0F2010158464FF00102FFF76EF908B131
:10B570004FF0120605F10100C5B2039800F0FF007C
:10B58000854201D2002ED8D004F10100C4B2002CB3
:10B59000A8D0304604B0BDE8F08B30B581B0044689
:10B5A0004FF000052046FFF787FF054604F107002E
:10B5B00000F10100007800F07F00C0B22DB9003822
:10B5C00003D14FF00000FFF7E2FC3DB9E07900F154
:10B5D0004000C0B2E0714FF00200A080284601B0E8
:10B5E00030BD2DE9F04B82B083464FF003004FF0A1
:10B5F00000054FF000044FF000064FF00007FFF782
:10B600007DF907460BF1070000F10100007800F01A
:10B610007F00C0B24FF0000412E021464FEA8102E1
:10B6200001EB02014FEA81014FF67C72C0F2010288
:10B6300001EB02010988884204D004F10101CCB277
:10B64000032CEAD3032C54D020464FEA800100EBB0
:10B6500001004FEA80004FF67C71C0F2010100EB5F
:10B660000100D0F80C80D0F81090CDF80080CDF813
:10B6700004904FF0000634E020464FEA800100EBD2
:10B6800001004FEA80004FF67C71C0F2010100EB2F
:10B6900001008188009806EB00000078133802D082
:10B6A0006B3808D01AE0BBF80400FFF7ECF8A8B13B
:10B6B0004FF0130512E020464FEA800100EB010035
:10B6C0004FEA80004FF67C71C0F2010100EB0100EF
:10B6D000807800EA070008B94FF07E0506F1010006
:10B6E000C6B2019800F0FF00864204D2002DC3D0FC
:10B6F00001E04FF01205284602B0BDE8F08B30B5EE
:10B7000081B004464FF000052046FFF76AFF05466A
:10B7100004F1070000F10100007800F07F00C0B2E2
:10B72000A5B9013812D303D0023806D30CD00DE0EE
:10B730004FF0000000F032F808E000F050F84FF051
:10B74000010000F085F801E000F059F81DBBE07938
:10B7500000F14000C0B2E07104F1070000F1020006
:10B760004FF00001017004F1070000F103004FF0F9
:10B770003201017004F1070000F104004FF00101F3
:10B78000017004F1070000F105004FF0F4010170B1
:10B790004FF00600A080284601B030BD30B581B022
:10B7A0000546FFF7ABF804464FF00100FFF7B1F88C
:10B7B0004FF0000000F0F9FF012D06D14FF001011C
:10B7C0004FF0030000F078F907E0022C05D14FF0AC
:10B7D00001014FF0030000F06FF901B030BD00B57A
:10B7E00081B04FF00200FFF794F84FF00000FFF730
:10B7F000CEFB4FF0000000F0D8FF01B000BD00B557
:10B8000081B04FF00400FFF784F84FF00000FFF71D
:10B81000BEFB4FF0000000F0C8FF01B000BD00B556
:10B8200081B0018891B10188A1F1010189B2018043
:10B83000008858B9FFF762F8012807D04FF00100DF
:10B84000FFF7ACFF4FF0000000F0AFFF01B000BD0C
:10B850004DF8048D44F26848C2F2000888F80000F0
:10B860005DF8048B70472DE9F04B84B083464FF0B0
:10B8700002004FF000054FF000040BF1070000F14B
:10B880000100007800F07F00C0B207464FF00004CE
:10B8900092E020464FEA800100EB01004FEA800071
:10B8A0004FF6C071C0F2010100EB0100D0F80C802E
:10B8B000D0F81090CDF80880CDF80C9020464FEAD3
:10B8C000800100EB01004FEA80004FF6C071C0F22A
:10B8D000010100EB0100B0F80480ADF806804FF0E4
:10B8E000000620464FEA800100EB01004FEA80008D
:10B8F0004FF6C071C0F2010100EB010000788DF835
:10B9000005004FF000064DE0029806EB00000078BD
:10B91000123810D0013804D00F3819D0113832D075
:10B920003DE0BDF80610BBF80400FEF7ACFFB0B375
:10B930004FF0130533E04FF6C071C0F201013846F5
:10B940004FF00202FEF781FF48B34FF0120526E0E8
:10B950009DF80580B84516D14FF00000FEF7CEFFE8
:10B9600021464FEA810201EB02014FEA81014FF6C5
:10B97000C072C0F2010201EB0201897801EA000005
:10B9800008B94FF022054FF6C071C0F201013846E8
:10B990004FF00202FEF781FF08B14FF0330506F1C8
:10B9A0000100C6B2039800F0FF00864201D2002DCC
:10B9B000AAD004F10100C4B2022CFFF46AAF2846F9
:10B9C00004B0BDE8F08B2DE900414FF0000044F2D7
:10B9D0006948C2F2000888F802004FF0FF3040F6D4
:10B9E0008418C2F20008C8F80000F9F7DBFABDE8D5
:10B9F00000812DE9304104464FF0000004F10700BA
:10BA000000F10100007800F07F00C0B2054620463A
:10BA1000FFF729FF08BB294601391ED303D002399D
:10BA20000AD312D019E04FF0010144F26948C2F282
:10BA3000000888F8021010E04FF0010144F2694854
:10BA4000C2F2000888F8011007E04FF0010144F24B
:10BA50006948C2F2000888F8021038B94FF00201B4
:10BA6000A180E17901F14001C9B2E171BDE8308105
:10BA70004DF8048D4FF000010246013A18D303D06F
:10BA8000023A08D30ED013E044F26948C2F200082B
:10BA900098F800100CE044F26948C2F2000898F8E7
:10BAA000011005E044F26948C2F2000898F802105B
:10BAB00008465DF8048B70474DF8048D0246013A44
:10BAC00018D303D0023A08D30ED013E044F26948E9
:10BAD000C2F2000888F800100CE044F26948C2F293
:10BAE000000888F8011005E044F26948C2F2000835
:10BAF00088F802105DF8048B70474FEA002101F0CE
:10BB0000FF214FEA102000F0FF1040EA01004FEA49
:10BB100030407047884202D04FF0010001E04FF002
:10BB200000007047F0B581B005460C4616464FF050
:10BB30000000FEF7E3FE02464FF000014FF0000068
:10BB40001EE003464FEA830703EB07034FEA830334
:10BB500003EB04031B889D420FD103464FEA830584
:10BB600003EB05034FEA830303EB04039B7803EA2B
:10BB700002023AB94FF0010104E000F10100C0B245
:10BB8000B042DED3B04201D14FF00101084601B00E
:10BB9000F0BD2DE9F04B82B007464FF00A004FF0A0
:10BBA00000044FF000004FF000054FF0000607F1D1
:10BBB000070000F1010000784FEA002080B205463E
:10BBC00007F1070000F10200007845EA000085B2A5
:10BBD0004FF0000012E001464FEA810201EB020142
:10BBE0004FEA81014FF6EC72C0F2010201EB020153
:10BBF00009888D4204D000F10100C0B20A28EAD3BE
:10BC00000A285CD001464FEA810201EB02014FEAAB
:10BC100081014FF6EC72C0F2010201EB0201D1F892
:10BC20000C80D1F81090CDF80080CDF804904FEA48
:10BC3000800100EB01004FEA80004FF6EC71C0F28A
:10BC4000010100EB0100B0F804B04FF000062EE057
:10BC5000009806EB00000078133804D00F380AD0A3
:10BC6000113815D020E05946B888FFF753FFD8B1F6
:10BC70004FF0130418E04FF6EC71C0F201012846B2
:10BC80004FF00A02FFF74EFF70B14FF022040BE0B5
:10BC90004FF6EC71C0F2010128464FF00A02FEF7A0
:10BCA000FCFD08B14FF0330406F10100C6B2019863
:10BCB00000F0FF00864204D2002CC9D001E04FF012
:10BCC0003104204602B0BDE8F08B70B505464FF058
:10BCD0000A004FF000004FF000044FF0000605F19D
:10BCE000070000F1010000784FEA002080B206460C
:10BCF00005F1070000F10200007846EA000086B274
:10BD00002846FFF746FFF0BB4FF0000439E021461C
:10BD10004FEA810201EB02014FEA81014FF6EC721A
:10BD2000C0F2010201EB020109888E4226D12046B1
:10BD30004FEA800100EB01004FEA80004FF6EC7102
:10BD4000C0F2010100EB0100816805F1070000F17C
:10BD50000300884721464FEA810201EB02014FEAC6
:10BD600081014FF6EC72C0F2010201EB0201C988B9
:10BD7000A980E97901F14001C9B2E97104F1010139
:10BD8000CCB20A2CC3D370BD00B581B001464FF0D0
:10BD9000000000F0F3F8014611B94FF0000101E096
:10BDA0004FF02201084601B000BD00B581B0014648
:10BDB0004FF0010000F0E2F8014611B94FF0000128
:10BDC00001E04FF02201084601B000BD00B581B08E
:10BDD00001464FF0020000F0D1F84FF00001084694
:10BDE00001B000BD00B581B001464FF0030000F086
:10BDF000C5F8014611B94FF0000101E04FF02201F2
:10BE0000084601B000BD2DE9004140F60408C2F229
:10BE10000008B8F8001040F2022291420FD140F61B
:10BE20000608C2F20008B8F800104FF6FD52914221
:10BE300005D101464FF0050000F0A0F804E00146EE
:10BE40004FF0040000F09AF84FF00000BDE80081C8
:10BE50002DE93041044643F6F478C0F20208D8F8E0
:10BE600000104FF000050846FFF747FE01464FEA75
:10BE7000116000F0FF00C0B2207004F101004FEA31
:10BE8000114202F0FF02D2B2027004F102004FEA46
:10BE9000112202F0FF02D2B2027004F1030001F09D
:10BEA000FF01C9B201702846BDE8308110B50446D3
:10BEB00021464FF0040002F0B1FA01464FF00000B5
:10BEC00000EB04024FF0FF03137000F10100C0B259
:10BED0001828F5D311B94FF0000001E04FF022000F
:10BEE00010BD00B581B001464FF0020002F096FA95
:10BEF000014611B94FF0000101E04FF02201084660
:10BF000001B000BD10B50446FEF7F8FC0146042957
:10BF100001D14FF003014FF000022170104610BD17
:10BF20002DE93041044643F6EF78C0F20208D8F814
:10BF300000104FF000050846FFF7DFFD01464FEA0D
:10BF4000116000F0FF00C0B2207004F101004FEA60
:10BF5000114202F0FF02D2B2027004F102004FEA75
:10BF6000112202F0FF02D2B2027004F1030001F0CC
:10BF7000FF01C9B201702846BDE8308130B44FF0EE
:10BF8000000216E002EB010403464FEA8305A5EB2D
:10BF900003034FEA830340F2E005C0F2020503EB1E
:10BFA00005035B6802EB03031B78237002F10102B7
:10BFB000D2B203464FEA8304A4EB03034FEA8303A0
:10BFC00040F2E004C0F2020403EB04031B7A9A423D
:10BFD000D8D34FF0000030BC70474FF0000209E0AA
:10BFE00003464FEA43034FEAD07000EB030002F12F
:10BFF000010212B28A42F3DB704730B581B00446C9
:10C0000020464FF00201FFF7E8FF80EA04052046D2
:10C010004FF00A01FFF7E1FF80EA050520464FF0E7
:10C020001201FFF7DAFF80EA050520464FF01801FC
:10C03000FFF7D3FF80EA050001B030BD30B581B015
:10C04000044620464FF00D01FFF7C7FF80EA0405C4
:10C0500020464FF01701FFF7C0FF80EA050001B04E
:10C0600030BD82B04FEA1061C9B28DF8041001A949
:10C0700001F101014FEA1042D2B20A7001A901F1A7
:10C0800002014FEA1022D2B20A7001A901F10301A4
:10C09000C0B208709DF8040040F24C21C0F20201C9
:10C0A00000EB010000784FEA0060014601A800F1B2
:10C0B0000100007840F24C22C0F2020200EB0200C4
:10C0C00000784FEA004000EB010101A800F10200F6
:10C0D000007840F24C22C0F2020200EB020000782D
:10C0E0004FEA002000EB010001A901F103010978EA
:10C0F00040F24C22C0F2020201EB0201097801EB8E
:10C10000000002B0704700B581B0012904D1FFF7EB
:10C11000A8FFFFF772FF03E0FFF7A3FFFFF78EFF13
:10C1200001B000BD10B44FF0000213464FEA830384
:10C1300003EB0104C2F103034FEA830303EB0003A3
:10C140001B68236002F1010212B2042AEDDB10BC6D
:10C1500070472DE9F04405460E464FF0000404F107
:10C1600004004FEAE07101F0030100EB010121F04E
:10C170000301A0EB01004FEA800000EB0507204619
:10C180004FEAE07101F0030100EB010121F003012E
:10C19000A0EB01004FEA800000EB050A04F101006A
:10C1A0004FEAE07101F0030100EB010121F003010E
:10C1B000A0EB01004FEA800000EB050104F1020052
:10C1C0004FEAE07202F0030200EB020222F00302E7
:10C1D000A0EB02004FEA800000EB05000068096850
:10C1E00080EA010004F103014FEAE17202F0030268
:10C1F00001EB020222F00302A1EB02014FEA8101EE
:10C2000001EB0501096881EA000120464FEA800040
:10C2100000EB0600006880EA01004FF00101FFF723
:10C2200072FFDAF8001080EA0100386004F10100C2
:10C2300004B2202C93DBBDE8F08430B581B0044615
:10C2400015462046FFF785FF29462046FFF76AFF7F
:10C2500001B030BD70B44FF0000213464FEA8303C3
:10C2600003EB010314464FEA840404EB0005144673
:10C270004FEA840440F23C26C0F2020604EB0604B6
:10C2800024682D6884EA05041C6002F10102042A76
:10C29000E3DB70BC70472DE9F04406460D464FF0D5
:10C2A000000404F104004FEAE07101F0030100EB27
:10C2B000010121F00301A0EB01004FEA800000EB37
:10C2C000050720464FEAE07101F0030100EB010190
:10C2D00021F00301A0EB01004FEA800000EB050A0A
:10C2E00004F101004FEAE07101F0030100EB0101EC
:10C2F00021F00301A0EB01004FEA800000EB0501F3
:10C3000004F102004FEAE07202F0030200EB0202C5
:10C3100022F00302A0EB02004FEA800000EB0500D0
:10C320000068096880EA010004F103014FEAE17244
:10C3300002F0030201EB020222F00302A1EB020170
:10C340004FEA810101EB0501096881EA00012046FD
:10C350004FEA800040F2BC12C0F2020200EB020081
:10C36000006880EA01004FF00201FFF7CCFEDAF826
:10C37000001080EA0100386020464FEA800000EBA0
:10C38000060004F104014FEAE17202F0030201EB3E
:10C39000020222F00302A1EB02014FEA810101EB4C
:10C3A00005010968016004F1010004B2202CFFF6C8
:10C3B00078AFBDE8F08430B581B00C461546214613
:10C3C000FFF748FF21462846FFF765FF01B030BD63
:10C3D0002DE9004182B040F22818C0F20208D8F8D6
:10C3E0000010009140F22C18C0F20208D8F800109A
:10C3F0000191012806D169464FF0030001F00AFFC0
:10C40000014605E001A94FF0030001F003FF0146DA
:10C41000084602B0BDE800812DE9704183B00546B1
:10C4200044F27448C2F2000898F8000001281ED1B6
:10C430004FF0000401A804EB00004FF00001017070
:10C4400044F27040C2F2000004EB00004FF0000123
:10C45000017004F10100C4B2042CEBD34FF00100D1
:10C4600044F26C48C2F2000888F8000045E044F24B
:10C470006C48C2F2000898F8000018BB4FF00004A6
:10C4800044F27040C2F2000004EB000600F0DDF858
:10C49000307001A804EB000044F27041C2F20001C8
:10C4A00004EB01010978017004F10100C4B2042C0D
:10C4B000E6D34FF0010044F26C48C2F2000888F85D
:10C4C00000001AE04FF0000444F27040C2F2000095
:10C4D00004EB000600F0B9F8307001A804EB00008E
:10C4E00044F27041C2F2000104EB010109780170CD
:10C4F00004F10100C4B2042CE6D34FF00600A8807A
:10C50000E87900F14000C0B2E87101A905F1070027
:10C5100000F102004FF0040203F0A2F803B0BDE8FE
:10C5200070812DE9004182B044F27048C2F20008E7
:10C5300098F800108DF8041001A901F1010144F2EE
:10C540007042C2F2000202F1010212780A7001A9DF
:10C5500001F1020144F27042C2F2000202F1020251
:10C5600012780A7001A901F1030144F27042C2F28B
:10C57000000202F1030212780A70024601A84FF08D
:10C5800000034FF0040100F012FA02B0BDE8008190
:10C590002DE9104185B004464FF0000044F26C488C
:10C5A000C2F2000888F800006846FFF7BAFF02A947
:10C5B000684600F06AF804F1070000F10200014645
:10C5C00001A84FF0040203F04BF803A901A800F002
:10C5D0005CF802980399884232D144F27548C2F25D
:10C5E000000898F8000040B144F27541C2F2000121
:10C5F0000878A0F10100C0B208704FF0000044F2CA
:10C600007648C2F2000888F800004FF00000FFF7FB
:10C61000DFFE4FF0010044F27448C2F2000888F8CF
:10C6200000004FF00100FEF78AF94FF00200A080F1
:10C63000E07900F14000C0B2E0714FF0000001E08D
:10C6400000F018FA05B0BDE8108110B54FF00000F9
:10C65000FCF717FE4FF6FF71884202D200F101008D
:10C6600080B202F0F3FF02F0DDFF01464FF0FF0061
:10C6700091FBF0F0C0EB0020A1EB0000C0B204463B
:10C680002046FCF709FE204610BDD8B1D1B14FF0CD
:10C69000000203784FEA036342EA030200F1010358
:10C6A0001B784FEA034342EA030200F102031B78BE
:10C6B0004FEA032342EA030200F10300007842EA52
:10C6C00000020A6070472DE9004182B04FF000007F
:10C6D00044F27041C2F2000100EB01014FF0000290
:10C6E0000A7000F10100C0B20428F1D34FF000003D
:10C6F00044F26C48C2F2000888F800004FF00000D5
:10C7000044F27848C2F2000888F800004FF00000B8
:10C7100044F27448C2F2000888F8000001A94FF002
:10C72000030001F07BFE40B99DF8040044F2764816
:10C73000C2F2000888F8000007E04FF0000044F261
:10C740007648C2F2000888F8000044F27648C2F247
:10C75000000898F80000012814D14FF0030044F2BB
:10C760007548C2F2000888F800004FF0010044F25A
:10C770007748C2F2000888F800004FF00500FEF785
:10C7800006FC0FE04FF0000044F27748C2F20008C8
:10C7900088F800004FF0000044F27548C2F200082B
:10C7A00088F8000002B0BDE800814DF8048D44F225
:10C7B0007448C2F2000888F800005DF8048B7047E6
:10C7C0002DE9F04B84B083464FF004004FF0000594
:10C7D0004FF000040BF1070000F1010007784FF063
:10C7E000000412E020464FEA800100EB01004FEA0E
:10C7F000800040F23011C0F2020100EB010000881D
:10C80000874204D004F10100C4B2042CEAD3042C02
:10C8100000F08C8020464FEA800100EB01004FEAD7
:10C82000800040F23011C0F2020100EB0100D0F8AC
:10C830000C80D0F81090CDF80880CDF80C902046F0
:10C840004FEA800100EB01004FEA800040F2301116
:10C85000C0F2020100EB0100B0F80480ADF80680E0
:10C860004FF0000620464FEA800100EB01004FEA3E
:10C87000800040F23011C0F2020100EB01000078AC
:10C880008DF805004FF0000648E0029806EB000026
:10C890000078133806D00F380ED0023828D013385D
:10C8A00030D038E0BDF80610BBF80400FDF7EBFF10
:10C8B00088B34FF013052EE09DF80580B8452AD1C6
:10C8C0004FF00000FEF71AF821464FEA810201EB13
:10C8D00002014FEA810140F23012C0F2020201EB84
:10C8E0000201897801EA0000A8B94FF0220512E0A0
:10C8F00044F26C48C2F2000898F8000058B94FF0B2
:10C90000240508E044F27748C2F2000898F80000D5
:10C9100008B14FF0370506F10100C6B2039800F0E8
:10C92000FF00864204D2002DAFD001E04FF0120587
:10C93000284604B0BDE8F08B2DE9704181B0044673
:10C940004FF0000504F1070000F1010006782046D1
:10C95000FFF736FF054635BB3046013823D305D0F7
:10C96000023807D302D0013811D01CE02046FFF76F
:10C9700053FD18E04FF0010044F27848C2F200087D
